:10000000F4FB022099010000F54B0100AD4B01000B
:10001000AD4B0100AD4B0100AD4B0100AD4B0100FC
:10002000AD4B0100AD4B0100AD4B0100F54B0100A4
:10003000F54B0100AD4B0100DD6601002D690100AB
:10004000F54B0100F54B0100F54B0100F54B0100AC
:10005000F54B0100F54B0100F54B0100F54B01009C
:10006000F54B0100F54B0100F54B0100F54B01008C
:10007000F54B0100F54B0100F54B0100F54B01007C
:10008000F54B0100F54B0100F54B0100F54B01006C
:10009000F54B0100F54B0100F54B0100F54B01005C
:1000A000B5450100C9450100E546010009480100C8
:1000B000F54B0100F54B0100F54B0100CD6A010045
:1000C000F54B0100E96C0100F54B0100056F0100E3
:1000D000F54B010005700100F54B01008D45010055
:1000E000F54B0100F54B0100F54B01007145010096
:1000F000F54B0100F54B0100F54B0100F54B0100FC
:10010000F54B0100F54B0100F54B0100F54B0100EB
:10011000F54B010075580100F54B0100F54B01004E
:10012000F54B0100F54B0100F54B0100F54B0100CB
:10013000F54B0100F54B0100F54B0100F54B0100BB
:10014000F54B0100F54B010005710100F54B010075
:1001500005720100F54B0100F54B0100F54B010064
:10016000F54B0100A1450100DD450100F54B010003
:10017000F54B0100F54B0100F54B0100F54B01007B
:10018000F54B0100FD450100F54B0100F54B010069
:10019000F54B0100F54B01005B4B4CF220524DF644
:1001A000281010B51A80188000BF00BF574C14F0FB
:1001B00025FD4FF030612160554B564A5649A360EA
:1001C0004FF47000E260554C0860236813F48072AD
:1001D00004D153484FF4A85102602160514C237858
:1001E000190704D594F800C04CF0080222704E495B
:1001F0004E4C4F4B2A2008704E498B4204D254F883
:10020000040F43F8040BF8E74B4A4C4800248242A1
:1002100002D242F8044BFAE7494B4A4A002452F80A
:10022000240043F824000134662CF8D1464C474999
:100230004FF0800E04F801EB8C42FBD1444C454B4F
:100240003F4A1A60A4F5805C8A202421A0222070F5
:100250008CF801108CF800209CF806309A07FBD52A
:100260009CF80600C406FBD43B4CA1793A4B01F044
:100270000C02082AF9D10320462418715C7199797F
:100280008806FCD5344A9079334B4106FBD5334A76
:100290004FF08274092120201460516018709C79FD
:1002A00004F00C020C2AFAD12D4B2E4C2E49196069
:1002B0002E482F4B206000220721626044F8041C66
:1002C000C4F80C3D62B614F057FD15480468E20707
:1002D00005D5284814F03EFD2749284A0A60284BD6
:1002E0001878430609D5244C244922688A4204D14F
:1002F000204814F02FFD0023236017F08BFB14F02F
:1003000083FC14F0B1FBFEE70E2005403080044072
:10031000823F04000100002B88ED00E010D0034074
:1003200014D0034002D0074000E007405CD3010036
:10033000F806FF1FD068FF1FD068FF1F5CAF0220C8
:100340000002FF1F0000000000E400E056E400E0AF
:100350000050064008ED00E00040064044800440A4
:100360000480044014E000E0C0100500BFD4010088
:10037000000020206A79FB5F1CE00340A5C3945A6B
:1003800000F00740FFFFFFFFFFFFFFFFFFFFFFFF42
:10039000FFFFFFFFFFFFFFFFFFFFFFFFFFFFFFFF6D
:1003A000FFFFFFFFFFFFFFFFFFFFFFFFFFFFFFFF5D
:1003B000FFFFFFFFFFFFFFFFFFFFFFFFFFFFFFFF4D
:1003C000FFFFFFFFFFFFFFFFFFFFFFFFFFFFFFFF3D
:1003D000FFFFFFFFFFFFFFFFFFFFFFFFFFFFFFFF2D
:1003E000FFFFFFFFFFFFFFFFFFFFFFFFFFFFFFFF1D
:1003F000FFFFFFFFFFFFFFFFFFFFFFFFFFFFFFFF0D
:10040000FFFFFFFFFFFFFFFFFFFFFFFFDEF9FFFF23
:1004100010B5054C237833B9044B13B10448AFF33E
:1004200000800123237010BDD068FF1F0000000072
:1004300058D30100084B10B51BB108490848AFF369
:1004400000800848036803B910BD074B002BFBD0A0
:10045000BDE81040184700BF00000000D468FF1F2F
:1004600058D30100D068FF1F0000000030B40446DC
:100470000120D4F81C3304EBC3050344C4F81C3337
:10048000C5F8B410C5F8B82030BC7047704700BF3D
:10049000704700BF034B586810B101680A681047E5
:1004A000704700BFC0A90220034B986810B10168D3
:1004B0000A681047704700BFC0A90220034BD868E4
:1004C00010B101680A681047704700BFC0A9022038
:1004D000034B186910B101680A681047704700BFE4
:1004E000C0A90220034B586910B101680A6810477F
:1004F000704700BFC0A90220034B986910B1016882
:100500000A681047704700BFC0A90220034BD86992
:1005100010B101680A681047704700BFC0A90220E7
:10052000034B186A10B101680A681047704700BF92
:10053000C0A90220034B586A10B101680A6810472D
:10054000704700BFC0A90220034B986A10B1016830
:100550000A681047704700BFC0A90220034BD86A41
:1005600010B101680A681047704700BFC0A9022097
:10057000034B186B10B101680A681047704700BF41
:10058000C0A90220034B586B10B101680A681047DC
:10059000704700BFC0A90220034B986B10B10168DF
:1005A0000A681047704700BFC0A90220034BD86BF0
:1005B00010B101680A681047704700BFC0A9022047
:1005C000034B186C10B101680A681047704700BFF0
:1005D000C0A90220034B586C10B101680A6810478B
:1005E000704700BFC0A90220034B986C10B101688E
:1005F0000A681047704700BFC0A90220034BD86C9F
:1006000010B101680A681047704700BFC0A90220F6
:10061000034B186D10B101680A681047704700BF9E
:10062000C0A90220034B586D10B101680A68104739
:10063000704700BFC0A90220034B986D10B101683C
:100640000A681047704700BFC0A90220034BD86D4D
:1006500010B101680A681047704700BFC0A90220A6
:10066000034B186E10B101680A681047704700BF4D
:10067000C0A90220034B586E10B101680A681047E8
:10068000704700BFC0A90220034B986E10B10168EB
:100690000A681047704700BFC0A90220034BD86EFC
:1006A00010B101680A681047704700BFC0A9022056
:1006B000034B186F10B101680A681047704700BFFC
:1006C000C0A90220034B586F10B101680A68104797
:1006D000704700BFC0A90220034B986F10B101689A
:1006E0000A681047704700BFC0A90220034BD86FAB
:1006F00010B101680A681047704700BFC0A9022006
:10070000034BD3F8800010B101680A6810477047A6
:10071000C0A90220034BD3F8840010B101680A6815
:1007200010477047C0A90220034BD3F8880010B1CE
:1007300001680A6810477047C0A90220034BD3F82C
:100740008C0010B101680A6810477047C0A90220E8
:10075000034BD3F8900010B101680A681047704746
:10076000C0A90220034BD3F8940010B101680A68B5
:1007700010477047C0A90220034BD3F8980010B16E
:1007800001680A6810477047C0A90220034BD3F8DC
:100790009C0010B101680A6810477047C0A9022088
:1007A000034BD3F8A00010B101680A6810477047E6
:1007B000C0A90220034BD3F8A40010B101680A6855
:1007C00010477047C0A90220034BD3F8A80010B10E
:1007D00001680A6810477047C0A90220034BD3F88C
:1007E000AC0010B101680A6810477047C0A9022028
:1007F000034BD3F8B00010B101680A681047704786
:10080000C0A90220034BD3F8B40010B101680A68F4
:1008100010477047C0A90220034BD3F8B80010B1AD
:1008200001680A6810477047C0A90220034BD3F83B
:10083000BC0010B101680A6810477047C0A90220C7
:10084000034BD3F8C00010B101680A681047704725
:10085000C0A90220034BD3F8C40010B101680A6894
:1008600010477047C0A90220034BD3F8C80010B14D
:1008700001680A6810477047C0A90220034BD3F8EB
:10088000CC0010B101680A6810477047C0A9022067
:10089000034BD3F8D00010B101680A6810477047C5
:1008A000C0A90220034BD3F8D40010B101680A6834
:1008B00010477047C0A90220034BD3F8D80010B1ED
:1008C00001680A6810477047C0A90220034BD3F89B
:1008D000DC0010B101680A6810477047C0A9022007
:1008E000034BD3F8E00010B101680A681047704765
:1008F000C0A90220034BD3F8E40010B101680A68D4
:1009000010477047C0A90220034BD3F8E80010B18C
:1009100001680A6810477047C0A90220034BD3F84A
:10092000EC0010B101680A6810477047C0A90220A6
:10093000F8B50646044690F8587000252DE0042BC3
:1009400000F0C080022B00F0B1800834A0690135AE
:1009500040B1227F032A00F09D80042A00F08F809E
:10096000022A7CD0206A6A1C38B194F82430032B08
:1009700069D0042B5CD0022B4CD0A06AAA1C38B1E1
:1009800094F82C1003293AD004292DD0022917D02D
:100990000335082D04F1180425D0A0690028D4D00F
:1009A000237F032BCBD147FA05F1CB07CDD496F8A3
:1009B00058202A41D107C8D5036819688847C4E779
:1009C00047FA02FC5FEACC71E2D596F8583043FA58
:1009D00002F2D307DCD40368196888470335082D71
:1009E00004F11804D9D1F8BD96F85810794041FAAD
:1009F00002F3DB07CCD5036819688847EEE747FAAE
:100A000002F1C907C4D496F858C04CFA02F2D207D2
:100A1000BED5E0E747FA02F1C907AED596F858C04F
:100A20004CFA02F2D307A8D401680B689847A4E7F0
:100A300096F858307B4043FA02F1CB079DD5016808
:100A40000B68984799E747FA02FC5FEACC7194D4A7
:100A500096F8583043FA02F2D2078ED5E4E747FA07
:100A600005FC5FEACC727FF57DAF96F858302B41DC
:100A7000DB073FF577AF01680A68904772E796F8A1
:100A8000581079402941C9077FF56CAF01680A68A1
:100A9000904767E747FA05F2D2073FF563AF96F84C
:100AA00058302B41DB077FF55DAFE4E747FA05F1EE
:100AB000CA077FF54AAF96F858202A41D3073FF579
:100AC00044AF79E796F858307B402B41D9077FF542
:100AD0003CAF03681968884737E700BF30B48369C3
:100AE000164C027F93F858302568016982B0134193
:100AF000019503F00103019A81B14468551AA5429A
:100B000009D3A3B9826895424FF0010334BF002591
:100B100001254575037502B030BC7047002BFAD132
:100B200024680094009D056102B030BC704700212C
:100B300001610175417502B030BC704700AB022005
:100B4000F0B400F502340121D4F8D83284F8E4126C
:100B5000C3EB031300F503308B4000F5D072B3F5FF
:100B6000004FC4F8E0223BD3B3F5803F1AD3B3F56E
:100B7000003F44D3B3F5802F39D3B3F5002F46D3CC
:100B8000B3F5801F53D3B3F5001F48D3B3F5800FDF
:100B900055D32F4D2F4E072747F6FF732F70338005
:100BA0002F2005E02B4D2A4A5B082B80117029204D
:100BB000294A2A4F1168D4F8DC62294D294C01F0EA
:100BC00040010143002010603B60116013682E60FB
:100BD0004FF4006743F0400515602760F0BC704794
:100BE0001B491C4E00270F7033802820E0E7194D69
:100BF000174ADB0803212B8011702B20D8E7154EF4
:100C0000134F02209B08387033802A20D0E7114E02
:100C10000F4F04201B09387033802C20C8E70D4E7D
:100C20000B4F06209B09387033802E20C0E7094DFA
:100C3000074A5B0905212B8011702D20B8E7054D6F
:100C4000034ADB0907212B8011702F20B0E700BF7A
:100C5000B4A80220B6A802200090034008900340E8
:100C6000585CFF1F04E100E006490B6800F5023004
:100C7000002203F067030B60C0F8E02280F8E42252
:100C8000704700BF00900340012380F83031704767
:100C9000002380F830317047704700BF704700BFB5
:100CA000704700BFC368DA0706D55B1041688268E9
:100CB000C8588258C81810474168826801EB630021
:100CC000104700BFC368DA0706D55B104168826829
:100CD000C8588258C81810474168826801EB630001
:100CE000104700BFC368DA0706D55B104168826809
:100CF000C8588258C81810474168826801EB6300E1
:100D0000104700BFC9B2007914F03ABC4368074AE3
:100D1000D8B211F0FF0F52F830304FF0010014BF7D
:100D200083F8800083F80001704700BF34CE0100D3
:100D300010B50121044690F8200014F021FC04F1C4
:100D40001C000121FFF7E2FF10BD00BF38B50446CB
:100D5000002300F10C05C0F82833284613F08EFB61
:100D6000D4F8280304EBC001284691F82C13BDE801
:100D7000384013F09DBB00BFF8B5002490F85C73B9
:100D8000C0F82843064600F54F752B6847FA04F172
:100D900028469A6801F0010101349047042C05F1BE
:100DA0000805F2D10C36304613F068FB304642217C
:100DB000BDE8F84013F07CBBF8B5D0F82833C16C1F
:100DC00000EBC30201330F2B0646C8BF002306EB1E
:100DD000C307D2F860030C6897F85C73048006F5CB
:100DE0004F75C6F8283300242B6847FA04FC2846C0
:100DF0009A680CF0010101349047042C05F10805B4
:100E0000F2D106F10C004221BDE8F84013F050BBCE
:100E1000D0F82833C16C00EBC3020133012BC8BFEB
:100E20000023D2F830230968118000EBC30CC0F80E
:100E300028339CF82C130C3013F03ABB08B500791A
:100E400014F090FB08BD00BF2DE9F047294B82B09C
:100E500019680191019CC4F30805B5F5807F40F63F
:100E6000FF769146804698BF0026151F002415275F
:100E7000D8F80C006F6000EB84023146107914F052
:100E800099F8D8F80C10AF6004F1010A01EB8A0C54
:100E900031469CF8040014F08DF8D8F80C30EF605F
:100EA00003EB8A003146007A14F084F8D8F80C205D
:100EB0002F6102EB840A31469AF8100014F07AF898
:100EC000D8F80C1045F8147F01EB840C31469CF8DF
:100ED0001400053414F06EF80F2C4FF01503C7D131
:100EE0001326C9F84430C9F84060C9F83C6002B024
:100EF000BDE8F08700AB022038B5427B8368951EC1
:100F0000012DD9789C7900D938BD5FFA81FC5FEA60
:100F1000CC652BD45FEA4C622ED4E2B212F0500FB3
:100F2000044612D0987940F050019971A568AB79C8
:100F300003F0DF02AA71A0680221C17025690DB11A
:100F4000606DA8470222A3686273606D3F2804D8D1
:100F5000411C616520441D79057593F806C04CF06D
:100F600050029A71A4680223E37038BD1021D97031
:100F70005FEA4C611CD5836800254565856593F85B
:100F800006C04CF020029A718468C023A370816867
:100F90000D796A0880F85C208C7944F050038B71DD
:100FA00081684225CD70826803249279447338BDEC
:100FB000816891F806C04CF050038B71806802255F
:100FC000C57038BD90F8643063B310B48268274CA4
:100FD00092F802C026490CF0FE039370026E13795A
:100FE0002370046E22790A70816891F803C05FEA69
:100FF0000C63FAD5046E1F4B22791A7081680224A3
:10100000CC70826892F802C00CF0C70393708368BA
:1010100042F21071DC78A40605D400225DF8044B7E
:1010200080F864207047DA789206F6D5DC78A4065A
:10103000F3D593F803C05FEA8C62EED5DA789406B4
:10104000EBD5DC78A206E8D593F803C05FEA8C64A0
:10105000E3D5DA789206E0D50839DBD19970836858
:101060008021997000BF01240473D6E71F800040DF
:101070001A8000401C80004091F8313013B191F883
:10108000300000B97047054B03F50B3241F6E461BF
:10109000D2F8EC015B5C0371704700BF2C7A002032
:1010A0002DE9F04F541E099D71D403F1FF3ABAF1B6
:1010B000000F6CDB461C7F2E69DC4F1C3F2F66DC6B
:1010C0007F2CA8BF7F2426EAE678BAF13F0FA8BF9D
:1010D0004FF03F0A444527EAE77958DBCD4E3768A1
:1010E00009EB881607EB860C04F1010BACF1040C3C
:1010F0000AF10107D14544DC6FEA090E09F1010646
:10110000BE44BE42CCF804500EF0070E0CF10404AD
:1011100037D0BEF1000F28D0BEF1010F20D0BEF1B4
:10112000020F1AD0BEF1030F14D0BEF1040F0ED07F
:10113000BEF1050F08D0BEF1060F1CBF44F8045FD6
:10114000013644F8045F013644F8045F013644F880
:10115000045F013644F8045F013644F8045F013649
:101160000136BE4244F8045F0BD00836BE426560CB
:10117000A560E56025616561A561E56144F8205FD2
:10118000F3D108F10108D8450CF5807CB2D1002BD1
:101190005DDB7F285BD83F2959DC3F2B1F469D4CE8
:1011A00021EAE176A8BF3F27B74225684FDBB400AC
:1011B00004EB002EAEF104080137A8440125F41B0E
:1011C0002E44E443B74248F8045F04F0070E3ED0D3
:1011D000BEF1000F28D0BEF1010F20D0BEF1020FEA
:1011E0001AD0BEF1030F14D0BEF1040F0ED0BEF121
:1011F000050F08D0BEF1060F1CBF48F8045F01368A
:1012000048F8045F013648F8045F013648F8045F87
:10121000013648F8045F013648F8045F01360136AC
:10122000B74248F8045F12D00836B742C8F80450F5
:10123000C8F80850C8F80C50C8F81050C8F8145036
:10124000C8F81850C8F81C5048F8205FECD1002AA4
:10125000C0F234817F2862DC3F2960D87F2A16469D
:1012600020EAE07AA8BF7F26564558DB694F741CF8
:101270003D68CAEB04074FEA0729A9F5807401EB22
:101280008A1B05EB8B05C4F302274FF480740126FB
:10129000A1452E6043D01FB3012F1CD0022F17D0C1
:1012A000032F12D0042F0DD0052F08D0062F1CBFFE
:1012B0004FF40074C5F800612E5104F580742E516E
:1012C00004F580742E5104F580742E5104F5807459
:1012D0002E5104F580742E5104F58074A1451ED062
:1012E00004F580772E5104F5007BEE5104F5407A29
:1012F00004F5806804F5A06C04F5C06E04F5E067A1
:1013000004F50064A14545F80B6045F80A6045F80E
:10131000086045F80C6045F80E60EE51E0D1002BF6
:10132000C0F2CE807F2A53DC3F2951DC3F2B1E4682
:10133000384C21EAE175A8BF3F26B542276847DC53
:10134000A90001EB022901360124A9F1040BBB44D9
:10135000AF1B2544F943AE424BF8044F01F0070799
:1013600036D017B3012F1BD0022F16D0032F11D068
:10137000042F0CD0052F07D0062F1CBF4BF8044FAD
:1013800001354BF8044F01354BF8044F01354BF84C
:10139000044F01354BF8044F01354BF8044F01352C
:1013A0000135AE424BF8044F12D00835AE42CBF8AF
:1013B0000440CBF80840CBF80C40CBF81040CBF8F9
:1013C0001440CBF81840CBF81C404BF8204FECD120
:1013D0007F286FDC3F2B6DDC7F2A20EAE070A8BFFE
:1013E0007F22904266DC0B4D561C2A68341A03EBB0
:1013F00080134FEA042A02EB83084FF48079AAF5A0
:1014000080770121D145C7F30220C8F8001059D0D8
:1014100060B301E0ACA80220012821D002281BD033
:10142000032815D004280FD0052809D006281CBF92
:101430004FF40079C8F8001148F8091009F58079CF
:1014400048F8091009F5807948F8091009F58079FC
:1014500048F8091009F5807948F8091009F58079EC
:1014600048F8091009F58079D14525D048F80910C8
:1014700009F5807209F5007309F5407E09F5806C65
:1014800009F5A06B09F5C06509F5E06609F5006985
:10149000D14548F8021048F8031048F80E1048F8F3
:1014A0000C1048F80B1048F8051048F80610DDD16C
:1014B000BDE8F08FBDE8F08FBDE8F08FBDE8F08F9C
:1014C000BDE8F08FBDE8F08F234B10B4D3F8BC20FB
:1014D00011685068097892F809C00478137A14EA00
:1014E0000C0F01EA03011DD0947A04F0030009B146
:1014F00040F0040040F00803991003F1FF3C9172A2
:10150000BCF10D0F0BD8DFE80CF021071B070A1503
:101510002121150A071B0721D1684B1ED3605DF8F6
:10152000044B7047907A00F003030029E4D043F0A5
:101530000403E1E7D3689C1ED4605DF8044B704758
:10154000D0685DF8044B0230D0607047D468013435
:10155000D4605DF8044B7047B8A80220234B10B448
:10156000D3F8C02011685068097892F809C004784F
:10157000137A14EA0C0F01EA03011DD0947A04F0E7
:10158000030009B140F0040040F00803991003F192
:10159000FF3C9172BCF10D0F0BD8DFE80CF0210776
:1015A0001B070A152121150A071B0721D1684B1EAD
:1015B000D3605DF8044B7047907A00F00303002974
:1015C000E4D043F00403E1E7D3689C1ED4605DF8E7
:1015D000044B7047D0685DF8044B0230D060704710
:1015E000D4680134D4605DF8044B7047B8A8022079
:1015F000234B10B4D3F8C42011685068097892F8CE
:1016000009C00478137A14EA0C0F01EA03011DD013
:10161000947A04F0030009B140F0040040F008039C
:10162000991003F1FF3C9172BCF10D0F0BD8DFE86C
:101630000CF021071B070A152121150A071B07219A
:10164000D1684B1ED3605DF8044B7047907A00F070
:1016500003030029E4D043F00403E1E7D3689C1EB0
:10166000D4605DF8044B7047D0685DF8044B0230DD
:10167000D0607047D4680134D4605DF8044B704783
:10168000B8A80220234B10B4D3F8C82011685068C2
:10169000097892F809C00478137A14EA0C0F01EA69
:1016A00003011DD0947A04F0030009B140F0040056
:1016B00040F00803991003F1FF3C9172BCF10D0F4B
:1016C0000BD8DFE80CF021071B070A152121150AAA
:1016D000071B0721D1684B1ED3605DF8044B704790
:1016E000907A00F003030029E4D043F00403E1E71B
:1016F000D3689C1ED4605DF8044B7047D0685DF8D9
:10170000044B0230D0607047D4680134D4605DF877
:10171000044B7047B8A80220234B10B4D3F8CC2058
:1017200011685068097892F809C00478137A14EAAD
:101730000C0F01EA03011DD0947A04F0030009B1F3
:1017400040F0040040F00803991003F1FF3C91724F
:10175000BCF10D0F0BD8DFE80CF021071B070A15B1
:101760002121150A071B0721D1684B1ED3605DF8A4
:10177000044B7047907A00F003030029E4D043F053
:101780000403E1E7D3689C1ED4605DF8044B704706
:10179000D0685DF8044B0230D0607047D4680134E3
:1017A000D4605DF8044B7047B8A80220234B10B4F6
:1017B000D3F8D02011685068097892F809C00478ED
:1017C000137A14EA0C0F01EA03011DD0947A04F095
:1017D000030009B140F0040040F00803991003F140
:1017E000FF3C9172BCF10D0F0BD8DFE80CF0210724
:1017F0001B070A152121150A071B0721D1684B1E5B
:10180000D3605DF8044B7047907A00F00303002921
:10181000E4D043F00403E1E7D3689C1ED4605DF894
:10182000044B7047D0685DF8044B0230D0607047BD
:10183000D4680134D4605DF8044B7047B8A8022026
:10184000234B10B4D3F8D42011685068097892F86B
:1018500009C00478137A14EA0C0F01EA03011DD0C1
:10186000947A04F0030009B140F0040040F008034A
:10187000991003F1FF3C9172BCF10D0F0BD8DFE81A
:101880000CF021071B070A152121150A071B072148
:10189000D1684B1ED3605DF8044B7047907A00F01E
:1018A00003030029E4D043F00403E1E7D3689C1E5E
:1018B000D4605DF8044B7047D0685DF8044B02308B
:1018C000D0607047D4680134D4605DF8044B704731
:1018D000B8A80220234B10B4D3F8D8201168506860
:1018E000097892F809C00478137A14EA0C0F01EA17
:1018F00003011DD0947A04F0030009B140F0040004
:1019000040F00803991003F1FF3C9172BCF10D0FF8
:101910000BD8DFE80CF021071B070A152121150A57
:10192000071B0721D1684B1ED3605DF8044B70473D
:10193000907A00F003030029E4D043F00403E1E7C8
:10194000D3689C1ED4605DF8044B7047D0685DF886
:10195000044B0230D0607047D4680134D4605DF825
:10196000044B7047B8A80220234B10B4D3F8DC20F6
:1019700011685068097892F809C00478137A14EA5B
:101980000C0F01EA03011DD0947A04F0030009B1A1
:1019900040F0040040F00803991003F1FF3C9172FD
:1019A000BCF10D0F0BD8DFE80CF021071B070A155F
:1019B0002121150A071B0721D1684B1ED3605DF852
:1019C000044B7047907A00F003030029E4D043F001
:1019D0000403E1E7D3689C1ED4605DF8044B7047B4
:1019E000D0685DF8044B0230D0607047D468013491
:1019F000D4605DF8044B7047B8A80220234B10B4A4
:101A0000D3F8E02011685068097892F809C004788A
:101A1000137A14EA0C0F01EA03011DD0947A04F042
:101A2000030009B140F0040040F00803991003F1ED
:101A3000FF3C9172BCF10D0F0BD8DFE80CF02107D1
:101A40001B070A152121150A071B0721D1684B1E08
:101A5000D3605DF8044B7047907A00F003030029CF
:101A6000E4D043F00403E1E7D3689C1ED4605DF842
:101A7000044B7047D0685DF8044B0230D06070476B
:101A8000D4680134D4605DF8044B7047B8A80220D4
:101A9000234B10B4D3F8E42011685068097892F809
:101AA00009C00478137A14EA0C0F01EA03011DD06F
:101AB000947A04F0030009B140F0040040F00803F8
:101AC000991003F1FF3C9172BCF10D0F0BD8DFE8C8
:101AD0000CF021071B070A152121150A071B0721F6
:101AE000D1684B1ED3605DF8044B7047907A00F0CC
:101AF00003030029E4D043F00403E1E7D3689C1E0C
:101B0000D4605DF8044B7047D0685DF8044B023038
:101B1000D0607047D4680134D4605DF8044B7047DE
:101B2000B8A80220234B10B4D3F8E82011685068FD
:101B3000097892F809C00478137A14EA0C0F01EAC4
:101B400003011DD0947A04F0030009B140F00400B1
:101B500040F00803991003F1FF3C9172BCF10D0FA6
:101B60000BD8DFE80CF021071B070A152121150A05
:101B7000071B0721D1684B1ED3605DF8044B7047EB
:101B8000907A00F003030029E4D043F00403E1E776
:101B9000D3689C1ED4605DF8044B7047D0685DF834
:101BA000044B0230D0607047D4680134D4605DF8D3
:101BB000044B7047B8A80220234B10B4D3F8EC2094
:101BC00011685068097892F809C00478137A14EA09
:101BD0000C0F01EA03011DD0947A04F0030009B14F
:101BE00040F0040040F00803991003F1FF3C9172AB
:101BF000BCF10D0F0BD8DFE80CF021071B070A150D
:101C00002121150A071B0721D1684B1ED3605DF8FF
:101C1000044B7047907A00F003030029E4D043F0AE
:101C20000403E1E7D3689C1ED4605DF8044B704761
:101C3000D0685DF8044B0230D0607047D46801343E
:101C4000D4605DF8044B7047B8A80220234B10B451
:101C50005A6811685068097892F809C00478137AB4
:101C600014EA0C0F01EA03011DD0947A04F003007A
:101C700009B140F0040040F00803991003F1FF3C63
:101C80009172BCF10D0F0BD8DFE80CF021071B0798
:101C90000A152121150A071B0721D1684B1ED360A5
:101CA0005DF8044B7047907A00F003030029E4D0FC
:101CB00043F00403E1E7D3689C1ED4605DF8044B55
:101CC0007047D0685DF8044B0230D0607047D4682C
:101CD0000134D4605DF8044B704700BFB8A80220FF
:101CE000234B10B49A6811685068097892F809C0BB
:101CF0000478137A14EA0C0F01EA03011DD0947AD8
:101D000004F0030009B140F0040040F0080399100A
:101D100003F1FF3C9172BCF10D0F0BD8DFE80CF022
:101D200021071B070A152121150A071B0721D16866
:101D30004B1ED3605DF8044B7047907A00F00303AC
:101D40000029E4D043F00403E1E7D3689C1ED4608B
:101D50005DF8044B7047D0685DF8044B0230D060EA
:101D60007047D4680134D4605DF8044B704700BFFD
:101D7000B8A80220234B10B4DA68116850680978BB
:101D800092F809C00478137A14EA0C0F01EA0301EF
:101D90001DD0947A04F0030009B140F0040040F033
:101DA0000803991003F1FF3C9172BCF10D0F0BD8A1
:101DB000DFE80CF021071B070A152121150A071B74
:101DC0000721D1684B1ED3605DF8044B7047907AB1
:101DD00000F003030029E4D043F00403E1E7D368F3
:101DE0009C1ED4605DF8044B7047D0685DF8044BCE
:101DF0000230D0607047D4680134D4605DF8044B81
:101E0000704700BFB8A80220234B10B41A691168AC
:101E10005068097892F809C00478137A14EA0C0F14
:101E200001EA03011DD0947A04F0030009B140F0E7
:101E3000040040F00803991003F1FF3C9172BCF1DB
:101E40000D0F0BD8DFE80CF021071B070A15212125
:101E5000150A071B0721D1684B1ED3605DF8044BA0
:101E60007047907A00F003030029E4D043F00403A4
:101E7000E1E7D3689C1ED4605DF8044B7047D068DE
:101E80005DF8044B0230D0607047D4680134D460F0
:101E90005DF8044B704700BFB8A802204FF47A7277
:101EA000704B02FB01F19942F0B400F2B0806E4C2D
:101EB000A14200F2B0806D4DA94200F2AE806C4E9E
:101EC000B14200F2AF806B4FB94200F2AF806A4B73
:101ED000994200F2B180694CA14200F2AF804EF20B
:101EE000E045A94200F28A8047F26F26B14288BFDE
:101EF0004FF4807200F28380614F4FF400464FF43C
:101F00008072B94280F08B8053005E4FB7FBF3FCC8
:101F1000614580F089801344B7FBF3F5A94280F056
:101F200087801344B7FBF3F4A14280F0838013440D
:101F3000B7FBF3FC614580F083801344B7FBF3F5F6
:101F4000A9427FD21344B7FBF3F4A1427CD21344DD
:101F5000B7FBF3FC614579D21344B7FBF3F5A94213
:101F600076D21344B7FBF3F7B94273D21344454C0E
:101F7000B4FBF3FC61456FD21344B4FBF3F5A94203
:101F80006CD21344B4FBF3F7B9423ED21344B4FB12
:101F9000F3FC614564D21344B4FBF3F5A94229D2A2
:101FA0001344B4FBF3F2914228BF102223D2F02451
:101FB000354D3449354A4FF47A7707FB03F3B1FBCB
:101FC000F3F34360286820F008072F60296821F4A4
:101FD0007F2C2CF47F6343F460203043204328603F
:101FE00016683307FCD5284C256845F008022260A6
:101FF000F0BC70470F22511E0C01D9E78022530814
:10200000204CB4FBF2F71E027BE70D22F3E71D4FD5
:102010000026012275E70222F1E70422EFE71346CA
:102020000024C5E70822EAE70222E4E71022E6E7F7
:102030000322E0E70422DEE72022E0E74022DEE799
:102040000522D8E70622D6E70722D4E70822D2E7FE
:102050000922D0E70A22CEE70B22CCE70C22CAE7FE
:102060000E22C8E7DF7072006F383900379C1C0001
:102070001B4E0E000D27070086930300C2C9010006
:102080000E270700000E27072C100B4024100B40D2
:102090002DE9F0410746884613F0AEFA194C1A4E66
:1020A000054604E013F0A8FA431BB34226D8236880
:1020B000DB07F7D4154A1648C2F80080076013F012
:1020C0009BFA144C104F064604E013F095FA851B5A
:1020D000BD4213D82568104B0E492B40002BF4D07D
:1020E0000E480A6802600A6006680B4C3440A4F18E
:1020F0000104B4FA84F77809BDE8F0810020BDE856
:10210000F08100BF24100B4040420F0008100B402C
:102110000C100B4030100B4001000F00DCAA022015
:102120002DE9F04F85B03F4F01900291039213F0DB
:1021300063FADFF82CA13C4EBB468146DAF80080FA
:102140003A4D13F059FA044604E013F055FA011B16
:10215000A94225D83368D907F7D4354A3548C2F89B
:102160000080506013F048FA304C054604E013F04C
:1021700043FA401BA04213D839682F4B0B40002B69
:10218000F5D02E4CDBF800002060CBF80000226870
:10219000294B1340012B03D1294D2968CA050FD4BF
:1021A00013F02AFA214BC9EB00049C42C6D90198CE
:1021B00040F23312292105B0BDE8F04F12F018BAF1
:1021C000204D214F2B701A48039B2049029E00226C
:1021D00022603B601E4A1F4B06600A601E481F4972
:1021E000B863196013F008FA104E074604E013F0C4
:1021F00003FAC21BB2420BD82B78002BF7D124680C
:10220000154D2540022D03D1012005B0BDE8F08F0A
:10221000019840F23D12232105B0BDE8F04F12F0C5
:10222000E7B900BF30100B4024100B4040420F00B4
:1022300008100B4000001A0D01000F00DCAA02205C
:1022400010100B40E0AA022000100B4004100B40BD
:10225000400001000C100B4002007F1111003A06F3
:10226000D8AA02202DE9F04F93B0804613F0C4F9AC
:10227000A44CA54E054605E013F0BEF9421BB24240
:1022800000F2DC80236813F00100F5D19F49A04AD9
:102290000860106013F0B0F99E4C9B4D064605E0B7
:1022A00013F0AAF9871BAF4200F2C88020689A4B4E
:1022B000984F0340002BF3D0DFF884A23968CAF8A6
:1022C00000103960DAF80020934E1640012E40F0DD
:1022D000B5808C4EBB464FF00A0913F08DF98A4D3C
:1022E000044604E013F088F9021BAA4225D830689E
:1022F000C207F7D48549864D884B834C4FF4D5727D
:102300000A602B6013F078F9054604E013F074F9C5
:10231000401BA04211D838687F4A0240002AF5D0FD
:10232000DBF80030CAF80030CBF80030DAF80010E3
:10233000794D0D40012D00F00582B9F10109CCD194
:1023400098F81110764B002908BF4FF44013019301
:1023500013F052F96F4F6B4CDFF8B0B10090B946F3
:1023600013F04AF9684E054604E013F045F9401BA6
:10237000B04258D8206810F00101F6D1644B694A88
:10238000CBF800101A6013F037F95F4D064604E0F1
:1023900013F032F9811BA94245D838685E490140E3
:1023A0000029F5D0D9F80020CAF80020C9F800208B
:1023B000DAF80060584B3340012B34D113F01CF98C
:1023C000514E054604E013F017F9431BB3422AD8D7
:1023D0002068C307F7D44E4B019A5349CBF800202D
:1023E000196013F009F9484D064604E013F004F9AA
:1023F000821BAA4217D83868474901400029F5D006
:10240000D9F80020CAF80020C9F80020DAF8003016
:10241000414E1E40012E06D113F0EEF800993A4DC0
:10242000401AA84215D9404640F29112432112F0B9
:10243000DFF88346584613B0BDE8F08F40464FF4AE
:10244000BF72202112F0D4F88346584613B0BDE87D
:10245000F08F364B1A68002A82DA354D19682960E8
:102460001C68284F600044BF324C267013F0C4F83B
:10247000254E054605E013F0BFF8401BB04200F2C0
:102480006B81386810F00103F5D1214A1F4C2A49AD
:102490002360116013F0B0F81E4E1B4D074605E097
:1024A00013F0AAF8C11BA94200F2568130681A4BFA
:1024B000184C0340002BF3D02268CAF80020226099
:1024C000DAF80010144F0F40012F40F0458113F04F
:1024D00093F80C4C0C4E054605E013F08DF8431BA9
:1024E000B34200F24981206810F00103F5D1084A97
:1024F000064F12493B60116013F07EF8054C024D07
:10250000064625E024100B4040420F0008100B4007
:102510000C100B4030100B4001000F0000001A0897
:102520000000304000001A370000022910100B4054
:10253000D0AA0220CCAA02200000090200001A033F
:10254000DCAA022013F058F8871BAF4200F2148176
:102550002068B24BB24F0340002BF3D03A68CAF860
:1025600000203A60DAF80010AC4E0E40012E40F028
:102570000381AC4CDFF8D8922568AB4EAB4C280CED
:102580000704C9F8007013F037F8054605E013F0AA
:1025900033F8421BB24200F2F7802368D907F6D421
:1025A000A349A44CA44A0F60226013F025F89C4F65
:1025B0009D4D064605E013F01FF8841BAC4200F267
:1025C000E3803868954B96490340002BF3D00C68A4
:1025D000CAF800400C60DAF80020904E1640012E38
:1025E00040F0D2808F4F954D954B964938682A68B8
:1025F0001F68096888F82410040A060C050E130ADF
:1026000088F82F4088F830003C0C100C88F82C20FB
:1026100088F8287088F82E60120E3E0A88F82D502F
:1026200088F82B300D0A3F0E090C002388F827602C
:1026300088F8264088F8257088F8235088F82A0002
:1026400088F8292088F8221088F83130D9F80070ED
:10265000764E754D12F0D0FF044605E012F0CCFF27
:10266000001BA84200F298803068C207F6D4704977
:10267000704B754A0F601A6012F0BEFF684D6A4CCD
:10268000064605E012F0B8FF811BA14200F28480EB
:1026900028686249624F01400029F3D03B68CAF8BC
:1026A00000303B60DAF800205C4E1640012E73D1FA
:1026B0005C4D624C2868624B624A21681B68126854
:1026C00088F82000050A060C0C0A88F81F50050E31
:1026D000080C88F8142088F81C1088F81830090EA7
:1026E00088F81E6088F81D501E0A1D0C88F81B40D3
:1026F0001B0E140A88F81A00120C002088F8191012
:1027000088F8176088F8210088F8165088F8153086
:1027100088F8134088F81220D9F800104B484C4E26
:10272000FFF7B6FC00283FD031684A48FFF7B0FCFD
:10273000002841D1404640F2AB12402111F058FF31
:10274000834682E6374F3C68B4F5D57F0CD1424EC4
:1027500088F811500196FBE5404640F2991221217C
:1027600011F046FF834670E640464FF4C2722521C1
:1027700011F03EFF834668E640464FF4CE722221B8
:1027800011F036FF834660E6404640F2A112262152
:1027900011F02EFF834658E640464FF4D2722721AF
:1027A00011F026FF834650E6404640F2A71224214E
:1027B00011F01EFF834648E602212848FFF768FC17
:1027C00083460028B6D0264D264B2968174C21F0A9
:1027D00006022A60286840F002062E604FF01015AD
:1027E0001D6012F009FF8DE80101D9F800800E4E3E
:1027F00012F002FF054604E012F0FEFE401BB0425C
:102800004FD82368DB07F7D4094A1749C2F800807C
:10281000516012F0F1FE044D06462CE001000F005D
:1028200030100B4010100B4040420F0024100B40A2
:1028300008100B400C100B400000090914100B404D
:1028400018100B401C100B400000090A00001B0769
:10285000D8AA022000001A370000304000001A06F3
:1028600028100B4044100B4000001A0D12F0C4FE5B
:10287000811BA94215D83868484B0340002BF5D07E
:102880004749474A0E68CAF800601660DAF80050F7
:10289000424A44492A40012A03D143480368D805E3
:1028A00037D412F0A9FE009D404E421BB2429CD983
:1028B000DDF8048040F233122921404611F098FEE1
:1028C00000284FD146F2A811DFF81CA1DFF81C91B7
:1028D000374F384E384D394C0020CAF80000C9F83F
:1028E000000038603060286020604046FFF7D6FA6C
:1028F00040F243424FF488634FF0010CCAF80020C5
:10290000C9F800203B6032602A60226088F810C05D
:102910009BE52B4C2B4F2C4D3A70002602AB0E60E2
:10292000DDF80480294923606FF07F442C6028483B
:10293000284A294D0D60294E29490660116012F080
:102940005BFE1A4D044604E012F056FE031BAB4238
:102950001CD838780028F7D1DAF800701F4A3A40BE
:10296000022A13D19DF81540A307ABD502AA1D4931
:102970004046FFF7D5FB0028A4D09DF8187007F05B
:102980000F03012B9ED14CF250319DE740F23D12D6
:102990002321404611F02CFE92E700BF01000F00FA
:1029A00030100B40DCAA022010100B4040420F00F8
:1029B00008D004400CD0044010D0044014D004408F
:1029C00000100B40E0AA022008100B4004100B403E
:1029D00038100B400C100B404000010002007F112A
:1029E00011003A06F1FFFF8000D0044004D00440FB
:1029F000F8B51C4B1C4C1F681C4E12F0FDFD054623
:102A000004E012F0F9FD411BB14228D82068C30749
:102A1000F7D41749174B184A0F601A6012F0ECFDF3
:102A2000164C124F064604E012F0E6FD801BB84239
:102A300015D825681248114928400028F4D0114BB8
:102A40000A681A600A601E680D4C3440012C06D1D9
:102A50000D4F3D6885F4807CCCF30020F8BD01204B
:102A6000F8BD00BFD8AA022024100B4040420F003E
:102A700008100B400C100B4000001A0D30100B40DA
:102A800001000F00DCAA022010100B402DE9F04FCE
:102A900085B08DE80E003C4FDFF82C91DFF800A1E7
:102AA0003A4E0390BB46D9F80080394D12F0A4FD90
:102AB000044604E012F0A0FD031BAB42F3D83368D8
:102AC000D907F7D4334A3448C2F80080506012F076
:102AD00093FD2F4C054604E012F08EFD411BA142F0
:102AE000E1D839682D4B0B40002BF5D0DBF8000006
:102AF000CAF80000CBF80000DAF80020274D28497A
:102B00001540012DCFD1274C2368DA05CBD5264FB0
:102B100026483D70264D00222E780A6001990160FA
:102B200036BB009C6202029B1A4D224E2A601C0496
:102B30002148224A2249234D44F400733360056042
:102B4000116012F059FD124C064604E012F054FDDB
:102B5000851BA5420ED838780028F7D1DAF8007026
:102B6000184A3A40022A05D1012005B0BDE8F08F8D
:102B7000009AD8E703984FF4F472312105B0BDE80C
:102B8000F04F11F035BD00BF30100B4024100B404A
:102B900040420F0008100B4000001A0D01000F000A
:102BA000DCAA022010100B40E0AA022000100B400B
:102BB000CCAA022004100B4038100B400C100B4024
:102BC00037003A1202007F11D8AA02202DE9F04FF7
:102BD00085B08DE80E003C4FDFF82C91DFF800A1A6
:102BE0003A4E0390BB46D9F80080394D12F004FDEF
:102BF000044604E012F000FD031BAB42F3D8336837
:102C0000D907F7D4334A3448C2F80080506012F034
:102C1000F3FC2F4C054604E012F0EEFC411BA142F0
:102C2000E1D839682D4B0B40002BF5D0DBF80000C4
:102C3000CAF80000CBF80000DAF80020274D284938
:102C40001540012DCFD1274C2368DA05CBD5264F6F
:102C500026483D70264D00222E780A6001990160B9
:102C600036BB009C6202029B1A4D224E2A601C0455
:102C70002148224A2249234D44F400733360056001
:102C8000116012F0B9FC124C064604E012F0B4FCDC
:102C9000851BA5420ED838780028F7D1DAF80070E5
:102CA000184A3A40022A05D1012005B0BDE8F08F4C
:102CB000009AD8E703984FF40272332105B0BDE8BB
:102CC000F04F11F095BC00BF30100B4024100B40AA
:102CD00040420F0008100B4000001A0D01000F00C9
:102CE000DCAA022010100B40E0AA022000100B40CA
:102CF000CCAA022004100B4038100B400C100B40E3
:102D000027003A1902007F11D8AA0220F0B5002A44
:102D1000059C5FDB002B5DDB7F285BDC3F2959DCFA
:102D20007F2AA8BF7F2220EAE0763F2BA8BF3F235F
:102D3000B24221EAE1779E464CDB274B186807EB4D
:102D4000861500EB85010D1F02F1010C0EF101014A
:102D5000BE4539DBFB437A1C0B448A4203F0070073
:102D60006C6005F104032FD010B301281BD002289A
:102D700016D0032811D004280CD0052807D0062827
:102D80001CBF43F8044F013243F8044F013243F8AB
:102D9000044F013243F8044F013243F8044F01322B
:102DA00043F8044F013201328A4243F8044F0BD0FA
:102DB00008328A425C609C60DC601C615C619C61E2
:102DC000DC6143F8204FF3D10136664505F5807587
:102DD000BED1F0BDF0BD00BFACA80220014642F25A
:102DE00010708B68DA7892060CD593F803C05FEA0E
:102DF0008C6207D5DA78920604D593F803C05FEAAF
:102E00008C6233D4B02098708A6842F2107392F8C2
:102E100003C05FEA8C6025D4D078800622D492F873
:102E200003C05FEA8C601DD4D07880061AD492F873
:102E300003C05FEA8C6015D4D078800612D492F873
:102E400003C05FEA8C600DD4D07880060AD4083BBA
:102E5000DDD193708A688020907000BF01221846EF
:102E60000A737047D178C1F340107047DA78920640
:102E7000C8D593F803C05FEA8C62C3D5DA789206AE
:102E8000C0D593F803C05FEA8C62BBD50838A9D1DE
:102E900098708B688020987000BF01220A731046DA
:102EA000704700BF01380B463A2800F25C82DFE829
:102EB00010F053024C0245023E0237023002290252
:102EC00022021B02AE01A701A001990192018B0110
:102ED00084017D0176016F01680161015A0153018E
:102EE0004C0145013E0137013001290122011B013E
:102EF00013010B010301FB00F300EB00E300DB0017
:102F0000D300CB00C300BB00B300AB00A3009B0009
:102F100093008B0083007B0073006B0063005B00F9
:102F200053004B0043003B00BC48BD49C0F8EC20B7
:102F30001A463B2011F08EBEB848BA49C0F8E820C6
:102F40001A463A2011F086BEB448B749C0F8E420CA
:102F50001A46392011F07EBEB048B449C0F8E020CE
:102F60001A46382011F076BEAC48B149C0F8DC20D2
:102F70001A46372011F06EBEA848AE49C0F8D820D6
:102F80001A46362011F066BEA448AB49C0F8D420DA
:102F90001A46352011F05EBEA048A849C0F8D020DE
:102FA0001A46342011F056BE9C48A549C0F8CC20E2
:102FB0001A46332011F04EBE9848A249C0F8C820E6
:102FC0001A46322011F046BE94489F49C0F8C420EA
:102FD0001A46312011F03EBE90489C49C0F8C020EE
:102FE0001A46302011F036BE8C489949C0F8BC20F2
:102FF0001A462F2011F02EBE88489649C0F8B820F6
:103000001A462E2011F026BE84489349C0F8B420F9
:103010001A462D2011F01EBE80489049C0F8B020FD
:103020001A462C2011F016BE7C488D49C0F8AC2001
:103030001A462B2011F00EBE78488A49C0F8A82005
:103040001A462A2011F006BE74488749C0F8A42009
:103050001A46292011F0FEBD70488449C0F8A0200E
:103060001A46282011F0F6BD6C488149C0F89C2012
:103070001A46272011F0EEBD68487E49C0F8982016
:103080001A46262011F0E6BD64487B49C0F894201A
:103090001A46252011F0DEBD60487849C0F890201E
:1030A0001A46242011F0D6BD5C487549C0F88C2022
:1030B0001A46232011F0CEBD58487249C0F8882026
:1030C0001A46222011F0C6BD54486F49C0F884202A
:1030D0001A46212011F0BEBD50486C49C0F880202E
:1030E0001A46202011F0B6BD4C486949C2671A46FD
:1030F0001F2011F0AFBD4948664982671A461E205D
:1031000011F0A8BD4548644942671A461D2011F0D8
:10311000A1BD4248614902671A461C2011F09ABDC0
:103120003E485F49C2661A461B2011F093BD3B48DA
:103130005C4982661A461A2011F08CBD37485A49FC
:1031400042661A46192011F085BD34485749026677
:103150001A46182011F07EBD30485549C2651A46FE
:10316000172011F077BD2D48524982651A46162066
:1031700011F070BD2948504942651A46152011F0DA
:1031800069BD26484D4902651A46142011F062BDFA
:1031900022484B49C2641A46132011F05BBD1F48F8
:1031A000484982641A46122011F054BD1B48464912
:1031B00042641A46112011F04DBD1848434902647B
:1031C0001A46102011F046BD14484149C2631A4600
:1031D0000F2011F03FBD11483E4982631A460E2070
:1031E00011F038BD0D483C4942631A460D2011F0DC
:1031F00031BD0A48394902631A460C2011F02ABD34
:1032000006483749C2621A460B2011F023BD034815
:10321000344982621A460A2011F01CBDC0A902205E
:103220001D09000009090000F5080000E108000080
:10323000CD080000B9080000A508000091080000B2
:103240007D080000690800005508000041080000E2
:103250002D0800001908000005080000F107000013
:10326000DD070000C9070000B5070000A107000046
:103270008D07000079070000650700005107000076
:103280003D070000290700001507000001070000A6
:10329000ED060000D9060000C5060000B1060000DA
:1032A0009D0600008906000075060000610600000A
:1032B0004D0600003906000025060000110600003A
:1032C000FD050000E9050000D5050000C10500006E
:1032D000AD0500009905000085050000710500009E
:1032E0005D050000490500001F48204942621A465A
:1032F000092011F0AFBC1C481D4902621A46082083
:1033000011F0A8BC18481B49C2611A46072011F0E9
:10331000A1BC1548184982611A46062011F09ABCD2
:103320001148164942611A46052011F093BC0E4817
:10333000134902611A46042011F08CBC0A48114955
:10334000C2601A46032011F085BC07480E4982600E
:103350001A46022011F07EBC03480C4942601A460E
:10336000012011F077BC7047C0A90220350500008C
:10337000210500000D050000F9040000E50400002F
:10338000D1040000BD040000A90400009504000061
:1033900008B5134640680A461946FFF783FD08BD85
:1033A0003C2370B5037191F86460826004460D4659
:1033B0000160002E04F057828B6842F21070DD78B5
:1033C0002D0622D4DE7832061FD493F803C05FEABC
:1033D0000C661AD4DA78150617D4DD782A0614D4C8
:1033E000DE78360611D493F803C05FEA0C650CD47E
:1033F000DA78120609D40838E1D1987088688022FA
:10340000827000BF01230B7328E00220D8708D6802
:10341000AB7843F01006AE708868002202718A68AB
:1034200042F21070D578AB0708D492F803C05FEA77
:103430008C7603D4D3789E0741F15A83D578022045
:103440005FFA85FCD0701CF0100244F0D0875FEA70
:10345000CC7504F1C08789680225CD7021688B681E
:1034600042F21070DE78320602F1F483DD782E0627
:1034700002F1F08393F803C05FEA0C6602F1EA837D
:10348000DA78150602F1E683DE78320602F1E2838D
:10349000DD782E0602F1DE8393F803C05FEA0C6547
:1034A00002F1D883DA78120602F1D4830838D9D130
:1034B000987088688022827000BF01230B73216896
:1034C0008D68AE7806F0C700A8708B6842F2107065
:1034D00093F803C05FEA8C6502F15585256895F87D
:1034E0006410002902F07D85AB6842F21071D87833
:1034F000000602F18183DE78320602F17D8393F8C3
:1035000003C05FEA0C6002F17783DA78120602F1F9
:103510007383D878060602F16F83DE78300602F1F5
:103520006B8393F803C05FEA0C6202F16583DA787B
:10353000160602F161830839D9D19970A9688022F1
:103540008A7000BF01232B7321688B6842F21070D0
:10355000DE78320602F12283DD782E0602F11E8328
:1035600093F803C05FEA0C6202F11883DA7816065A
:1035700002F11483DE78350602F11083DD782A0625
:1035800002F10C8393F803C05FEA0C6602F1068334
:10359000DA78150602F102830838D9D19870886864
:1035A0008022827000BF01230B7321688D68AE7882
:1035B00006F0C700A8708B6842F2107093F803C041
:1035C0005FEA8C6502F17484256895F8641000291F
:1035D00002F09C84AB6842F21071D878000602F1C8
:1035E000AF82DE78320602F1AB8293F803C05FEA65
:1035F0000C6002F1A582DA78120602F1A182D87875
:10360000060602F19D82DE78300602F1998293F877
:1036100003C05FEA0C6202F19382DA78160602F1C7
:103620008F820839D9D19970A96880228A7000BF29
:1036300001232B7321688B6842F21070DE7832060A
:1036400002F15082DD782E0602F14C8293F803C01D
:103650005FEA0C6202F14682DA78160602F14282D3
:10366000DE78350602F13E82DD782A0602F13A82E2
:1036700093F803C05FEA0C6602F13482DA7815062B
:1036800002F130820838D9D198708868802282701F
:1036900000BF01230B7321688D68AE7806F0C70068
:1036A000A8708B6842F2107093F803C05FEA8C65D3
:1036B00002F19383256895F86410002902F0BB831A
:1036C000AB6842F21071D878000602F1DD81DE7835
:1036D000320602F1D98193F803C05FEA0C6002F16F
:1036E000D381DA78120602F1CF81D878060602F18A
:1036F000CB81DE78300602F1C78193F803C05FEA20
:103700000C6202F1C181DA78160602F1BD81083936
:10371000D9D19970A96880228A7000BF01232B73C8
:1037200021688B6842F21070DE78320602F17E81E9
:10373000DD782E0602F17A8193F803C05FEA0C620D
:1037400002F17481DA78160602F17081DE783506AE
:1037500002F16C81DD782A0602F1688193F803C0DA
:103760005FEA0C6602F16281DA78150602F15E8189
:103770000838D9D1987088688022827000BF0123F0
:103780000B7321688D68AE7806F0C700A8708B684F
:1037900042F2107093F803C05FEA8C6502F1B282C6
:1037A000256895F86410002902F0DA82AB6842F2CD
:1037B0001071D878000602F10B81DE78320602F132
:1037C000078193F803C05FEA0C6002F10181DA78A7
:1037D000120602F1FD80D878060602F1F980DE7843
:1037E000300602F1F58093F803C05FEA0C6202F143
:1037F000EF80DA78160602F1EB800839D9D199709A
:10380000A96880228A7000BF01232B7321688B680E
:1038100042F21070DE78320602F1AC80DD782E06BE
:1038200002F1A88093F803C05FEA0C6202F1A28063
:10383000DA78160602F19E80DE78350602F19A806B
:10384000DD782A0602F1968093F803C05FEA0C66E1
:1038500002F19080DA78150602F18C800838D9D10F
:10386000987088688022827000BF01230B732168E2
:103870008D68AE7806F0C700A8708B6842F21070B1
:1038800093F803C05FEA8C6502F12985256895F8F5
:103890006410002902F05185AB6842F21071D878AB
:1038A000000602F13980DE78320602F1358093F8A5
:1038B00003C05FEA0C6002F12F80DA78120602F191
:1038C0002B80D878060602F12780DE78300602F1D8
:1038D000238093F803C05FEA0C6202F11D80DA785E
:1038E000160602F119800839D9D19970A968802289
:1038F0008A7000BF01232B7321688B6842F210701D
:10390000DE78320601F1DA87DD782E0601F1D687FE
:1039100093F803C05FEA0C6201F1D087DA781606EB
:1039200001F1CC87DE78350601F1C887DD782A06FB
:1039300001F1C48793F803C05FEA0C6601F1BE870A
:10394000DA78150601F1BA870838D9D198708868F5
:103950008022827000BF01230B7321688D68AE78CE
:1039600006F0C700A8708B6842F2107093F803C08D
:103970005FEA8C6502F14884256895F86410002997
:1039800002F07084AB6842F21071D878000601F141
:103990006787DE78320601F1638793F803C05FEA38
:1039A0000C6001F15D87DA78120601F15987D87849
:1039B000060601F15587DE78300601F1518793F84C
:1039C00003C05FEA0C6201F14B87DA78160601F159
:1039D00047870839D9D19970A96880228A7000BFB9
:1039E00001232B7321688B6842F21070DE78320657
:1039F00001F10887DD782E0601F1048793F803C0F2
:103A00005FEA0C6201F1FE86DA78160601F1FA86A9
:103A1000DE78350601F1F686DD782A0601F1F286B8
:103A200093F803C05FEA0C6601F1EC86DA781506BC
:103A300001F1E8860838D9D19870886880228270B0
:103A400000BF01230B7321688D68AE7806F0C700B4
:103A5000A8708B6842F2107093F803C05FEA8C651F
:103A600002F16783256895F86410002902F08F83BE
:103A7000AB6842F21071D878000601F19586DE78C5
:103A8000320601F1918693F803C05FEA0C6001F100
:103A90008B86DA78120601F18786D878060601F15E
:103AA0008386DE78300601F17F8693F803C05FEAF3
:103AB0000C6201F17986DA78160601F1758608390B
:103AC000D9D19970A96880228A7000BF01232B7315
:103AD00021688B6842F21070DE78320601F136867A
:103AE000DD782E0601F1328693F803C05FEA0C629E
:103AF00001F12C86DA78160601F12886DE78350683
:103B000001F12486DD782A0601F1208693F803C0AE
:103B10005FEA0C6601F11A86DA78150601F116865D
:103B20000838D9D1987088688022827000BF01233C
:103B30000B7321688D68AE7806F0C700A8708B689B
:103B400042F2107093F803C05FEA8C6502F186823E
:103B5000256895F86410002902F0AE82AB6842F245
:103B60001071D878000601F1C385DE78320601F1C4
:103B7000BF8593F803C05FEA0C6001F1B985DA787C
:103B8000120601F1B585D878060601F1B185DE7817
:103B9000300601F1AD8593F803C05FEA0C6201F1D4
:103BA000A785DA78160601F1A3850839D9D199706D
:103BB000A96880228A7000BF01232B7321688B685B
:103BC00042F21070DE78320601F16485DD782E064F
:103BD00001F1608593F803C05FEA0C6201F15A8538
:103BE000DA78160601F15685DE78350601F1528540
:103BF000DD782A0601F14E8593F803C05FEA0C6672
:103C000001F14885DA78150601F144850838D9D1E3
:103C1000987088688022827000BF01230B7321682E
:103C20008D68AE7806F0C700A8708B6842F21070FD
:103C300093F803C05FEA8C6502F1FD84256895F86E
:103C40006410002902F02585AB6842F21071D87823
:103C5000000601F1F184DE78320601F1ED8493F87B
:103C600003C05FEA0C6001F1E784DA78120601F123
:103C7000E384D878060601F1DF84DE78300601F1AE
:103C8000DB8493F803C05FEA0C6201F1D584DA7833
:103C9000160601F1D1840839D9D19970A96880221A
:103CA0008A7000BF01232B7321688B6842F2107069
:103CB000DE78320601F19284DD782E0601F18E84E1
:103CC00093F803C05FEA0C6201F18884DA78160683
:103CD00001F18484DE78350601F18084DD782A06DE
:103CE00001F17C8493F803C05FEA0C6601F17684ED
:103CF000DA78150601F172840838D9D1987088688D
:103D00008022827000BF01230B7321688D68AE781A
:103D100006F0C700A8708B6842F2107093F803C0D9
:103D20005FEA8C6502F11C84256895F8641000290F
:103D300002F04484AB6842F21071D878000601F1B9
:103D40001F84DE78320601F11B8493F803C05FEA1A
:103D50000C6001F11584DA78120601F11184D8782B
:103D6000060601F10D84DE78300601F1098493F82E
:103D700003C05FEA0C6201F10384DA78160601F1F0
:103D8000FF830839D9D19970A96880228A7000BF51
:103D900001232B7321688B6842F21070DE783206A3
:103DA00001F1C083DD782E0601F1BC8393F803C0D6
:103DB0005FEA0C6201F1B683DA78160601F1B2838C
:103DC000DE78350601F1AE83DD782A0601F1AA839B
:103DD00093F803C05FEA0C6601F1A483DA78150654
:103DE00001F1A0830838D9D1987088688022827048
:103DF00000BF01230B7321688D68AE7806F0C70001
:103E0000A8708B6842F2107093F803C05FEA8C656B
:103E100002F13B83256895F86410002902F0638362
:103E2000AB6842F21071D878000601F14D83DE785C
:103E3000320601F1498393F803C05FEA0C6001F197
:103E40004383DA78120601F13F83D878060601F140
:103E50003B83DE78300601F1378393F803C05FEAD5
:103E60000C6201F13183DA78160601F12D830839ED
:103E7000D9D19970A96880228A7000BF01232B7361
:103E800021688B6842F21070DE78320601F1EE8212
:103E9000DD782E0601F1EA8293F803C05FEA0C6236
:103EA00001F1E482DA78160601F1E082DE78350667
:103EB00001F1DC82DD782A0601F1D88293F803C093
:103EC0005FEA0C6601F1D282DA78150601F1CE8242
:103ED0000838D9D1987088688022827000BF012389
:103EE0000B7321688D68AE7806F0C700A8708B68E8
:103EF00042F2107093F803C05FEA8C6502F15A82B7
:103F0000256895F86410002902F08282AB6842F2BD
:103F10001071D878000601F17B82DE78320601F15B
:103F2000778293F803C05FEA0C6001F17182DA785E
:103F3000120601F16D82D878060601F16982DE78F9
:103F4000300601F1658293F803C05FEA0C6201F16B
:103F50005F82DA78160601F15B820839D9D199704F
:103F6000A96880228A7000BF01232B7321688B68A7
:103F700042F21070DE78320601F11C82DD782E06E6
:103F800001F1188293F803C05FEA0C6201F112821A
:103F9000DA78160601F10E82DE78350601F10A8222
:103FA000DD782A0601F1068293F803C05FEA0C6609
:103FB00001F10082DA78150601F1FC810838D9D1C7
:103FC000987088688022827000BF01230B7321687B
:103FD0008D68AE7806F0C700A8708B6842F210704A
:103FE00093F803C05FEA8C6502F1D184256895F8E7
:103FF0006410002902F0F984AB6842F21071D8789D
:10400000000601F1A981DE78320601F1A58193F85D
:1040100003C05FEA0C6001F19F81DA78120601F1BA
:104020009B81D878060601F19781DE78300601F190
:10403000938193F803C05FEA0C6201F18D81DA7815
:10404000160601F189810839D9D19970A9688022B1
:104050008A7000BF01232B7321688B6842F21070B5
:10406000DE78320601F14A81DD782E0601F14681C3
:1040700093F803C05FEA0C6201F14081DA7816061A
:1040800001F13C81DE78350601F13881DD782A06C0
:1040900001F1348193F803C05FEA0C6601F12E81CF
:1040A000DA78150601F12A810838D9D19870886824
:1040B0008022827000BF01230B7321688D68AE7867
:1040C00006F0C700A8708B6842F2107093F803C026
:1040D0005FEA8C6502F1F083256895F86410002989
:1040E00002F01884AB6842F21071D878000601F132
:1040F000D780DE78320601F1D38093F803C05FEAFF
:104100000C6001F1CD80DA78120601F1C980D8780F
:10411000060601F1C580DE78300601F1C18093F812
:1041200003C05FEA0C6201F1BB80DA78160601F188
:10413000B7800839D9D19970A96880228A7000BFE8
:1041400001232B7321688B6842F21070DE783206EF
:1041500001F17880DD782E0601F1748093F803C0B8
:104160005FEA0C6201F16E80DA78160601F16A806E
:10417000DE78350601F16680DD782A0601F162807D
:1041800093F803C05FEA0C6601F15C80DA781506EB
:1041900001F158800838D9D19870886880228270DF
:1041A00000BF01230B7321688D68AE7806F0C7004D
:1041B000A8708B6842F2107093F803C05FEA8C65B8
:1041C00002F10F83256895F86410002902F0378307
:1041D000AB6842F21071D878000601F10580DE78F4
:1041E000320601F1018093F803C05FEA0C6000F130
:1041F000FB87DA78120600F1F787D878060600F117
:10420000F387DE78300600F1EF8793F803C05FEAAA
:104210000C6200F1E987DA78160600F1E5870839C3
:10422000D9D19970A96880228A7000BF01232B73AD
:1042300021688B6842F21070DE78320600F1A687A2
:10424000DD782E0600F1A28793F803C05FEA0C62C6
:1042500000F19C87DA78160600F19887DE7835063B
:1042600000F19487DD782A0600F1908793F803C067
:104270005FEA0C6600F18A87DA78150600F1868716
:104280000838D9D1987088688022827000BF0123D5
:104290000B7321688D68AE7806F0C700A8708B6834
:1042A00042F2107093F803C05FEA8C6502F12E822F
:1042B000256895F86410002902F05682AB6842F236
:1042C0001071D878000600F13387DE78320600F1ED
:1042D0002F8793F803C05FEA0C6000F12987DA7832
:1042E000120600F12587D878060600F12187DE78CE
:1042F000300600F11D8793F803C05FEA0C6200F1FD
:104300001787DA78160600F113870839D9D1997022
:10431000A96880228A7000BF01232B7321688B68F3
:1043200042F21070DE78320600F1D486DD782E0677
:1043300000F1D08693F803C05FEA0C6200F1CA86F0
:10434000DA78160600F1C686DE78350600F1C286F8
:10435000DD782A0600F1BE8693F803C05FEA0C669A
:1043600000F1B886DA78150600F1B4860838D9D19C
:10437000987088688022827000BF01230B732168C7
:104380008D68AE7806F0C700A8708B6842F2107096
:1043900093F803C05FEA8C6502F1A284256895F862
:1043A0006410002902F0CA84AB6842F21071D87818
:1043B000000600F16186DE78320600F15D8693F832
:1043C00003C05FEA0C6000F15786DA78120600F14C
:1043D0005386D878060600F14F86DE78300600F165
:1043E0004B8693F803C05FEA0C6200F14586DA78E9
:1043F000160600F141860839D9D19970A968802242
:104400008A7000BF01232B7321688B6842F2107001
:10441000DE78320600F10286DD782E0600F1FE8598
:1044200093F803C05FEA0C6200F1F885DA781606AB
:1044300000F1F485DE78350600F1F085DD782A0696
:1044400000F1EC8593F803C05FEA0C6600F1E685A5
:10445000DA78150600F1E2850838D9D198708868B5
:104460008022827000BF01230B7321688D68AE78B3
:1044700006F0C700A8708B6842F2107093F803C072
:104480005FEA8C6502F1C283256895F86410002903
:1044900002F0EA83AB6842F21071D878000600F1AE
:1044A0008F85DE78320600F18B8593F803C05FEAD2
:1044B0000C6000F18585DA78120600F18185D878E4
:1044C000060600F17D85DE78300600F1798593F8E7
:1044D00003C05FEA0C6200F17385DA78160600F11A
:1044E0006F850839D9D19970A96880228A7000BF78
:1044F00001232B7321688B6842F21070DE7832063C
:1045000000F13085DD782E0600F12C8593F803C08C
:104510005FEA0C6200F12685DA78160600F1228542
:10452000DE78350600F11E85DD782A0600F11A8551
:1045300093F803C05FEA0C6600F11485DA7815067B
:1045400000F110850838D9D198708868802282706F
:1045500000BF01230B7321688D68AE7806F0C70099
:10456000A8708B6842F2107093F803C05FEA8C6504
:1045700002F1E282256895F86410002902F00A83AE
:10458000AB6842F21071D878000600F1BD84DE7885
:10459000320600F1B98493F803C05FEA0C6000F1C1
:1045A000B384DA78120600F1AF84D878060600F1F9
:1045B000AB84DE78300600F1A78493F803C05FEA8D
:1045C0000C6200F1A184DA78160600F19D840839A6
:1045D000D9D19970A96880228A7000BF01232B73FA
:1045E00021688B6842F21070DE78320600F15E843A
:1045F000DD782E0600F15A8493F803C05FEA0C625E
:1046000000F15484DA78160600F15084DE7835061D
:1046100000F14C84DD782A0600F1488493F803C049
:104620005FEA0C6600F14284DA78150600F13E84F8
:104630000838D9D1987088688022827000BF012321
:104640000B7321688D68AE7806F0C700A8708B6880
:1046500042F2107093F803C05FEA8C6502F10282A7
:10466000256895F86410002902F02A82AB6842F2AE
:104670001071D878000600F1EC83DE78320600F184
:10468000E88393F803C05FEA0C6000F1E283DA7814
:10469000120600F1DE83D878060600F1DA83DE78B0
:1046A000300600F1D68393F803C05FEA0C6200F194
:1046B000D083DA78160600F1CC830839D9D1997005
:1046C000A96880228A7000BF01232B7321688B6840
:1046D00042F21070DE78320600F18E83DD782E060D
:1046E00000F18A8393F803C05FEA0C6200F18483CF
:1046F000DA78160600F18083DE78350600F17C83D7
:10470000DD782A0600F1788393F803C05FEA0C662F
:1047100000F17283DA78150600F16E830838D9D17A
:10472000987088688022827000BF01230B73216813
:104730008D68AE7806F0C700A8708B6842F21070E2
:1047400093F803C05FEA8C6502F16B84256895F8E5
:104750006410002902F09384AB6842F21071D8789B
:10476000000600F11C83DE78320600F1188393F80E
:1047700003C05FEA0C6000F11283DA78120600F1E0
:104780000E83D878060600F10A83DE78300600F141
:10479000068393F803C05FEA0C6200F10083DA78C5
:1047A000160600F1FC820839D9D19970A9688022D7
:1047B0008A7000BF01232B7321688B6842F210704E
:1047C000DE78320600F1BE82DD782E0600F1BA8274
:1047D00093F803C05FEA0C6200F1B482DA7816063F
:1047E00000F1B082DE78350600F1AC82DD782A0671
:1047F00000F1A88293F803C05FEA0C6600F1A28280
:10480000DA78150600F19E820838D9D19870886848
:104810008022827000BF01230B7321688D68AE78FF
:1048200006F0C700A8708B6842F2107093F803C0BE
:104830005FEA8C6502F19283256895F8641000297F
:1048400002F0BA83AB6842F21071D878000600F12A
:104850004C82DE78320600F1488293F803C05FEAAA
:104860000C6000F14282DA78120600F13E82D878BC
:10487000060600F13A82DE78300600F1368293F8BF
:1048800003C05FEA0C6200F13082DA78160600F1AC
:104890002C820839D9D19970A96880228A7000BF0A
:1048A00001232B7321688B6842F21070DE78320688
:1048B00000F1EE81DD782E0600F1EA8193F803C065
:1048C0005FEA0C6200F1E481DA78160600F1E0811B
:1048D000DE78350600F1DC81DD782A0600F1D8812A
:1048E00093F803C05FEA0C6600F1D281DA7815060E
:1048F00000F1CE810838D9D1987088688022827002
:1049000000BF01230B7321688D68AE7806F0C700E5
:10491000A8708B6842F2107093F803C05FEA8C6550
:1049200002F1B282256895F86410002902F0DA825B
:10493000AB6842F21071D878000600F17C81DE7815
:10494000320600F1788193F803C05FEA0C6000F151
:104950007281DA78120600F16E81D878060600F1CD
:104960006A81DE78300600F1668193F803C05FEA61
:104970000C6200F16081DA78160600F15C8108397A
:10498000D9D19970A96880228A7000BF01232B7346
:1049900021688B6842F21070DE78320600F11E81C9
:1049A000DD782E0600F11A8193F803C05FEA0C62ED
:1049B00000F11481DA78160600F11081DE783506F0
:1049C00000F10C81DD782A0600F1088193F803C01C
:1049D0005FEA0C6600F10281DA78150600F1FE80CC
:1049E0000838D9D1987088688022827000BF01236E
:1049F0000B7321688D68AE7806F0C700A8708B68CD
:104A000042F2107093F803C05FEA8C6502F1D28124
:104A1000256895F86410002902F0FA81AB6842F22B
:104A20001071D878000600F1AC80DE78320600F113
:104A3000A88093F803C05FEA0C6000F1A280DA78E6
:104A4000120600F19E80D878060600F19A80DE7882
:104A5000300600F1968093F803C05FEA0C6200F123
:104A60009080DA78160600F18C800839D9D19970D7
:104A7000A96880228A7000BF01232B7321688B688C
:104A800042F21070DE7832064ED4DD782E064BD41A
:104A900093F803C05FEA0C6246D4DA78160643D472
:104AA000DE78350640D4DD782A063DD493F803C07D
:104AB0005FEA0C6638D4DA78150635D40838E1D1C7
:104AC000987088688022827000BF01230B73216870
:104AD0008D68AE7806F0C700A8708B6842F210703F
:104AE00093F803C05FEA8C6501F1E280204670BD57
:104AF000D678B5073EF5A2ACD578AB073EF59EACAF
:104B000092F803C05FEA8C763EF598ACD3789D07A7
:104B10003EF594ACD678B3073EF590AC08387EF4F9
:104B200081AC9070FEF76ABC0220D8708E68B378B2
:104B300043F01005B5708868AF2202718A6842F2AE
:104B40001070D678B5070BD492F803C05FEA8C7367
:104B500006D4D3789B0703D4D578AE0743F12384DA
:104B6000D67802205FFA86FCD0701CF0100243F069
:104B700066875FEACC7603F1708789680226CE707B
:104B8000A5E70221D970A868837843F010068670E3
:104B9000A96800220A71AA6842F21071D0788307CE
:104BA0000BD492F803C05FEA8C7606D4D3789807CA
:104BB00003D4D678B30743F1DE83D07802215FFABD
:104BC00080FCD1701CF0100243F04D875FEACC707E
:104BD00003F15787AD680220E8704FE70220D870D4
:104BE0008E68B37843F01005B5708868A72202710B
:104BF0008A6842F21070D678B5070BD492F803C0D9
:104C00005FEA8C7306D4D3789B0703D4D578AE07BC
:104C100043F19983D67802205FFA86FCD0701CF0AD
:104C2000100243F0E4865FEACC7603F1EE868968F1
:104C30000226CE70DDE60221D970A868837843F0A1
:104C400010068670A96800220A71AA6842F21071E3
:104C5000D07883070BD492F803C05FEA8C7606D431
:104C6000D378980703D4D678B30743F15483D07828
:104C700002215FFA80FCD1701CF0100243F0CB8659
:104C80005FEACC7003F1D586AD680220E8707FE65C
:104C90000220D8708E68B37843F01005B57088682C
:104CA000A42202718A6842F21070D678B5070BD43C
:104CB00092F803C05FEA8C7306D4D3789B0703D4C1
:104CC000D578AE0743F10F83D67802205FFA86FCD1
:104CD000D0701CF0100243F0DA865FEACC7603F164
:104CE000E48689680226CE700DE60221D970A86894
:104CF000837843F010068670A96800220A71AA68BA
:104D000042F21071D07883070BD492F803C05FEAA7
:104D10008C7606D4D378980703D4D678B30743F1BA
:104D2000CA82D07802215FFA80FCD1701CF0100298
:104D300043F0C1865FEACC7003F1CB86AD680220F8
:104D4000E870AFE50220D8708E68B37843F01005A4
:104D5000B5708868402202718A6842F21070D67875
:104D6000B5070BD492F803C05FEA8C7306D4D378EE
:104D70009B0703D4D578AE0743F18582D67802200D
:104D80005FFA86FCD0701CF0100243F0A8865FEA40
:104D9000CC7603F1B28689680226CE703DE5022109
:104DA000D970A868837843F010068670A96800223D
:104DB0000A71AA6842F21071D07883070BD492F876
:104DC00003C05FEA8C7606D4D378980703D4D678EC
:104DD000B30743F14082D07802215FFA80FCD170A2
:104DE0001CF0100243F08F865FEACC7003F19986C5
:104DF000AD680220E870DFE40220D8708E68B378D6
:104E000043F01005B5708868DB2202718A6842F2AF
:104E10001070D678B5070BD492F803C05FEA8C7394
:104E200006D4D3789B0703D4D578AE0743F1FB8132
:104E3000D67802205FFA86FCD0701CF0100243F096
:104E40007E835FEACC7603F1888389680226CE7080
:104E50006DE40221D970A868837843F0100686704B
:104E6000A96800220A71AA6842F21071D0788307FB
:104E70000BD492F803C05FEA8C7606D4D3789807F7
:104E800003D4D678B30743F1B681D07802215FFA14
:104E900080FCD1701CF0100243F0ED825FEACC7010
:104EA00003F1F782AD680220E8700FE40220D870A9
:104EB0008E68B37843F01005B5708868F1220271EE
:104EC0008A6842F21070D678B5070BD492F803C006
:104ED0005FEA8C7306D4D3789B0703D4D578AE07EA
:104EE00043F17181D67802205FFA86FCD0701CF005
:104EF000100243F0FC825FEACC7603F106838968F6
:104F00000226CE70FFF79DBB0221D970A868837876
:104F100043F010068670A96800220A71AA6842F25E
:104F20001071D07883070BD492F803C05FEA8C76B7
:104F300006D4D378980703D4D678B30743F12B81EE
:104F4000D07802215FFA80FCD1701CF0100243F08F
:104F5000E2825FEACC7003F1EC82AD680220E87077
:104F6000FFF73EBB0220D8708E68B37843F010057F
:104F7000B5708868D92202718A6842F21070D678BA
:104F8000B5070BD492F803C05FEA8C7306D4D378CC
:104F90009B0703D4D578AE0743F1E580D67802208D
:104FA0005FFA86FCD0701CF0100243F0C0855FEA07
:104FB000CC7603F1CA8589680226CE70FFF7CBBA9A
:104FC0000221D970A868837843F010068670A9681A
:104FD00000220A71AA6842F21071D07883070BD4BC
:104FE00092F803C05FEA8C7606D4D378980703D48E
:104FF000D678B30743F19F80D07802215FFA80FC16
:10500000D1701CF0100243F0A6855FEACC7003F16A
:10501000B085AD680220E870FFF76CBA0220D87046
:105020008E68B37843F01005B5708868FF2202716E
:105030008A6842F21070D678B5070BD492F803C094
:105040005FEA8C7306D4D3789B0703D4D578AE0778
:1050500043F15980D67802205FFA86FCD0701CF0AC
:10506000100243F08C855FEACC7603F1968589685F
:105070000226CE70FFF7F9B90221D970A8688378AB
:1050800043F010068670A96800220A71AA6842F2ED
:105090001071D07883070BD492F803C05FEA8C7646
:1050A00006D4D378980703D4D678B30743F1138096
:1050B000D07802215FFA80FCD1701CF0100243F01E
:1050C00002825FEACC7003F10C82AD680220E870C6
:1050D000FFF79AB90220D8708E68B37843F01005B4
:1050E000B5708868812202718A6842F21070D678A1
:1050F000B5070BD492F803C05FEA8C7306D4D3785B
:105100009B0703D4D578AE0742F1CD87D67802202D
:105110005FFA86FCD0701CF0100243F0B0825FEAA8
:10512000CC7603F1BA8289680226CE70FFF727B9E0
:105130000221D970A868837843F010068670A968A8
:1051400000220A71AA6842F21071D07883070BD44A
:1051500092F803C05FEA8C7606D4D378980703D41C
:10516000D678B30742F18787D07802215FFA80FCB6
:10517000D1701CF0100243F096825FEACC7003F10C
:10518000A082AD680220E870FFF7C8B80220D8708E
:105190008E68B37843F01005B570886812220271EA
:1051A0008A6842F21070D678B5070BD492F803C023
:1051B0005FEA8C7306D4D3789B0703D4D578AE0707
:1051C00042F14187D67802205FFA86FCD0701CF04D
:1051D000100243F02C825FEACC7603F136828968B4
:1051E0000226CE70FFF755B80221D970A8688378DF
:1051F00043F010068670A96800220A71AA6842F27C
:105200001071D07883070BD492F803C05FEA8C76D4
:1052100006D4D378980703D4D678B30742F1FB8637
:10522000D07802215FFA80FCD1701CF0100243F0AC
:1052300012825FEACC7003F11C82AD680220E87034
:10524000FEF7F6BF0220D8708E68B37843F01005E1
:10525000B5708868DA2202718A6842F21070D678D6
:10526000B5070BD492F803C05FEA8C7306D4D378E9
:105270009B0703D4D578AE0742F1B586D6780220D5
:105280005FFA86FCD0701CF0100243F020825FEAC7
:10529000CC7603F12A8289680226CE70FEF783BF9E
:1052A0000221D970A868837843F010068670A96837
:1052B00000220A71AA6842F21071D07883070BD4D9
:1052C00092F803C05FEA8C7606D4D378980703D4AB
:1052D000D678B30742F16F86D07802215FFA80FC5E
:1052E000D1701CF0100243F006825FEACC7003F12B
:1052F0001082AD680220E870FEF724BF0220D8704B
:105300008E68B37843F01005B5708868C8220271C2
:105310008A6842F21070D678B5070BD492F803C0B1
:105320005FEA8C7306D4D3789B0703D4D578AE0795
:1053300042F12986D67802205FFA86FCD0701CF0F4
:10534000100243F0EC815FEACC7603F1F6818968C4
:105350000226CE70FEF7B1BE0221D970A86883780C
:1053600043F010068670A96800220A71AA6842F20A
:105370001071D07883070BD492F803C05FEA8C7663
:1053800006D4D378980703D4D678B30742F1E385DF
:10539000D07802215FFA80FCD1701CF0100243F03B
:1053A000D2815FEACC7003F1DC81AD680220E87045
:1053B000FEF752BE0220D8708E68B37843F0100515
:1053C000B5708868A12202718A6842F21070D6789E
:1053D000B5070BD492F803C05FEA8C7306D4D37878
:1053E0009B0703D4D578AE0742F19D85D67802207D
:1053F0005FFA86FCD0701CF0100243F0D0825FEAA6
:10540000CC7603F1DA8289680226CE70FEF7DFBD22
:105410000221D970A868837843F010068670A968C5
:1054200000220A71AA6842F21071D07883070BD467
:1054300092F803C05FEA8C7606D4D378980703D439
:10544000D678B30742F15785D07802215FFA80FC05
:10545000D1701CF0100243F0B6825FEACC7003F109
:10546000C082AD680220E870FEF780BD0220D870CF
:105470008E68B37843F01005B57088680122027118
:105480008A6842F21070D678B5070BD492F803C040
:105490005FEA8C7306D4D3789B0703D4D578AE0724
:1054A00042F11185D67802205FFA86FCD0701CF09C
:1054B000100243F04C825FEACC7603F15682896891
:1054C0000226CE70FEF70DBD0221D970A868837840
:1054D00043F010068670A96800220A71AA6842F299
:1054E0001071D07883070BD492F803C05FEA8C76F2
:1054F00006D4D378980703D4D678B30742F1CB8487
:10550000D07802215FFA80FCD1701CF0100243F0C9
:1055100032825FEACC7003F13C82AD680220E87011
:10552000FEF7AEBC0220D8708E68B37843F0100549
:10553000B5708868202202718A6842F21070D678AD
:10554000B5070BD492F803C05FEA8C7306D4D37806
:105550009B0703D4D578AE0742F18584D678022024
:105560005FFA86FCD0701CF0100243F0A0815FEA65
:10557000CC7603F1AA8189680226CE70FEF73BBC87
:105580000221D970A868837843F010068670A96854
:1055900000220A71AA6842F21071D07883070BD4F6
:1055A00092F803C05FEA8C7606D4D378980703D4C8
:1055B000D678B30742F13F84D07802215FFA80FCAD
:1055C000D1701CF0100243F086815FEACC7003F1C9
:1055D0009081AD680220E870FEF7DCBB0220D87035
:1055E0008E68B37843F01005B57088681422027194
:1055F0008A6842F21070D678B5070BD492F803C0CF
:105600005FEA8C7306D4D3789B0703D4D578AE07B2
:1056100042F1F983D67802205FFA86FCD0701CF044
:10562000100243F06C815FEACC7603F176818968E1
:105630000226CE70FEF769BB0221D970A868837874
:1056400043F010068670A96800220A71AA6842F227
:105650001071D07883070BD492F803C05FEA8C7680
:1056600006D4D378980703D4D678B30742F1B3832E
:10567000D07802215FFA80FCD1701CF0100243F058
:1056800052815FEACC7003F15C81AD680220E87062
:10569000FEF70ABB0220D8708E68B37843F010057D
:1056A000B57088688D2202718A6842F21070D678CF
:1056B000B5070BD492F803C05FEA8C7306D4D37895
:1056C0009B0703D4D578AE0742F16D83D6780220CC
:1056D0005FFA86FCD0701CF0100243F070805FEA25
:1056E000CC7603F17A8089680226CE70FEF797BAED
:1056F0000221D970A868837843F010068670A968E3
:1057000000220A71AA6842F21071D07883070BD484
:1057100092F803C05FEA8C7606D4D378980703D456
:10572000D678B30742F12783D07802215FFA80FC54
:10573000D1701CF0100243F056805FEACC7003F188
:105740006080AD680220E870FEF738BA0220D87099
:105750008E68B37843F01005B570886840220271F6
:105760008A6842F21070D678B5070BD492F803C05D
:105770005FEA8C7306D4D3789B0703D4D578AE0741
:1057800042F1E182D67802205FFA86FCD0701CF0EC
:10579000100242F0EC875FEACC7602F1F687896866
:1057A0000226CE70FEF7C5B90221D970A8688378A9
:1057B00043F010068670A96800220A71AA6842F2B6
:1057C0001071D07883070BD492F803C05FEA8C760F
:1057D00006D4D378980703D4D678B30742F19B82D6
:1057E000D07802215FFA80FCD1701CF0100242F0E8
:1057F000D2875FEACC7002F1DC87AD680220E870E6
:10580000FEF766B90220D8708E68B37843F01005B1
:10581000B5708868002202718A6842F21070D678EA
:10582000B5070BD492F803C05FEA8C7306D4D37823
:105830009B0703D4D578AE0742F15582D678022073
:105840005FFA86FCD0701CF0100242F0E0875FEA3D
:10585000CC7602F1EA8789680226CE70FEF7F3B8AB
:105860000221D970A868837843F010068670A96871
:1058700000220A71AA6842F21071D07883070BD413
:1058800092F803C05FEA8C7606D4D378980703D4E5
:10589000D678B30742F10F82D07802215FFA80FCFC
:1058A000D1701CF0100242F0C6875FEACC7002F1A2
:1058B000D087AD680220E870FEF794B80220D87057
:1058C0008E68B37843F01005B5708868D3220271F2
:1058D0008A6842F21070D678B5070BD492F803C0EC
:1058E0005FEA8C7306D4D3789B0703D4D578AE07D0
:1058F00042F1C981D67802205FFA86FCD0701CF094
:10590000100242F0AC875FEACC7602F1B687896874
:105910000226CE70FEF721B80221D970A8688378DC
:1059200043F010068670A96800220A71AA6842F244
:105930001071D07883070BD492F803C05FEA8C769D
:1059400006D4D378980703D4D678B30742F183817D
:10595000D07802215FFA80FCD1701CF0100242F076
:1059600092875FEACC7002F19C87AD680220E870F4
:10597000FDF7C2BF0220D8708E68B37843F01005DF
:10598000B57088683F2202718A6842F21070D6783A
:10599000B5070BD492F803C05FEA8C7306D4D378B2
:1059A0009B0703D4D578AE0742F13D81D67802201B
:1059B0005FFA86FCD0701CF0100242F010865FEA9D
:1059C000CC7602F11A8689680226CE70FDF74FBFA9
:1059D0000221D970A868837843F010068670A96800
:1059E00000220A71AA6842F21071D07883070BD4A2
:1059F00092F803C05FEA8C7606D4D378980703D474
:105A0000D678B30742F1F780D07802215FFA80FCA4
:105A1000D1701CF0100242F0F6855FEACC7002F102
:105A20000086AD680220E870FDF7F0BE0220D87055
:105A30008E68B37843F01005B5708868A8220271AB
:105A40008A6842F21070D678B5070BD492F803C07A
:105A50005FEA8C7306D4D3789B0703D4D578AE075E
:105A600042F1B180D67802205FFA86FCD0701CF03B
:105A7000100242F08C855FEACC7602F19685896847
:105A80000226CE70FDF77DBE0221D970A86883780A
:105A900043F010068670A96800220A71AA6842F2D3
:105AA0001071D07883070BD492F803C05FEA8C762C
:105AB00006D4D378980703D4D678B30742F16B8025
:105AC000D07802215FFA80FCD1701CF0100242F005
:105AD00072855FEACC7002F17C85AD680220E870C7
:105AE000FDF71EBE0220D8708E68B37843F0100513
:105AF000B5708868802202718A6842F21070D67888
:105B0000B5070BD492F803C05FEA8C7306D4D37840
:105B10009B0703D4D578AE0742F12580D6780220C2
:105B20005FFA86FCD0701CF0100242F068845FEAD5
:105B3000CC7602F1728489680226CE70FDF7ABBD87
:105B40000221D970A868837843F010068670A9688E
:105B500000220A71AA6842F21071D07883070BD430
:105B600092F803C05FEA8C7606D4D378980703D402
:105B7000D678B30741F1DF87D07802215FFA80FC45
:105B8000D1701CF0100242F04E845FEACC7002F13A
:105B90005884AD680220E870FDF74CBD0220D87033
:105BA0008E68B37843F01005B5708868D52202710D
:105BB0008A6842F21070D678B5070BD492F803C009
:105BC0005FEA8C7306D4D3789B0703D4D578AE07ED
:105BD00041F19987D67802205FFA86FCD0701CF0DC
:105BE000100242F034845FEACC7602F13E84896888
:105BF0000226CE70FDF7D9BC0221D970A86883783F
:105C000043F010068670A96800220A71AA6842F261
:105C10001071D07883070BD492F803C05FEA8C76BA
:105C200006D4D378980703D4D678B30741F15387C5
:105C3000D07802215FFA80FCD1701CF0100242F093
:105C400092845FEACC7002F19C84AD680220E87017
:105C5000FDF77ABC0220D8708E68B37843F0100547
:105C6000B5708868AE2202718A6842F21070D678E8
:105C7000B5070BD492F803C05FEA8C7306D4D378CF
:105C80009E0703D4D578AD0741F10D87D678022061
:105C90005FFA86FCD0701CF0100242F000845FEACC
:105CA000CC7602F10A8489680226CE70FDF707BC23
:105CB000DA7892067EF51AAFDD78AE067EF516AF7D
:105CC000DE78B5067EF512AF93F803C05FEA8C620A
:105CD0007EF50CAFDA7896067EF508AFDD78AD0676
:105CE0007EF504AFDE78B2067EF500AF08387EF4AC
:105CF000F7AE98708B688020987000BF01220A73FD
:105D0000204670BDDA7892067DF54AADDD78AE06A4
:105D10007DF546ADDE78B5067DF542AD93F803C05E
:105D20005FEA8C627DF53CADDA7896067DF538AD9C
:105D3000DD78AD067DF534ADDE78B2067DF530ADAB
:105D400008387DF427AD98708B688020987000BF6C
:105D5000256801220A7395F8641000297DF426ADA8
:105D600028462679FDF73AF8002801F04985A86809
:105D700090F802E04EF030038370AA6842F210718E
:105D8000D078830601F10F8592F803C05FEA8C603A
:105D900001F1098592F803E05FEA8E6001F1038565
:105DA000D3789B0601F1FF84D078800601F1FB8453
:105DB00092F803C05FEA8C6301F1F58492F803E086
:105DC0005FEA8E6001F1EF84D3789B0601F1EB84EA
:105DD0000839D5D1917001F00DBDDA7892067DF5C4
:105DE00069ACDD78AE067DF565ACDE78B5067DF58F
:105DF00061AC93F803C05FEA8C627DF55BACDA7846
:105E000096067DF557ACDD78AD067DF553ACDE78B2
:105E1000B2067DF54FAC08387DF446AC98708B68BF
:105E20008020987000BF256801220A7395F86410DD
:105E300000297DF445AC28462679FCF7CFFF0028E1
:105E400001F00E85A86890F802E04EF030038370F0
:105E5000AA6842F21071D078830601F1D48492F8D6
:105E600003C05FEA8C6001F1CE8492F803E05FEA40
:105E70008E6001F1C884D3789B0601F1C484D07888
:105E8000800601F1C08492F803C05FEA8C6301F1DF
:105E9000BA8492F803E05FEA8E6001F1B484D378AB
:105EA0009B0601F1B0840839D5D1917001F0D2BCC4
:105EB000DA7892067DF588ABDD78AE067DF584ABA9
:105EC000DE78B5067DF580AB93F803C05FEA8C629F
:105ED0007DF57AABDA7896067DF576ABDD78AD06A2
:105EE0007DF572ABDE78B2067DF56EAB08387DF4D9
:105EF00065AB98708B688020987000BF2568012280
:105F00000A7395F8641000297DF464AB284626795D
:105F1000FCF764FF002801F09385A86890F802E080
:105F20004EF030038370AA6842F21071D078830675
:105F300001F1598592F803C05FEA8C6001F1538545
:105F400092F803E05FEA8E6001F14D85D3789B06FD
:105F500001F14985D078800601F1458592F803C0AA
:105F60005FEA8C6301F13F8592F803E05FEA8E609F
:105F700001F13985D3789B0601F135850839D5D1F2
:105F8000917001F057BDDA7892067DF5A7AADD7809
:105F9000AE067DF5A3AADE78B5067DF59FAA93F837
:105FA00003C05FEA8C627DF599AADA7896067DF5E2
:105FB00095AADD78AD067DF591AADE78B2067DF56D
:105FC0008DAA08387DF484AA98708B688020987018
:105FD00000BF256801220A7395F8641000297DF43A
:105FE00083AA28462679FCF7F9FE002801F0588597
:105FF000A86890F802E04EF030038370AA6842F27D
:106000001071D078830601F11E8592F803C05FEA13
:106010008C6001F1188592F803E05FEA8E6001F16F
:106020001285D3789B0601F10E85D078800601F1A8
:106030000A8592F803C05FEA8C6301F1048592F847
:1060400003E05FEA8E6001F1FE84D3789B0601F1E4
:10605000FA840839D5D1917001F01CBDDA78920626
:106060007DF576ADDD78AE067DF572ADDE78B506F0
:106070007DF56EAD93F803C05FEA8C627DF568AD87
:10608000DA7896067DF564ADDD78AD067DF560AD18
:10609000DE78B2067DF55CAD08387DF453AD9870BE
:1060A0008B688020987000BF256801220A7395F8DC
:1060B000641000297DF452AD28462679FCF78EFE47
:1060C000002801F05D84A86890F802E04EF03003EB
:1060D0008370AA6842F21071D078830601F123849C
:1060E00092F803C05FEA8C6001F11D8492F803E02E
:1060F0005FEA8E6001F11784D3789B0601F1138467
:10610000D078800601F10F8492F803C05FEA8C63B7
:1061100001F1098492F803E05FEA8E6001F10384E3
:10612000D3789B0601F1FF830839D5D1917001F036
:1061300021BCDA7892067DF595ACDD78AE067DF56A
:1061400091ACDE78B5067DF58DAC93F803C05FEABF
:106150008C627DF587ACDA7896067DF583ACDD78C8
:10616000AD067DF57FACDE78B2067DF57BAC0838F8
:106170007DF472AC98708B688020987000BF2568A1
:1061800001220A7395F8641000297DF471AC284649
:106190002679FCF723FE002801F02284A86890F8F5
:1061A00002E04EF030038370AA6842F21071D0789A
:1061B000830601F1E88392F803C05FEA8C6001F185
:1061C000E28392F803E05FEA8E6001F1DC83D3782A
:1061D0009B0601F1D883D078800601F1D48392F830
:1061E00003C05FEA8C6301F1CE8392F803E05FEABB
:1061F0008E6001F1C883D3789B0601F1C48308390E
:10620000D5D1917001F0E6BBDA7892067DF5B4AB9A
:10621000DD78AE067DF5B0ABDE78B5067DF5ACABCE
:1062200093F803C05FEA8C627DF5A6ABDA78960638
:106230007DF5A2ABDD78AD067DF59EABDE78B206CE
:106240007DF59AAB08387DF491AB98708B6880200F
:10625000987000BF256801220A7395F86410002920
:106260007DF490AB28462679FCF7B8FD002801F0B4
:10627000A781A86890F802E04EF030038370AA6806
:1062800042F21071D078830601F16D8192F803C05B
:106290005FEA8C6001F1678192F803E05FEA8E604B
:1062A00001F16181D3789B0601F15D81D078800690
:1062B00001F1598192F803C05FEA8C6301F15381C7
:1062C00092F803E05FEA8E6001F14D81D3789B067E
:1062D00001F149810839D5D1917001F06BB9DA78B3
:1062E00092067DF5D3AADD78AE067DF5CFAADE78DD
:1062F000B5067DF5CBAA93F803C05FEA8C627DF505
:10630000C5AADA7896067DF5C1AADD78AD067DF5D9
:10631000BDAADE78B2067DF5B9AA08387DF4B0AA28
:1063200098708B688020987000BF256801220A73DE
:1063300095F8641000297DF4AFAA28462679FCF769
:106340004DFD002801F06C81A86890F802E04EF045
:1063500030038370AA6842F21071D078830601F18D
:10636000328192F803C05FEA8C6001F12C8192F8CF
:1063700003E05FEA8E6001F12681D3789B0601F18C
:106380002281D078800601F11E8192F803C05FEA75
:106390008C6301F1188192F803E05FEA8E6001F1ED
:1063A0001281D3789B0601F10E810839D5D1917005
:1063B00001F030B9DA7892067DF5A2ADDD78AE064F
:1063C0007DF59EADDE78B5067DF59AAD93F803C0F8
:1063D0005FEA8C627DF594ADDA7896067DF590AD36
:1063E000DD78AD067DF58CADDE78B2067DF588AD45
:1063F00008387DF47FAD98708B688020987000BF5E
:10640000256801220A7395F8641000297DF47EAD99
:1064100028462679FCF7E2FC002801F07180A86884
:1064200090F802E04EF030038370AA6842F21071D7
:10643000D078830601F1378092F803C05FEA8C6060
:1064400001F1318092F803E05FEA8E6001F12B8068
:10645000D3789B0601F12780D078800601F1238054
:1064600092F803C05FEA8C6301F11D8092F803E0AB
:106470005FEA8E6001F11780D3789B0601F11380EB
:106480000839D5D1917001F035B8DA7892067DF5EA
:10649000C1ACDD78AE067DF5BDACDE78B5067DF528
:1064A000B9AC93F803C05FEA8C627DF5B3ACDA78DF
:1064B00096067DF5AFACDD78AD067DF5ABACDE784C
:1064C000B2067DF5A7AC08387DF49EAC98708B6859
:1064D0008020987000BF256801220A7395F8641027
:1064E00000297DF49DAC28462679FCF777FC00282E
:1064F00001F03680A86890F802E04EF03003837017
:10650000AA6842F21071D078830600F1FC8792F8F5
:1065100003C05FEA8C6000F1F68792F803E05FEA5F
:106520008E6000F1F087D3789B0600F1EC87D0787D
:10653000800600F1E88792F803C05FEA8C6300F1FF
:10654000E28792F803E05FEA8E6000F1DC87D3789F
:106550009B0600F1D8870839D5D1917000F0FABFB9
:10656000DA7892067DF5E0ABDD78AE067DF5DCAB42
:10657000DE78B5067DF5D8AB93F803C05FEA8C6290
:106580007DF5D2ABDA7896067DF5CEABDD78AD063B
:106590007DF5CAABDE78B2067DF5C6AB08387DF472
:1065A000BDAB98708B688020987000BF2568012271
:1065B0000A7395F8641000297DF4BCAB284626794F
:1065C000FCF70CFC002801F0BB80A86890F802E002
:1065D0004EF030038370AA6842F21071D0788306BF
:1065E00001F1818092F803C05FEA8C6001F17B8049
:1065F00092F803E05FEA8E6001F17580D3789B0624
:1066000001F17180D078800601F16D8092F803C0AD
:106610005FEA8C6301F1678092F803E05FEA8E60C5
:1066200001F16180D3789B0601F15D800839D5D1F5
:10663000917001F07FB8DA7892067DF5FFAADD78D7
:10664000AE067DF5FBAADE78B5067DF5F7AA93F8D0
:1066500003C05FEA8C627DF5F1AADA7896067DF5D3
:10666000EDAADD78AD067DF5E9AADE78B2067DF506
:10667000E5AA08387DF4DCAA98708B6880209870B1
:1066800000BF256801220A7395F8641000297DF483
:10669000DBAA28462679FCF7A1FB002801F08080C0
:1066A000A86890F802E04EF030038370AA6842F2C6
:1066B0001071D078830601F1468092F803C05FEA3A
:1066C0008C6001F1408092F803E05FEA8E6001F196
:1066D0003A80D3789B0601F13680D078800601F1AC
:1066E000328092F803C05FEA8C6301F12C8092F84B
:1066F00003E05FEA8E6001F12680D3789B0601F10A
:1067000022800839D5D1917001F044B8DA78920628
:106710007DF5CEADDD78AE067DF5CAADDE78B50689
:106720007DF5C6AD93F803C05FEA8C627DF5C0AD20
:10673000DA7896067DF5BCADDD78AD067DF5B8ADB1
:10674000DE78B2067DF5B4AD08387DF4ABAD987057
:106750008B688020987000BF256801220A7395F825
:10676000641000297DF4AAAD28462679FCF736FB93
:10677000002800F08587A86890F802E04EF030030A
:106780008370AA6842F21071D078830600F14B87BB
:1067900092F803C05FEA8C6000F1458792F803E04D
:1067A0005FEA8E6000F13F87D3789B0600F13B875C
:1067B000D078800600F1378792F803C05FEA8C63D7
:1067C00000F1318792F803E05FEA8E6000F12B87D9
:1067D000D3789B0600F127870839D5D1917000F056
:1067E00049BFDA7892067DF5EDACDD78AE067DF531
:1067F000E9ACDE78B5067DF5E5AC93F803C05FEA59
:106800008C627DF5DFACDA7896067DF5DBACDD7861
:10681000AD067DF5D7ACDE78B2067DF5D3AC083891
:106820007DF4CAAC98708B688020987000BF256892
:1068300001220A7395F8641000297DF4C9AC28463A
:106840002679FCF7CBFA002800F04A87A86890F870
:1068500002E04EF030038370AA6842F21071D078E3
:10686000830600F1108792F803C05FEA8C6000F1A4
:106870000A8792F803E05FEA8E6000F10487D3781C
:106880009B0600F10087D078800600F1FC8692F824
:1068900003C05FEA8C6300F1F68692F803E05FEADA
:1068A0008E6000F1F086D3789B0600F1EC86083903
:1068B000D5D1917000F00EBFDA7892067DF50CAC60
:1068C000DD78AE067DF508ACDE78B5067DF504AC66
:1068D00093F803C05FEA8C627DF5FEABDA7896062A
:1068E0007DF5FAABDD78AD067DF5F6ABDE78B20668
:1068F0007DF5F2AB08387DF4E9AB98708B688020A9
:10690000987000BF256801220A7395F86410002969
:106910007DF4E8AB28462679FCF760FA002800F001
:10692000CF84A86890F802E04EF030038370AA6824
:1069300042F21071D078830600F1958492F803C07A
:106940005FEA8C6000F18F8492F803E05FEA8E606A
:1069500000F18984D3789B0600F18584D078800685
:1069600000F1818492F803C05FEA8C6300F17B84BC
:1069700092F803E05FEA8E6000F17584D3789B069D
:1069800000F171840839D5D1917000F093BCDA78A8
:1069900092067DF52BABDD78AE067DF527ABDE7874
:1069A000B5067DF523AB93F803C05FEA8C627DF5F5
:1069B0001DABDA7896067DF519ABDD78AD067DF571
:1069C00015ABDE78B2067DF511AB08387DF408AB67
:1069D00098708B688020987000BF256801220A7328
:1069E00095F8641000297DF407AB28462679FCF75A
:1069F000F5F9002800F09484A86890F802E04EF0C1
:106A000030038370AA6842F21071D078830600F1D7
:106A10005A8492F803C05FEA8C6000F1548492F8C3
:106A200003E05FEA8E6000F14E84D3789B0600F1AC
:106A30004A84D078800600F1468492F803C05FEA69
:106A40008C6300F1408492F803E05FEA8E6000F10D
:106A50003A84D3789B0600F136840839D5D19170F9
:106A600000F058BCDA7892067DF5FAADDD78AE0616
:106A70007DF5F6ADDE78B5067DF5F2AD93F803C091
:106A80005FEA8C627DF5ECADDA7896067DF5E8ADCF
:106A9000DD78AD067DF5E4ADDE78B2067DF5E0ADDE
:106AA00008387DF4D7AD98708B688020987000BF4F
:106AB000256801220A7395F8641000297DF4D6AD8B
:106AC00028462679FCF78AF9002800F09983A868FF
:106AD00090F802E04EF030038370AA6842F2107121
:106AE000D078830600F15F8392F803C05FEA8C6080
:106AF00000F1598392F803E05FEA8E6000F153835E
:106B0000D3789B0600F14F83D078800600F14B8349
:106B100092F803C05FEA8C6300F1458392F803E0CA
:106B20005FEA8E6000F13F83D3789B0600F13B83E0
:106B30000839D5D191705DE3DA7892067DF51AAD0A
:106B4000DD78AE067DF516ADDE78B5067DF512ADC5
:106B500093F803C05FEA8C627DF50CADDA78960697
:106B60007DF508ADDD78AD067DF504ADDE78B206C5
:106B70007DF500AD08387DF4F7AC98708B68802007
:106B8000987000BF256801220A7395F864100029E7
:106B90007DF4F6AC28462679FCF720F9002800F0B1
:106BA0005F83A86890F802E04EF030038370AA6813
:106BB00042F21071D078830600F1258392F803C069
:106BC0005FEA8C6000F11F8392F803E05FEA8E6059
:106BD00000F11983D3789B0600F11583D0788006E5
:106BE00000F1118392F803C05FEA8C6300F10B831C
:106BF00092F803E05FEA8E6000F10583D3789B068C
:106C000000F101830839D5D1917023E3DA78920637
:106C10007DF53AACDD78AE067DF536ACDE78B506AE
:106C20007DF532AC93F803C05FEA8C627DF52CAC45
:106C3000DA7896067DF528ACDD78AD067DF524ACD6
:106C4000DE78B2067DF520AC08387DF417AC98707C
:106C50008B688020987000BF256801220A7395F820
:106C6000641000297DF416AC28462679FCF7B6F8A6
:106C7000002800F0E583A86890F802E04EF03003A9
:106C80008370AA6842F21071D078830600F1AB835A
:106C900092F803C05FEA8C6000F1A58392F803E0EC
:106CA0005FEA8E6000F19F83D3789B0600F19B839F
:106CB000D078800600F1978392F803C05FEA8C6376
:106CC00000F1918392F803E05FEA8E6000F18B831C
:106CD000D3789B0600F187830839D5D19170A9E359
:106CE000DA7892067DF55AABDD78AE067DF556ABC7
:106CF000DE78B5067DF552AB93F803C05FEA8C628F
:106D00007DF54CABDA7896067DF548ABDD78AD06BF
:106D10007DF544ABDE78B2067DF540AB08387DF4F6
:106D200037AB98708B688020987000BF256801226F
:106D30000A7395F8641000297DF436AB284626794D
:106D4000FCF74CF8002800F0AB83A86890F802E04C
:106D50004EF030038370AA6842F21071D078830637
:106D600000F1718392F803C05FEA8C6000F16B83DD
:106D700092F803E05FEA8E6000F16583D3789B06AA
:106D800000F16183D078800600F15D8392F803C042
:106D90005FEA8C6300F1578392F803E05FEA8E604C
:106DA00000F15183D3789B0600F14D830839D5D18A
:106DB00091706FE3DA7892067DF52AAEDD78AE0643
:106DC0007DF526AEDE78B5067DF522AE93F803C0DC
:106DD0005FEA8C627DF51CAEDA7896067DF518AE1A
:106DE000DD78AD067DF514AEDE78B2067DF510AE29
:106DF00008387DF407AE98708B688020987000BFCB
:106E0000256801220A7395F8641000297DF406AE06
:106E100028462679FBF7E2FF002800F0B182A86837
:106E200090F802E04EF030038370AA6842F21071CD
:106E3000D078830600F1778292F803C05FEA8C6015
:106E400000F1718292F803E05FEA8E6000F16B82DC
:106E5000D3789B0600F16782D078800600F16382C8
:106E600092F803C05FEA8C6300F15D8292F803E060
:106E70005FEA8E6000F15782D3789B0600F153825F
:106E80000839D5D1917075E2DA7892067DF54AAD70
:106E9000DD78AE067DF546ADDE78B5067DF542AD12
:106EA00093F803C05FEA8C627DF53CADDA78960614
:106EB0007DF538ADDD78AD067DF534ADDE78B20612
:106EC0007DF530AD08387DF427AD98708B68802053
:106ED000987000BF256801220A7395F86410002994
:106EE0007DF426AD28462679FBF778FF002800F0D0
:106EF0007782A86890F802E04EF030038370AA68A9
:106F000042F21071D078830600F13D8292F803C0FE
:106F10005FEA8C6000F1378292F803E05FEA8E60EE
:106F200000F13182D3789B0600F12D82D078800663
:106F300000F1298292F803C05FEA8C6300F123829A
:106F400092F803E05FEA8E6000F11D82D3789B0621
:106F500000F119820839D5D191703BE2DA789206B6
:106F60007DF56AACDD78AE067DF566ACDE78B506FB
:106F70007DF562AC93F803C05FEA8C627DF55CAC92
:106F8000DA7896067DF558ACDD78AD067DF554AC23
:106F9000DE78B2067DF550AC08387DF447AC9870C9
:106FA0008B688020987000BF256801220A7395F8CD
:106FB000641000297DF446AC28462679FBF70EFFC5
:106FC000002800F0BD80A86890F802E04EF0300381
:106FD0008370AA6842F21071D078830600F1838032
:106FE00092F803C05FEA8C607DD492F803E05FEA18
:106FF0008E6078D4D3789B0675D4D078800672D40E
:1070000092F803C05FEA8C636DD492F803E05FEA04
:107010008E6068D4D3789B0665D40839DCD1917032
:1070200088E0DA7892067DF591ABDD78AE067DF5E5
:107030008DABDE78B5067DF589AB93F803C05FEACA
:107040008C627DF583ABDA7896067DF57FABDD78D3
:10705000AD067DF57BABDE78B2067DF577AB083803
:107060007DF46EAB98708B688020987000BF2568A7
:1070700001220A7395F8641000297DF46DAB28464F
:107080002679FBF7ABFE002800F08A80A86890F80C
:1070900002E04EF030038370AA6842F21071D0789B
:1070A000830650D492F803C05FEA8C604BD492F808
:1070B00003E05FEA8E6046D4D3789B0643D4D07851
:1070C000800640D492F803C05FEA8C633BD492F808
:1070D00003E05FEA8E6036D4D3789B0633D4083958
:1070E000DDD1917056E07600F1B21171AB6842F2D9
:1070F0001072D878810723D4DE78B60720D493F8AD
:1071000003C05FEA8C701BD493F803E05FEA8E71D2
:1071100016D4D9788E0713D4D878800710D4DE78A7
:10712000B1070DD493F803C05FEA8C7608D4083A0F
:10713000DFD19A70AB6880229A7000BF0121297359
:107140002568FDF77FBB7600F1B21171AB6842F2A2
:107150001072D878810723D4DE78B60720D493F84C
:1071600003C05FEA8C701BD493F803E05FEA8E7172
:1071700016D4D9788E0713D4D878800710D4DE7847
:10718000B1070DD493F803C05FEA8C7608D4083AAF
:10719000DFD19A70AB6880229A7000BF01212973F9
:1071A0002568FDF7D9BA7600F1B21171AB6842F2E9
:1071B0001072D878810723D4DE78B60720D493F8EC
:1071C00003C05FEA8C701BD493F803E05FEA8E7112
:1071D00016D4D9788E0713D4D878800710D4DE78E7
:1071E000B1070DD493F803C05FEA8C7608D4083A4F
:1071F000DFD19A70AB6880229A7000BF0121297399
:107200002568FDF733BA7600F1B21171AB6842F22E
:107210001072D878810723D4DE78B60720D493F88B
:1072200003C05FEA8C701BD493F803E05FEA8E71B1
:1072300016D4D9788E0713D4D878800710D4DE7886
:10724000B1070DD493F803C05FEA8C7608D4083AEE
:10725000DFD19A70AB6880229A7000BF0121297338
:107260002568FDF78DB97600F1B21171AB6842F275
:107270001072D878810723D4DE78B60720D493F82B
:1072800003C05FEA8C701BD493F803E05FEA8E7151
:1072900016D4D9788E0713D4D878800710D4DE7826
:1072A000B1070DD493F803C05FEA8C7608D4083A8E
:1072B000DFD19A70AB6880229A7000BF01212973D8
:1072C0002568FCF70FBF7600F1B21171AB6842F28E
:1072D0001072D878810723D4DE78B60720D493F8CB
:1072E00003C05FEA8C701BD493F803E05FEA8E71F1
:1072F00016D4D9788E0713D4D878800710D4DE78C6
:10730000B1070DD493F803C05FEA8C7608D4083A2D
:10731000DFD19A70AB6880229A7000BF0121297377
:107320002568FCF769BE7600F1B21171AB6842F2D4
:107330001072D878810723D4DE78B60720D493F86A
:1073400003C05FEA8C701BD493F803E05FEA8E7190
:1073500016D4D9788E0713D4D878800710D4DE7865
:10736000B1070DD493F803C05FEA8C7608D4083ACD
:10737000DFD19A70AB6880229A7000BF0121297317
:107380002568FDF74BBB7600F1B21171AB6842F294
:107390001072D878810723D4DE78B60720D493F80A
:1073A00003C05FEA8C701BD493F803E05FEA8E7130
:1073B00016D4D9788E0713D4D878800710D4DE7805
:1073C000B1070DD493F803C05FEA8C7608D4083A6D
:1073D000DFD19A70AB6880229A7000BF01212973B7
:1073E0002568FDF7A5BA7600F1B21171AB6842F2DB
:1073F0001072D878810723D4DE78B60720D493F8AA
:1074000003C05FEA8C701BD493F803E05FEA8E71CF
:1074100016D4D9788E0713D4D878800710D4DE78A4
:10742000B1070DD493F803C05FEA8C7608D4083A0C
:10743000DFD19A70AB6880229A7000BF0121297356
:107440002568FDF727B87600F1B21171AB6842F2FA
:107450001072D878810723D4DE78B60720D493F849
:1074600003C05FEA8C701BD493F803E05FEA8E716F
:1074700016D4D9788E0713D4D878800710D4DE7844
:10748000B1070DD493F803C05FEA8C7608D4083AAC
:10749000DFD19A70AB6880229A7000BF01212973F6
:1074A0002568FCF781BF7600F1B21171AB6842F23A
:1074B0001072D878810723D4DE78B60720D493F8E9
:1074C00003C05FEA8C701BD493F803E05FEA8E710F
:1074D00016D4D9788E0713D4D878800710D4DE78E4
:1074E000B1070DD493F803C05FEA8C7608D4083A4C
:1074F000DFD19A70AB6880229A7000BF0121297396
:107500002568FCF703BD7600F1B21171AB6842F259
:107510001072D878810723D4DE78B60720D493F888
:1075200003C05FEA8C701BD493F803E05FEA8E71AE
:1075300016D4D9788E0713D4D878800710D4DE7883
:10754000B1070DD493F803C05FEA8C7608D4083AEB
:10755000DFD19A70AB6880229A7000BF0121297335
:107560002568FCF75DBC7600F1B21171AB6842F2A0
:107570001072D878810723D4DE78B60720D493F828
:1075800003C05FEA8C701BD493F803E05FEA8E714E
:1075900016D4D9788E0713D4D878800710D4DE7823
:1075A000B1070DD493F803C05FEA8C7608D4083A8B
:1075B000DFD19A70AB6880229A7000BF01212973D5
:1075C0002568FCF7DFB97600F1B21171AB6842F2C1
:1075D0001072D878810723D4DE78B60720D493F8C8
:1075E00003C05FEA8C701BD493F803E05FEA8E71EE
:1075F00016D4D9788E0713D4D878800710D4DE78C3
:10760000B1070DD493F803C05FEA8C7608D4083A2A
:10761000DFD19A70AB6880229A7000BF0121297374
:107620002568FCF739B97600F1B21171AB6842F206
:107630001072D878810723D4DE78B60720D493F867
:1076400003C05FEA8C701BD493F803E05FEA8E718D
:1076500016D4D9788E0713D4D878800710D4DE7862
:10766000B1070DD493F803C05FEA8C7608D4083ACA
:10767000DFD19A70AB6880229A7000BF0121297314
:107680002568FCF71BBE7600F1B21171AB6842F2BF
:107690001072D878810723D4DE78B60720D493F807
:1076A00003C05FEA8C701BD493F803E05FEA8E712D
:1076B00016D4D9788E0713D4D878800710D4DE7802
:1076C000B1070DD493F803C05FEA8C7608D4083A6A
:1076D000DFD19A70AB6880229A7000BF01212973B4
:1076E0002568FCF775BD7600F1B21171AB6842F206
:1076F0001072D878810723D4DE78B60720D493F8A7
:1077000003C05FEA8C701BD493F803E05FEA8E71CC
:1077100016D4D9788E0713D4D878800710D4DE78A1
:10772000B1070DD493F803C05FEA8C7608D4083A09
:10773000DFD19A70AB6880229A7000BF0121297353
:107740002568FCF7F7BA7600F1B21171AB6842F226
:107750001072D878810723D4DE78B60720D493F846
:1077600003C05FEA8C701BD493F803E05FEA8E716C
:1077700016D4D9788E0713D4D878800710D4DE7841
:10778000B1070DD493F803C05FEA8C7608D4083AA9
:10779000DFD19A70AB6880229A7000BF01212973F3
:1077A0002568FCF751BA7600F1B21171AB6842F26C
:1077B0001072D878810723D4DE78B60720D493F8E6
:1077C00003C05FEA8C701BD493F803E05FEA8E710C
:1077D00016D4D9788E0713D4D878800710D4DE78E1
:1077E000B1070DD493F803C05FEA8C7608D4083A49
:1077F000DFD19A70AB6880229A7000BF0121297393
:107800002568FBF7D3BF7600F1B21171AB6842F285
:107810001072D878810723D4DE78B60720D493F885
:1078200003C05FEA8C701BD493F803E05FEA8E71AB
:1078300016D4D9788E0713D4D878800710D4DE7880
:10784000B1070DD493F803C05FEA8C7608D4083AE8
:10785000DFD19A70AB6880229A7000BF0121297332
:107860002568FBF72DBF0846FBF7B8FA002857D06C
:10787000AA68907840F030019170AB6842F21071C4
:10788000DE78B60620D493F803C05FEA8C601BD480
:1078900093F803E05FEA8E6616D4DA78900613D484
:1078A000D878820610D4DE78B6060DD493F803C0DB
:1078B0005FEA8C6008D493F803E05FEA8E6203D439
:1078C0000839DDD1997025E078211971AB6842F251
:1078D0001072D878810723D4DE78B60720D493F8C5
:1078E00003C05FEA8C761BD493F803E05FEA8E70E6
:1078F00016D4D978890713D4D878860710D4DE78BF
:10790000B0070DD493F803C05FEA8C7108D4083A2D
:10791000DFD19A70AB6880229A7000BF0121297371
:107920002168FBF749BD7600F1B21171AB6842F2F4
:107930001072D878810723D4DE78B60720D493F864
:1079400003C05FEA8C701BD493F803E05FEA8E718A
:1079500016D4D9788E0713D4D878800710D4DE785F
:10796000B1070DD493F803C05FEA8C7608D4083AC7
:10797000DFD19A70AB6880229A7000BF0121297311
:107980002568FCF7EBB87600F1B21171AB6842F2F2
:107990001072D878810723D4DE78B60720D493F804
:1079A00003C05FEA8C701BD493F803E05FEA8E712A
:1079B00016D4D9788E0713D4D878800710D4DE78FF
:1079C000B1070DD493F803C05FEA8C7608D4083A67
:1079D000DFD19A70AB6880229A7000BF01212973B1
:1079E0002568FCF745B87600F1B21171AB6842F238
:1079F0001072D878810723D4DE78B60720D493F8A4
:107A000003C05FEA8C701BD493F803E05FEA8E71C9
:107A100016D4D9788E0713D4D878800710D4DE789E
:107A2000B1070DD493F803C05FEA8C7608D4083A06
:107A3000DFD19A70AB6880229A7000BF0121297350
:107A40002568FBF7C7BD7600F1B21171AB6842F251
:107A50001072D878810723D4DE78B60720D493F843
:107A600003C05FEA8C701BD493F803E05FEA8E7169
:107A700016D4D9788E0713D4D878800710D4DE783E
:107A8000B1070DD493F803C05FEA8C7608D4083AA6
:107A9000DFD19A70AB6880229A7000BF01212973F0
:107AA0002568FBF721BDD678B3073EF5EFA892F81D
:107AB00003C05FEA8C763EF5E9A8D3789D073EF5D2
:107AC000E5A8D578AB073EF5E1A808387EF4CFA845
:107AD0009070FBF7EEBCD07886073EF5A9A892F827
:107AE00003C05FEA8C703EF5A3A8D3789B073EF5F0
:107AF0009FA8D678B6073EF59BA808397EF489A8DA
:107B00009170FBF71BBDD678B5073EF563A892F8D8
:107B100003C05FEA8C733EF55DA8D3789E073EF5FF
:107B200059A8D578AD073EF555A808387EF443A886
:107B30009070FBF734BDD07886073EF51DA892F80B
:107B400003C05FEA8C703EF517A8D3789B073EF51B
:107B500013A8D678B6073EF50FA808397DF4FDAF17
:107B60009170FBF761BDD678B5073DF5D7AF92F8B8
:107B700003C05FEA8C733DF5D1AFD3789E073DF526
:107B8000CDAFD578AD073DF5C9AF08387DF4B7AFB7
:107B90009070FBF77ABDD07886073DF591AF92F8EB
:107BA00003C05FEA8C703DF58BAFD3789B073DF542
:107BB00087AFD678B6073DF583AF08397DF471AF4E
:107BC0009170FBF7A7BDD678B5073DF54BAF92F89E
:107BD00003C05FEA8C733DF545AFD3789E073DF552
:107BE00041AFD578AD073DF53DAF08387DF42BAFFB
:107BF0009070FBF7C0BDD07886073DF505AF92F8D1
:107C000003C05FEA8C703DF5FFAED3789B073DF56E
:107C1000FBAED678B6073DF5F7AE08397DF4E5AE94
:107C20009170FBF7EDBDD678B5073DF5BFAE92F884
:107C300003C05FEA8C733DF5B9AED3789E073DF57E
:107C4000B5AED578AD073DF5B1AE08387DF49FAE41
:107C50009070FBF706BED07886073DF579AE92F8B6
:107C600003C05FEA8C703DF573AED3789B073DF59A
:107C70006FAED678B6073DF56BAE08397DF459AED8
:107C80009170FBF733BED678B5073DF533AE92F869
:107C900003C05FEA8C733DF52DAED3789E073DF5AA
:107CA00029AED578AD073DF525AE08387DF413AE85
:107CB0009070FBF74CBED07886073DF5EDAD92F89D
:107CC00003C05FEA8C703DF5E7ADD3789B073DF5C7
:107CD000E3ADD678B6073DF5DFAD08397DF4CDAD1F
:107CE0009170FBF779BED678B5073DF5A7AD92F850
:107CF00003C05FEA8C733DF5A1ADD3789E073DF5D7
:107D00009DADD578AD073DF599AD08387DF487ADCB
:107D10009070FBF792BED07886073DF561AD92F882
:107D200003C05FEA8C703DF55BADD3789B073DF5F2
:107D300057ADD678B6073DF553AD08397DF441AD62
:107D40009170FBF7BFBED678B5073DF51BAD92F835
:107D500003C05FEA8C733DF515ADD3789E073DF502
:107D600011ADD578AD073DF50DAD08387DF4FBAC10
:107D70009070FBF7D8BED07886073DF5D5AC92F869
:107D800003C05FEA8C703DF5CFACD3789B073DF51F
:107D9000CBACD678B6073DF5C7AC08397DF4B5ACA9
:107DA0009170FBF705BFD678B5073DF58FAC92F81B
:107DB00003C05FEA8C733DF589ACD3789E073DF52F
:107DC00085ACD578AD073DF581AC08387DF46FAC56
:107DD0009070FBF71EBFD07886073DF549AC92F84E
:107DE00003C05FEA8C703DF543ACD3789B073DF54B
:107DF0003FACD678B6073DF53BAC08397DF429ACED
:107E00009170FBF74BBFD678B5073DF503AC92F800
:107E100003C05FEA8C733DF5FDABD3789E073DF55B
:107E2000F9ABD578AD073DF5F5AB08387DF4E3AB9C
:107E30009070FBF764BFD07886073DF5BDAB92F834
:107E400003C05FEA8C703DF5B7ABD3789B073DF577
:107E5000B3ABD678B6073DF5AFAB08397DF49DAB33
:107E60009170FBF791BFD678B5073DF577AB92F8E7
:107E700003C05FEA8C733DF571ABD3789E073DF587
:107E80006DABD578AD073DF569AB08387DF457ABE0
:107E90009070FBF7AABFD07886073DF531AB92F81A
:107EA00003C05FEA8C703DF52BABD3789B073DF5A3
:107EB00027ABD678B6073DF523AB08397DF411AB77
:107EC0009170FBF7D7BFD678B5073DF5EBAA92F8CE
:107ED00003C05FEA8C733DF5E5AAD3789E073DF5B4
:107EE000E1AAD578AD073DF5DDAA08387DF4CBAA27
:107EF0009070FBF7F0BFD07886073DF5A5AA92F801
:107F000003C05FEA8C703DF59FAAD3789B073DF5CF
:107F10009BAAD678B6073DF597AA08397DF485AABD
:107F20009170FCF71DB8D678B5073DF55FAA92F8B9
:107F300003C05FEA8C733DF559AAD3789E073DF5DF
:107F400055AAD578AD073DF551AA08387DF43FAA6A
:107F50009070FCF736B8D07886073DF519AA92F8EC
:107F600003C05FEA8C703DF513AAD3789B073DF5FB
:107F70000FAAD678B6073DF50BAA08397DF4F9A902
:107F80009170FCF763B8D678B5073DF5D3A992F8A0
:107F900003C05FEA8C733DF5CDA9D3789E073DF50C
:107FA000C9A9D578AD073DF5C5A908387DF4B3A9B1
:107FB0009070FCF77CB8D07886073DF58DA992F8D3
:107FC00003C05FEA8C703DF587A9D3789B073DF528
:107FD00083A9D678B6073DF57FA908397DF46DA948
:107FE0009170FCF7A9B8D678B5073DF547A992F886
:107FF00003C05FEA8C733DF541A9D3789E073DF538
:108000003DA9D578AD073DF539A908387DF427A9F4
:108010009070FCF7C2B8D07886073DF501A992F8B8
:1080200003C05FEA8C703DF5FBA8D3789B073DF554
:10803000F7A8D678B6073DF5F3A808397DF4E1A88E
:108040009170FCF7EFB8D678B5073DF5BBA892F86C
:1080500003C05FEA8C733DF5B5A8D3789E073DF564
:10806000B1A8D578AD073DF5ADA808387DF49BA83B
:108070009070FCF708B9D07886073DF575A892F89E
:1080800003C05FEA8C703DF56FA8D3789B073DF580
:108090006BA8D678B6073DF567A808397DF455A8D2
:1080A0009170FCF735B9D678B5073DF52FA892F851
:1080B00003C05FEA8C733DF529A8D3789E073DF590
:1080C00025A8D578AD073DF521A808387DF40FA87F
:1080D0009070FCF74EB9D07886073CF5E9AF92F87E
:1080E00003C05FEA8C703CF5E3AFD3789B073CF5A7
:1080F000DFAFD678B6073CF5DBAF08397CF4C9AF03
:108100009170FCF77BB9D678B5073CF5A3AF92F830
:1081100003C05FEA8C733CF59DAFD3789E073CF5B6
:1081200099AFD578AD073CF595AF08387CF483AFAF
:108130009070FCF794B9D07886073CF55DAF92F863
:1081400003C05FEA8C703CF557AFD3789B073CF5D2
:1081500053AFD678B6073CF54FAF08397CF43DAF46
:108160009170FCF7C1B9D678B5073CF517AF92F816
:1081700003C05FEA8C733CF511AFD3789E073CF5E2
:108180000DAFD578AD073CF509AF08387CF4F7AEF4
:108190009070FCF7DAB9D07886073CF5D1AE92F84A
:1081A00003C05FEA8C703CF5CBAED3789B073CF5FF
:1081B000C7AED678B6073CF5C3AE08397CF4B1AE8D
:1081C0009170FCF707BAD678B5073CF58BAE92F8FC
:1081D00003C05FEA8C733CF585AED3789E073CF50F
:1081E00081AED578AD073CF57DAE08387CF46BAE3A
:1081F0009070FCF720BAD07886073CF546AE92F82E
:1082000003C05FEA8C703CF540AED3789B073CF529
:108210003CAED678B6073CF538AE08397CF426AECD
:108220009170FCF74DBAD678B5073CF501AE92F8DF
:1082300003C05FEA8C733CF5FBADD3789E073CF539
:10824000F7ADD578AD073CF5F3AD08387CF4E1AD7A
:108250009070FCF766BAD07886073CF5BCAD92F812
:1082600003C05FEA8C703CF5B6ADD3789B073CF554
:10827000B2ADD678B6073CF5AEAD08397CF49CAD0E
:108280009170FCF793BAD678B5073CF577AD92F8C4
:1082900003C05FEA8C733CF571ADD3789E073CF563
:1082A0006DADD578AD073CF569AD08387CF457ADB8
:1082B0009070FCF7ACBAD07886073CF532AD92F8F6
:1082C00003C05FEA8C703CF52CADD3789B073CF57E
:1082D00028ADD678B6073CF524AD08397CF412AD4C
:1082E0009170FCF7D9BAD678B5073CF5EDAC92F8A9
:1082F00003C05FEA8C733CF5E7ACD3789E073CF58E
:10830000E3ACD578AD073CF5DFAC08387CF4CDACF8
:108310009070FCF7F2BAD07886073CF5A8AC92F8DA
:1083200003C05FEA8C703CF5A2ACD3789B073CF5A8
:108330009EACD678B6073CF59AAC08397CF488AC8C
:108340009170FCF71FBBD678B5073CF563AC92F88B
:1083500003C05FEA8C733CF55DACD3789E073CF5B7
:1083600059ACD578AD073CF555AC08387CF443AC36
:108370009070FCF738BBD07886073CF51EAC92F8BD
:1083800003C05FEA8C703CF518ACD3789B073CF5D2
:1083900014ACD678B6073CF510AC08397CF4FEABCB
:1083A0009170FCF765BBD678B5073CF5D9AB92F870
:1083B00003C05FEA8C733CF5D3ABD3789E073CF5E2
:1083C000CFABD578AD073CF5CBAB08387CF4B9AB77
:1083D0009070FCF776BB8B680126DE7000BF8D685D
:1083E0000873AA708B6880269E70FBF734B8886883
:1083F0001022C27000BF03208D680022F0E7886859
:108400001022C27000BF8E68032000220873B27071
:108410008B6880259D70FDF78EBB8B680125DD7014
:1084200000BF8E68F2E7A9681022CA7000BFA86872
:108430000321002229738270AB6880269E70FDF7AD
:10844000A8BBAB680126DE7000BFA868F2E78868A9
:108450001022C27000BF8E68032000220873B27021
:108460008B6880259D70FDF7C2BB8B680125DD7090
:1084700000BF8E68F2E7A9681022CA7000BFA86822
:108480000321002229738270AB6880269E70FCF75E
:1084900009BDAB680126DE7000BFA868F2E78868F6
:1084A0001022C27000BF8E68032000220873B270D1
:1084B0008B6880259D70FDF7F6BB8B680125DD700C
:1084C00000BF8E68F2E7A9681022CA7000BFA868D2
:1084D0000321002229738270AB6880269E70FCF70E
:1084E000F4BDAB680126DE7000BFA868F2E78868BB
:1084F0001022C27000BF8E68032000220873B27081
:108500008B6880259D70FCF7FABC8B680125DD70B7
:1085100000BF8E68F2E7A9681022CA7000BFA86881
:108520000321002229738270AB6880269E70FCF7BD
:1085300014BDAB680126DE7000BFA868F2E788684A
:108540001022C27000BF8E68032000220873B27030
:108550008B6880259D70FCF778BC8B680125DD70E9
:1085600000BF8E68F2E7A9681022CA7000BFA86831
:108570000321002229738270AB6880269E70FDF76C
:1085800064BBAB680126DE7000BFA868F2E78868AC
:108590001022C27000BF8E68032000220873B270E0
:1085A0008B6880259D70FDF76ABA8B680125DD70A8
:1085B00000BF8E68F2E7A9681022CA7000BFA868E1
:1085C0000321002229738270AB6880269E70FDF71C
:1085D00084BAAB680126DE7000BFA868F2E788683D
:1085E0001022C27000BF8E68032000220873B27090
:1085F0008B6880259D70FDF7E6B98B680125DD70DD
:1086000000BF8E68F2E7A9681022CA7000BFA86890
:108610000321002229738270AB6880269E70FDF7CB
:1086200000BAAB680126DE7000BFA868F2E7886870
:108630001022C27000BF8E68032000220873B2703F
:108640008B6880259D70FCF7CABD8B680125DD70A5
:1086500000BF8E68F2E7A9681022CA7000BFA86840
:108660000321002229738270AB6880269E70FCF77C
:10867000E4BDAB680126DE7000BFA868F2E7886839
:108680001022C27000BF8E68032000220873B270EF
:108690008B6880259D70FCF746BD8B680125DD70D9
:1086A00000BF8E68F2E7A9681022CA7000BFA868F0
:1086B0000321002229738270AB6880269E70FCF72C
:1086C00060BDAB680126DE7000BFA868F2E788686D
:1086D0001022C27000BF8E68032000220873B2709F
:1086E0008B6880259D70FCF7D6BD8B680125DD70F9
:1086F00000BF8E68F2E7A9681022CA7000BFA868A0
:108700000321002229738270AB6880269E70FCF7DB
:10871000F0BDAB680126DE7000BFA868F2E788688C
:108720001022C27000BF8E68032000220873B2704E
:108730008B6880259D70FCF70ABE8B680125DD7073
:1087400000BF8E68F2E7A9681022CA7000BFA8684F
:108750000321002229738270AB6880269E70FCF78B
:1087600024BEAB680126DE7000BFA868F2E7886807
:108770001022C27000BF8E68032000220873B270FE
:108780008B6880259D70FDF70AB88B680125DD7028
:1087900000BF8E68F2E7A9681022CA7000BFA868FF
:1087A0000321002229738270AB6880269E70FDF73A
:1087B00024B8AB680126DE7000BFA868F2E78868BD
:1087C0001022C27000BF8E68032000220873B270AE
:1087D0008B6880259D70FCF786BF8B680125DD7056
:1087E00000BF8E68F2E7A9681022CA7000BFA868AF
:1087F0000321002229738270AB6880269E70FCF7EB
:10880000A0BFAB680126DE7000BFA868F2E78868E9
:108810001022C27000BF8E68032000220873B2705D
:108820008B6880259D70FDF716B88B680125DD707B
:1088300000BF8E68F2E7A9681022CA7000BFA8685E
:108840000321002229738270AB6880269E70FDF799
:1088500030B8AB680126DE7000BFA868F2E7886810
:108860001022C27000BF8E68032000220873B2700D
:108870008B6880259D70FDF74AB88B680125DD70F7
:1088800000BF8E68F2E7A9681022CA7000BFA8680E
:108890000321002229738270AB6880269E70FDF749
:1088A00064B8AB680126DE7000BFA868F2E788688C
:1088B0001022C27000BF8E68032000220873B270BD
:1088C0008B6880259D70FCF756BE8B680125DD7096
:1088D00000BF8E68F2E7A9681022CA7000BFA868BE
:1088E0000321002229738270AB6880269E70FCF7FA
:1088F00070BEAB680126DE7000BFA868F2E788682A
:108900001022C27000BF8E68032000220873B2706C
:108910008B6880259D70FCF78ABE8B680125DD7011
:1089200000BF8E68F2E7A9681022CA7000BFA8686D
:108930000321002229738270AB6880269E70FCF7A9
:10894000A4BEAB680126DE7000BFA868F2E78868A5
:108950001022C27000BF8E68032000220873B2701C
:108960008B6880259D70FCF7AABD8B680125DD70A2
:1089700000BF8E68F2E7A9681022CA7000BFA8681D
:108980000321002229738270AB6880269E70FCF759
:10899000C4BDAB680126DE7000BFA868F2E7886836
:1089A0001022C27000BF8E68032000220873B270CC
:1089B0008B6880259D70FCF726BD8B680125DD70D6
:1089C00000BF8E68F2E7A9681022CA7000BFA868CD
:1089D0000321002229738270AB6880269E70FCF709
:1089E00040BDAB680126DE7000BFA868F2E788686A
:1089F0001022C27000BF8E68032000220873B2707C
:108A00008B6880259D70FCF712B98B680125DD709D
:108A100000BF8E68F2E7A9681022CA7000BFA8687C
:108A20000321002229738270AB6880269E70FCF7B8
:108A30002BB9AB680126DE7000BFA868F2E7886832
:108A40001022C27000BF8E68032000220873B2702B
:108A50008B6880259D70FCF790B88B680125DD70D0
:108A600000BF8E68F2E7A9681022CA7000BFA8682C
:108A70000321002229738270AB6880269E70FCF768
:108A8000A9B8AB680126DE7000BFA868F2E7886865
:108A90001022C27000BF8E68032000220873B270DB
:108AA0008B6880259D70FCF71CB98B680125DD70F3
:108AB00000BF8E68F2E7A9681022CA7000BFA868DC
:108AC0000321002229738270AB6880269E70FCF718
:108AD00035B9AB680126DE7000BFA868F2E7886888
:108AE0001022C27000BF8E68032000220873B2708B
:108AF0008B6880259D70FCF74EB98B680125DD7071
:108B000000BF8E68F2E7A9681022CA7000BFA8688B
:108B10000321002229738270AB6880269E70FCF7C7
:108B200067B9AB680126DE7000BFA868F2E7886805
:108B30001022C27000BF8E68032000220873B2703A
:108B40008B6880259D70FCF736BA8B680125DD7037
:108B500000BF8E68F2E7A9681022CA7000BFA8683B
:108B60000321002229738270AB6880269E70FCF777
:108B700050BAAB680126DE7000BFA868F2E78868CB
:108B80001022C27000BF8E68032000220873B270EA
:108B90008B6880259D70FCF76ABA8B680125DD70B3
:108BA00000BF8E68F2E700BFF8B5837B0446002B58
:108BB00000F0FD810568067B95F86400002800F050
:108BC0009E83AB6842F21071D878020622D4DF7817
:108BD0003F061FD493F803C05FEA0C601AD4DA781A
:108BE000120617D4D878070614D4DF78380611D4C3
:108BF00093F803C05FEA0C620CD4DA78170609D444
:108C00000839E1D19970A96880228A7000BF0123D8
:108C10002B7325E00221D970A868837843F01007F0
:108C20008770A96800220A71AA6842F21071D07890
:108C3000800705D492F803C05FEA8C7340F1BE81CF
:108C4000D07802215FFA80FCD1701CF0100242F053
:108C50005A805FEACC7701F13887AD680220E8706E
:108C600021688B6842F21070DF783D0622D4DD78EF
:108C70002A061FD493F803C05FEA0C621AD4DA788C
:108C8000170617D4DF783D0614D4DD782A0611D4F0
:108C900093F803C05FEA0C670CD4DA78150609D4A0
:108CA0000838E1D1987088688022827000BF012363
:108CB0000B7328E00220D8708F68BB7843F0100552
:108CC000BD708868812202718A6842F21070D7787C
:108CD000BF0708D492F803C05FEA8C7503D4D37839
:108CE0009B0740F1F182D77802205FFA87FCD070B1
:108CF0001CF0100241F0F9875FEACC7302F1558055
:108D000089680227CF7021688D68AF7807F0C700A7
:108D1000A8708B6842F2107093F803C05FEA8C670A
:108D200000F19481256895F86410002900F0BC8159
:108D3000AB6842F21071D878020616D4DF783F068D
:108D400013D493F803C05FEA0C600ED4DA781206ED
:108D50000BD4D878070608D4DF78380605D493F802
:108D600003C05FEA0C6240F134820221D970A86826
:108D7000837843F010078770A96800220A71AA68F7
:108D800042F21071D078800708D492F803C05FEAED
:108D90008C7303D4D378980740F17B82D07802217A
:108DA0005FFA80FCD1701CF0100241F0C2875FEACC
:108DB000CC7701F1F487AD680220E87021688B68F8
:108DC00042F21070DF783D0616D4DD782A0613D4FF
:108DD00093F803C05FEA0C620ED4DA7817060BD45E
:108DE000DF783D0608D4DD782A0605D493F803C061
:108DF0005FEA0C6740F1DE810220D8708F68BB7893
:108E000043F01005BD708A6816718A6842F21070CE
:108E1000D778BF0708D492F803C05FEA8C7503D4F3
:108E2000D3789B0740F11A82D77802205FFA87FC3B
:108E3000D0701CF0100241F08A875FEACC7301F118
:108E4000A28789680227CF7021688D68AF7807F004
:108E5000C700A8708B6842F2107093F803C05FEAF5
:108E60008C6700F1CA802568617B95F864700029E1
:108E70000CBFA626A726002F01F0BE85AB6842F2E4
:108E80001071D878020616D4DF783F0613D493F811
:108E900003C05FEA0C600ED4DA7812060BD4D878DF
:108EA000070608D4DF78380605D493F803C05FEAD4
:108EB0000C6240F170810221D970A868837843F078
:108EC00010078770A96800220A71AA6842F210711F
:108ED000D078800708D492F803C05FEA8C7303D47B
:108EE000D378980740F19F81D07802215FFA80FC07
:108EF000D1701CF0100241F00E875FEACC7701F1CF
:108F00005A87AD680220E87021688B6842F21070C1
:108F1000DF783D0616D4DD782A0613D493F803C013
:108F20005FEA0C620ED4DA7817060BD4DF783D06C0
:108F300008D4DD782A0605D493F803C05FEA0C67ED
:108F400040F11A810220D8708F68BB7843F0100579
:108F5000BD708A6816718A6842F21070D678B307BD
:108F600008D4D778BF0705D492F803C05FEA8C769F
:108F700040F13E81D3780220DDB2D07015F01002AE
:108F800041F0F386EE0701F1048789680227CF706C
:108F900021688E68B27802F0C707B7708B6842F21A
:108FA0001070DD78AD0600F1BC800021A17325684A
:108FB00095F86470002F00F00382F8BDD37898070D
:108FC0003FF53EAED778BB073FF53AAED07887077E
:108FD0003FF536AE92F803C05FEA8C703FF530AED5
:108FE000D3789B073FF52CAED778BF073FF528AE67
:108FF00008397FF41CAE917005E6DA7895067FF5A6
:1090000032AFDD78AF067FF52EAFDF78BD067FF596
:109010002AAF93F803C05FEA8C627FF524AFDA7859
:1090200097067FF520AFDD78AD067FF51CAFDF78C2
:10903000BA067FF518AF08387FF40FAF98708B68C9
:109040008020987000BF01220A730CE7DA78950639
:109050007FF568AEDD78AF067FF564AEDF78BD06DC
:109060007FF560AE93F803C05FEA8C627FF55AAE7D
:10907000DA7897067FF556AEDD78AD067FF552AE0D
:10908000DF78BA067FF54EAE08387FF445AE9870AB
:109090008B688020987000BF256801220A7395F8BC
:1090A000641000297FF444AE28462779F9F796FE2C
:1090B000002801F09E84A86890F802E04EF030038A
:1090C0008370AA6842F21071D078800601F164843E
:1090D00092F803C05FEA8C6301F15E8492F803E0CA
:1090E0005FEA8E6001F15884D3789B0601F15484C5
:1090F000D078800601F1508492F803C05FEA8C6357
:1091000001F14A8492F803E05FEA8E6001F1448441
:10911000D3789B0601F140840839D5D1917001F0D4
:1091200062BCDE78B2067FF540AF93F803C05FEA19
:109130008C627FF53AAFDA7897067FF536AFDF7845
:10914000BE067FF532AFDD78AD067FF52EAFDE7857
:10915000B2067FF52AAF93F803C05FEA8C677FF50C
:1091600024AF08387FF41DAF98708B68802098700A
:1091700000BF01220A7318E7DA7815063FF5E2AE60
:1091800008387FF4C5AE98708B688020987000BF57
:1091900001250D73FCE6DA7817063FF58CAE083929
:1091A0007FF46FAE9970A96880228A7000BF012396
:1091B0002B73A9E6DA7815063FF51EAE08387FF462
:1091C00001AE987088688022827000BF01230B7303
:1091D0003AE6DA7817063FF5C8AD08397FF4ABAD4B
:1091E0009970A96880228A7000BF01232B73E5E57E
:1091F000D3789D073FF5BEAED578AB073FF5BAAE45
:10920000D678B7073FF5B6AED778BE073FF5B2AE12
:1092100092F803C05FEA8C753FF5ACAE08387FF476
:109220009DAE9070B0E7D778BB073FF55DAED078C4
:1092300087073FF559AE92F803C05FEA8C703FF59F
:1092400053AED3789B073FF54FAED778BF073FF5B6
:109250004BAE08397FF43CAE9170A4E7D578AF07E8
:109260003FF5E2ADD778BD073FF5DEAD92F803C01C
:109270005FEA8C733FF5D8ADD3789F073FF5D4AD47
:10928000D578AD073FF5D0AD08387FF4C1AD90700B
:1092900098E7D778BB073FF581ADD07887073FF5D2
:1092A0007DAD92F803C05FEA8C703FF577ADD3785F
:1092B0009B073FF573ADD778BF073FF56FAD083912
:1092C0007FF460AD91708CE7D578AF073FF50BADBB
:1092D000D778BD073FF507AD92F803C05FEA8C73FE
:1092E0003FF501ADD3789F073FF5FDACD578AD07CD
:1092F0003FF5F9AC08387FF4EAAC9070D3E4284627
:109300002779F9F76BFD002858D0AA68917841F0C9
:1093100030039370AA6842F21071D078800620D48E
:1093200092F803C05FEA8C631BD492F803E05FEA13
:109330008E6016D4D3789B0613D4D078800610D4D0
:1093400092F803C05FEA8C630BD492F803E05FEA03
:109350008E6006D4D3789B0603D40839DDD1917092
:1093600026E07F00F9B21171AB6842F21072D87832
:10937000800723D4DF78B90720D493F803C05FEACD
:109380008C701BD493F803E05FEA8E7116D4D97801
:109390008F0713D4D878800710D4DF78B9070DD49D
:1093A00093F803C05FEA8C7708D4083ADFD19A704B
:1093B000AB6880229A7000BF01212973256800E400
:1093C00028462679F9F70AFD002837D0A86890F8D2
:1093D00002E04EF030038370AA6842F21071D77831
:1093E000BB0600F16083D078870600F15C8392F8B9
:1093F00003C05FEA8C6300F1568392F803E05FEAF2
:109400008E6700F15083D378980600F14C83D778AB
:10941000BB0600F14883D078870600F1448392F8B8
:1094200003C05FEA8C6000F13E830839D7D19170A8
:10943000AB6880229A7000BF01262E7321688B686A
:1094400042F21070DD782A0600F15B83DF783F0678
:1094500000F1578393F803E05FEA0E6600F1518351
:1094600093F803C05FEA0C6500F14B83DA781206CB
:1094700000F14783DE78370600F14383DD782E065E
:1094800000F13F83DF783D0600F13B830838D9D1F6
:1094900098708B688020987000BF01260E73216839
:1094A0008B6842F21070DF783F0600F1328693F845
:1094B00003E05FEA0E6600F12C8693F803C05FEAD2
:1094C0000C6500F12686DA78120600F12286DD7836
:1094D0002F0600F11E86DE78360600F11A86DF7848
:1094E0003D0600F1168693F803E05FEA0E6200F194
:1094F00010860838D7D198708B688020987000BF8C
:1095000001250D7321688E68B27802F0C707B77025
:109510008B6842F21070DD78AE0600F13C8625685B
:1095200095F86410002900F06686AB6842F210716D
:10953000D878000600F1AB85DF783A0600F1A78500
:1095400093F803C05FEA0C6000F1A18593F803E093
:109550005FEA0E6200F19B85DA78170600F19785C5
:10956000DE78360600F19385D878000600F18F8505
:10957000DF783A0600F18B850839D9D19970AB684C
:109580008021997000BF01262E7321688B6842F2FA
:109590001070DF783D0600F1388593F803C05FEA6C
:1095A0000C6200F1328593F803E05FEA0E6500F18A
:1095B0002C85DA78120600F12885DD782F0600F177
:1095C0002485DE78360600F12085DF783D0600F13F
:1095D0001C8593F803C05FEA0C6200F11685083819
:1095E000D7D198708B688020987000BF01250D73CB
:1095F00021688E68B27802F0C707B7708B6842F2B4
:109600001070DD78AD0600F11987256895F86410B3
:10961000002900F04387AB6842F21071D878020647
:1096200000F1B184DF783F0600F1AD8493F803E0E8
:109630005FEA0E6000F1A78493F803C05FEA0C6252
:1096400000F1A184DA78170600F19D84DE783606F1
:1096500000F19984D878000600F19584DF783A0605
:1096600000F191840839D9D19970AB688021997043
:1096700000BF01262E7321688B6842F21070DF78DC
:109680003F0600F13E8493F803E05FEA0E6600F1C6
:10969000388493F803C05FEA0C6500F13284DA780D
:1096A000120600F12E84DD782F0600F12A84DE7880
:1096B000360600F12684DF783D0600F1228493F817
:1096C00003E05FEA0E6200F11C840838D7D198707D
:1096D0008B688020987000BF01250D7321688E680B
:1096E000B27802F0C707B7708B6842F21070DD786D
:1096F000AE0600F11487256895F86410002900F083
:109700003E87AB6842F21071D878000600F1B98349
:10971000DF783A0600F1B58393F803C05FEA0C6086
:1097200000F1AF8393F803E05FEA0E6200F1A983D2
:10973000DA78170600F1A583DE78360600F1A183FA
:10974000D878000600F19D83DF783A0600F199830E
:109750000839D9D19970AB688021997000BF012672
:109760002E7321688B6842F21070DF783D0600F19D
:10977000488393F803C05FEA0C6200F1428393F8D8
:1097800003E05FEA0E6500F13C83DA78120600F12F
:109790003883DD782F0600F13483DE78360600F159
:1097A0003083DF783D0600F12C8393F803C05FEA35
:1097B0000C6200F126830838D7D198708B6880201E
:1097C000987000BF01250D7321688E68B27802F091
:1097D000C707B7708B6842F21070DD78AD0600F1F4
:1097E0004B85256895F86410002900F07585AB68F5
:1097F00042F21071D878020600F1C382DF783F068A
:1098000000F1BF8293F803E05FEA0E6000F1B982D5
:1098100093F803C05FEA0C6200F1B382DA781706AE
:1098200000F1AF82DE78360600F1AB82D878000610
:1098300000F1A782DF783A0600F1A3820839D9D176
:109840009970AB688021997000BF01262E73216842
:109850008B6842F21070DF783F0600F1528293F875
:1098600003E05FEA0E6600F14C8293F803C05FEA02
:109870000C6500F14682DA78120600F14282DD784A
:109880002F0600F13E82DE78360600F13A82DF785C
:109890003D0600F1368293F803E05FEA0E6200F1C4
:1098A00030820838D7D198708B688020987000BFBC
:1098B00001250D7321688E68B27802F0C707B77072
:1098C0008B6842F21070DD78AE0600F1468525689F
:1098D00095F86410002900F07085AB6842F21071B1
:1098E000D878000600F1CD81DF783A0600F1C98111
:1098F00093F803C05FEA0C6000F1C38193F803E0C2
:109900005FEA0E6200F1BD81DA78170600F1B981D5
:10991000DE78360600F1B581D878000600F1B18115
:10992000DF783A0600F1AD810839D9D19970AB687A
:109930008021997000BF01262E7321688B6842F246
:109940001070DF783D0600F15C8193F803C05FEA98
:109950000C6200F1568193F803E05FEA0E6500F1B6
:109960005081DA78120600F14C81DD782F0600F183
:109970004881DE78360600F14481DF783D0600F14B
:10998000408193F803C05FEA0C6200F13A81083825
:10999000D7D198708B688020987000BF01250D7317
:1099A00021688E68B27802F0C707B7708B6842F200
:1099B0001070DD78AD0600F12386256895F86410F7
:1099C000002900F04D86AB6842F21071D87802068B
:1099D00000F1D780DF783F0600F1D38093F803E0F1
:1099E0005FEA0E6000F1CD8093F803C05FEA0C627D
:1099F00000F1C780DA78170600F1C380DE783606FA
:109A000000F1BF80D878000600F1BB80DF783A060D
:109A100000F1B7800839D9D19970AB68802199706D
:109A200000BF01262E73236893F86470002F7FF423
:109A3000C4AAA5689A68DD664FF480641C6742F288
:109A4000107092F803E05FEA0E6700F1498692F821
:109A500003C05FEA0C6600F14386D1780C0600F182
:109A60003F86D678310600F13B86D7783F0600F175
:109A70003786D478260600F1338692F803E05FEA51
:109A80000E6400F12D8692F803C05FEA0C6100F1CC
:109A900027860838D5D1907098688021817000BFE2
:109AA00001241C73F8BD7600F1B21171AB6842F26B
:109AB0001072DF78B8073FF5C1ACD87881073FF561
:109AC000BDACDE78B0073FF5B9AC93F803E05FEAD0
:109AD0008E713FF5B3AC93F803C05FEA8C773FF526
:109AE000ADACD9788E073FF5A9ACDF78B8073FF564
:109AF000A5ACD87881073FF5A1AC083AD9D19A70C6
:109B000096E40220D8708A68937843F01006967025
:109B10008D6800272F718A6842F2107092F803E076
:109B20005FEA8E761ED492F803C05FEA8C7519D472
:109B3000D3789B0716D4D678B70713D4D578AE0759
:109B400010D4D778BD070DD492F803E05FEA8E7386
:109B500008D492F803C05FEA8C7703D40838DDD1CB
:109B6000907096E4D3780220DEB2D07016F0100226
:109B700040F0D187F30700F1C28789680225CD70D4
:109B80008DE40221D970AA68937843F0100696708C
:109B9000A86840270771AA6842F2107192F803E0A2
:109BA0005FEA8E761ED492F803C05FEA8C7019D4F7
:109BB000D3789F0716D4D678B60713D4D078800709
:109BC00010D4D778BB070DD492F803E05FEA8E7704
:109BD00008D492F803C05FEA8C7603D40839DDD14B
:109BE00091701AE7D3780221DEB2D17016F010021C
:109BF00041F03F80F30701F10880AD680220E87072
:109C000011E70220D8708A68937843F010059570A8
:109C10008E68072737718A6842F2107092F803E065
:109C20005FEA8E731ED492F803C05FEA8C7719D472
:109C3000D3789F0716D4D578AE0713D4D678B50756
:109C400010D4D778BB070DD492F803E05FEA8E7783
:109C500008D492F803C05FEA8C7603D40838DDD1CB
:109C6000907097E6D3780220DDB2D07015F0100224
:109C700040F0BB87EE0700F1AC8789680227CF7000
:109C80008EE60221D970AA68937843F01006967088
:109C9000A86800270771AA6842F2107192F803C001
:109CA0005FEA8C731ED492F803E05FEA8E7719D4D2
:109CB000D3789F0716D4D678B60713D4D078800708
:109CC00010D4D778BB070DD492F803C05FEA8C7725
:109CD00008D492F803E05FEA8E7603D40839DDD128
:109CE000917024E6D3780221DEB2D17016F0100212
:109CF00040F08387F60700F12487AD680220E87002
:109D00001BE60220D8708A68937843F0100595709E
:109D10008E68002737718A6842F2107092F803C08B
:109D20005FEA8C751ED492F803E05FEA8E7319D453
:109D3000D3789F0716D4D578AE0713D4D678B50755
:109D400010D4D778BB070DD492F803C05FEA8C77A4
:109D500008D492F803E05FEA8E7603D40838DDD1A8
:109D60009070A1E5D3780220DDB2D07015F010021A
:109D700040F0FF86EF0700F1F08689680227CF7078
:109D800098E50221D970AA68937843F0100696707E
:109D9000A86800270771AA6842F2107192F803E0E0
:109DA0005FEA8E761ED492F803C05FEA8C7019D4F5
:109DB000D3789F0716D4D678B60713D4D078800707
:109DC00010D4D778BB070DD492F803E05FEA8E7702
:109DD00008D492F803C05FEA8C7603D40839DDD149
:109DE00091702EE5D3780221DEB2D17016F0100208
:109DF00040F09986F30700F1E686AD680220E8702E
:109E000025E50220D8708A68937843F01005957094
:109E10008E68222737718A6842F2107092F803E048
:109E20005FEA8E731ED492F803C05FEA8C7719D470
:109E3000D3789F0716D4D578AE0713D4D678B50754
:109E400010D4D778BB070DD492F803E05FEA8E7781
:109E500008D492F803C05FEA8C7603D40838DDD1C9
:109E60009070ABE4D3780220DDB2D07015F0100210
:109E700040F09386EE0700F1848689680227CF7050
:109E8000A2E40221D970AA68937843F01006967074
:109E9000A86800270771AA6842F2107192F803C0FF
:109EA0005FEA8C731ED492F803E05FEA8E7719D4D0
:109EB000D3789F0716D4D678B60713D4D078800706
:109EC00010D4D778BB070DD492F803C05FEA8C7723
:109ED00008D492F803E05FEA8E7603D40839DDD126
:109EE000917038E4D3780221DEB2D17016F01002FE
:109EF00040F05B86F60700F1C486AD680220E8708A
:109F00002FE40220D8708A68937843F0100595708A
:109F10008E687F2737718A6842F2107092F803C00A
:109F20005FEA8C751FD492F803E05FEA8E731AD44F
:109F3000D3789F0717D4D578AE0714D4D678B50751
:109F400011D4D778BB070ED492F803C05FEA8C77A0
:109F500009D492F803E05FEA8E7604D40838DDD1A4
:109F60009070FFF7B5BBD3780220DDB2D07015F04A
:109F7000100240F09886EF0700F189868968022771
:109F8000CF70FFF7ABBB0221D970AA68937843F07A
:109F900010069670A86800270771AA6842F210712F
:109FA00092F803E05FEA8E761FD492F803C05FEA6E
:109FB0008C701AD4D3789F0717D4D678B60714D4E8
:109FC000D078800711D4D778BB070ED492F803E07D
:109FD0005FEA8E7709D492F803C05FEA8C7604D4E6
:109FE0000839DDD19170FFF740BBD3780221DEB292
:109FF000D17016F0100240F07485F30700F133863B
:10A00000AD680220E870FFF736BB0220D8708A687E
:10A01000937843F0100595708E68002737718A6831
:10A0200042F2107092F803E05FEA8E731FD492F848
:10A0300003C05FEA8C771AD4D3789F0717D4D578FA
:10A04000AE0714D4D678B50711D4D778BB070ED491
:10A0500092F803E05FEA8E7709D492F803C05FEAD2
:10A060008C7604D40838DDD19070FFF7BBBAD37872
:10A070000220DDB2D07015F0100240F0DE85EE0750
:10A0800000F1CF8589680227CF70FFF7B1BA0221AE
:10A09000D970AA68937843F010069670A8680027D4
:10A0A0000771AA6842F2107192F803C05FEA8C73DC
:10A0B0001FD492F803E05FEA8E771AD4D3789F0713
:10A0C00017D4D678B60714D4D078800711D4D778AF
:10A0D000BB070ED492F803C05FEA8C7709D492F8DC
:10A0E00003E05FEA8E7604D40839DDD19170FFF782
:10A0F00046BAD3780221DEB2D17016F0100240F0D9
:10A10000A485F60700F1D785AD680220E870FFF757
:10A110003CBA0220D8708A68937843F01005957095
:10A120008E68212737718A6842F2107092F803C056
:10A130005FEA8C751FD492F803E05FEA8E731AD43D
:10A14000D3789F0717D4D578AE0714D4D678B5073F
:10A1500011D4D778BB070ED492F803C05FEA8C778E
:10A1600009D492F803E05FEA8E7604D40838DDD192
:10A170009070FFF7C1B9D3780220DDB2D07015F02E
:10A18000100240F0AA85EF0700F19B85896802273D
:10A19000CF70FFF7B7B9DE78B5067FF5C0A993F8A1
:10A1A00003C05FEA8C657FF5BAA993F803E05FEA24
:10A1B0008E627FF5B4A9DA7897067FF5B0A9DF78CB
:10A1C000BE067FF5ACA9DD78AD067FF5A8A9DE78DF
:10A1D000B2067FF5A4A908387FF49DA998708B6812
:10A1E0008020987000BF256801220A7395F86410DA
:10A1F00000297FF49AA928462679F8F7EFFD002870
:10A2000037D0AF6897F802C04CF03003BB70AA6833
:10A2100042F21071D078800600F10183D778BB0636
:10A2200000F1FD8292F803E05FEA8E6000F1F782B0
:10A2300092F803C05FEA8C6300F1F182D3789F0645
:10A2400000F1ED82D078800600F1E982D778BB0674
:10A2500000F1E58292F803E05FEA8E6700F1DF82A9
:10A260000839D7D19170AB6880229A7000BF01265F
:10A270002E732568FFF759B9DE78B2067FF5B1AACB
:10A2800093F803E05FEA8E657FF5ABAA93F803C00D
:10A290005FEA8C627FF5A5AADA7897067FF5A1AA16
:10A2A000DF78BE067FF59DAADD78AD067FF599AA19
:10A2B000DE78B2067FF595AA08387FF48EAA9870EA
:10A2C0008B688020987000BF256801220A7395F87A
:10A2D000641000297FF48BAA28462679F8F77EFDC2
:10A2E000002837D0AF6897F802E04EF03003BB701B
:10A2F000AA6842F21071D078830600F1BE82D77846
:10A30000BF0600F1BA8292F803C05FEA8C6000F1E8
:10A31000B48292F803E05FEA8E6300F1AE82D378F4
:10A320009F0600F1AA82D078800600F1A682D77835
:10A33000BB0600F1A28292F803C05FEA8C6700F1CD
:10A340009C820839D7D19170AB6880229A7000BF87
:10A3500001262E732568FFF74ABADE78B5067FF529
:10A36000B6AA93F803C05FEA8C657FF5B0AA93F8AC
:10A3700003E05FEA8E627FF5AAAADA7897067FF596
:10A38000A6AADF78BE067FF5A2AADD78AD067FF526
:10A390009EAADE78B2067FF59AAA08387FF493AABF
:10A3A00098708B688020987000BF256801220A731E
:10A3B00095F8641000297FF490AA28462679F8F7CA
:10A3C0000DFD002837D0AF6897F802C04CF030037D
:10A3D000BB70AA6842F21071D078800600F17B82CF
:10A3E000D778BB0600F1778292F803E05FEA8E60CF
:10A3F00000F1718292F803C05FEA8C6300F16B8216
:10A40000D3789F0600F16782D078800600F16382DE
:10A41000D778BB0600F15F8292F803E05FEA8E67AF
:10A4200000F159820839D7D19170AB6880229A70B7
:10A4300000BF01262E732568FFF74FBADE78B206FB
:10A440007FF5E3A893F803E05FEA8E657FF5DDA86A
:10A4500093F803C05FEA8C627FF5D7A8DA78970695
:10A460007FF5D3A8DF78BE067FF5CFA8DD78AD06EF
:10A470007FF5CBA8DE78B2067FF5C7A808387FF451
:10A48000C0A898708B688020987000BF2568012252
:10A490000A7395F8641000297FF4BDA82846267930
:10A4A000F8F79CFC002837D0AF6897F802E04EF030
:10A4B0003003BB70AA6842F21071D078830600F1B5
:10A4C0003882D778BF0600F1348292F803C05FEA81
:10A4D0008C6000F12E8292F803E05FEA8E6300F157
:10A4E0002882D3789F0600F12482D078800600F17C
:10A4F0002082D778BB0600F11C8292F803C05FEA85
:10A500008C6700F116820839D7D19170AB68802230
:10A510009A7000BF01262E732568FFF77CB8DE789D
:10A52000B5067FF5E8A893F803C05FEA8C657FF570
:10A53000E2A893F803E05FEA8E627FF5DCA8DA78A0
:10A5400097067FF5D8A8DF78BE067FF5D4A8DD781A
:10A55000AD067FF5D0A8DE78B2067FF5CCA8083826
:10A560007FF4C5A898708B688020987000BF25681C
:10A5700001220A7395F8641000297FF4C2A82846C6
:10A580002679F8F72BFC002837D0AF6897F802C07F
:10A590004CF03003BB70AA6842F21071D07880068C
:10A5A00000F1E280D778BB0600F1DE8092F803E08C
:10A5B0005FEA8E6000F1D88092F803C05FEA8C6396
:10A5C00000F1D280D3789F0600F1CE80D07880064B
:10A5D00000F1CA80D778BB0600F1C68092F803E08C
:10A5E0005FEA8E6700F1C0800839D7D19170AB68FF
:10A5F00080229A7000BF01262E732568FFF781B86C
:10A60000DE78B2067FF5D9A993F803E05FEA8E659C
:10A610007FF5D3A993F803C05FEA8C627FF5CDA9DB
:10A62000DA7897067FF5C9A9DF78BE067FF5C5A958
:10A63000DD78AD067FF5C1A9DE78B2067FF5BDA94C
:10A6400008387FF4B6A998708B688020987000BF96
:10A65000256801220A7395F8641000297FF4B3A9D4
:10A6600028462679F8F7BAFB002836D0AF6897F865
:10A6700002E04EF03003BB70AA6842F21071D0784D
:10A68000830600F19F80D778BF0600F19B8092F887
:10A6900003C05FEA8C6000F1958092F803E05FEA06
:10A6A0008E6300F18F80D3789F0600F18B80D07885
:10A6B000800600F18780D778BB0600F1838092F88E
:10A6C00003C05FEA8C677DD40839D8D19170AB683C
:10A6D00080229A7000BF01262E732568FFF773B998
:10A6E0009079AB4E40F0500191719A681227D77063
:10A6F0009C68A07840F01001A1701A6E11680020CB
:10A70000C871D2F800E001276C1C0C608F80CEF875
:10A710000870146840F2FF3CA4F81EC01268E6609E
:10A72000A2F816C01E6E9F6831680437B7F1804FDB
:10A730000F618882887180F0C28132680124946040
:10A7400032681E6E934F00219161307938709C6899
:10A7500094F802C04CF00102A2709E682D78357109
:10A76000012783F86470F8BD7600F1B21171AB680F
:10A7700042F21072D87887073FF53FAFDF78BE0707
:10A780003FF53BAFDE78B7073FF537AF93F803C02F
:10A790005FEA8C763FF531AF93F803E05FEA8E70A5
:10A7A0003FF52BAFD97889073FF527AFD8788707D2
:10A7B0003FF523AFDF78BE073FF51FAF083AD9D189
:10A7C0009A7014E77600F1B21171AB6842F2107220
:10A7D000D878800781D4DF78B9073FF57EAFDE787F
:10A7E000B7073FF57AAF93F803E05FEA8E763FF55F
:10A7F00074AF93F803C05FEA8C703FF56EAFD97801
:10A8000089073FF56AAFD87887073FF566AFDF78ED
:10A81000BE073FF562AF083ADAD19A7057E7760083
:10A82000F1B21171AB6842F21072D87887073FF528
:10A8300020ADDF78BE073FF51CADDE78B7073FF5EA
:10A8400018AD93F803C05FEA8C763FF512AD93F82C
:10A8500003E05FEA8E703FF50CADD97889073FF5CC
:10A8600008ADD87887073FF504ADDF78BE073FF520
:10A8700000AD083AD9D19A70F5E47600F1B21171C1
:10A88000AB6842F21072D87880073FF563ADDF788D
:10A89000B9073FF55FADDE78B7073FF55BAD93F8DD
:10A8A00003E05FEA8E763FF555AD93F803C05FEAAB
:10A8B0008C703FF54FADD97889073FF54BADD8780F
:10A8C00087073FF547ADDF78BE073FF543AD083A50
:10A8D000D9D19A7038E57600F1B21171AB6842F2C5
:10A8E0001072D87887073FF5A6ADDF78BE073FF531
:10A8F000A2ADDE78B7073FF59EAD93F803C05FEADF
:10A900008C763FF598AD93F803E05FEA8E703FF5E3
:10A9100092ADD97889073FF58EADD87887073FF596
:10A920008AADDF78BE073FF586AD083AD9D19A7077
:10A930007BE57600F1B21171AB6842F21072D87803
:10A9400080073FF5E9ADDF78B9073FF5E5ADDE7883
:10A95000B7073FF5E1AD93F803E05FEA8E763FF588
:10A96000DBAD93F803C05FEA8C703FF5D5ADD978C5
:10A9700089073FF5D1ADD87887073FF5CDADDF78B2
:10A98000BE073FF5C9AD083AD9D19A70BEE500BF00
:10A9900001FCFFFF1B8000407F00F9B21171AB6822
:10A9A00042F21072D878800723D4DF78B90720D418
:10A9B00093F803C05FEA8C701BD493F803E05FEA5E
:10A9C0008E7116D4D9788F0713D4D878800710D415
:10A9D000DF78B9070DD493F803C05FEA8C7708D409
:10A9E000083ADFD19A70AB6880229A7000BF0121CB
:10A9F00029732568FEF79CB928462779F8F7EEF900
:10AA0000002859D0A86890F802E04EF03003837017
:10AA1000AA6842F21071D078800620D492F803C060
:10AA20005FEA8C631BD492F803E05FEA8E6016D471
:10AA3000D3789B0613D4D078800610D492F803C044
:10AA40005FEA8C630BD492F803E05FEA8E6006D471
:10AA5000D3789B0603D40839DDD1917026E07F00BE
:10AA6000F9B21171AB6842F21072D878800723D422
:10AA7000DF78B90720D493F803C05FEA8C701BD449
:10AA800093F803E05FEA8E7116D4D9788F0713D458
:10AA9000D878800710D4DF78B9070DD493F803C0B5
:10AAA0005FEA8C7708D4083ADFD19A70AB688022CD
:10AAB0009A7000BF012129732568FEF7DFB932685B
:10AAC000906800287FF43DAE38E6AB680127DF7060
:10AAD00000BFA86829738270AB6880279F70FEF75B
:10AAE000BCB8A9681026CE7000BFAB680321002255
:10AAF00029739A70AF688022BA70FFF781BA8F68A5
:10AB00000125FD7000BF8B6808739A708F688022E2
:10AB1000BA70FFF732B888681026C67000BF0320ED
:10AB20008B680022F0E7A9681026CE7000BFAB68E2
:10AB30000321002229739A70AF688022BA70FFF750
:10AB40005CB9AF680120F87000BFAB6829739A70D8
:10AB5000AF688022BA70FFF7D0B88E680127F7700F
:10AB600000BF8B6808739A708E688022B270FFF7FE
:10AB700004B988681025C57000BF03208B680022C7
:10AB8000F0E78E680127F77000BF8B6808739A7032
:10AB90008E688022B270FFF770B988681025C57082
:10ABA00000BF03208B680022F0E7A9681026CE7052
:10ABB00000BFAB680321002229739A70AF6880221E
:10ABC000BA70FFF79AB9AF680120F87000BFAB68A0
:10ABD000B0E78E680127F77000BF8B6808739A7022
:10ABE0008E688022B270FFF748B888681025C5705B
:10ABF00000BF03208B680022F0E7A9681026CE7002
:10AC000000BF0321AB680022A0E7AF680120F87005
:10AC100000BFAB6829739A70AF688022BA70FEF7E4
:10AC2000ECBF8E680127F77000BF8B6808739A70BD
:10AC30008E688022B270FFF725BA88681025C5702B
:10AC400000BF03208B680022F0E7A9681026CE70B1
:10AC500000BFAB680321002229739A70AF6880227D
:10AC6000BA70FFF751BAAF680120F87000BFAB6847
:10AC70003EE7A9681026CE7000BF0321AB68002212
:10AC8000C8E7AF680120F87000BFAB6894E78E6832
:10AC90000127F77000BF8B6808739A708E68802256
:10ACA000B270FFF76BB988681025C57000BF03202C
:10ACB0008B680022F0E7AF680120F87000BFAB6836
:10ACC000CAE78E680127F77000BF8B6808739A7017
:10ACD0008E688022B270FFF759BA88681025C57057
:10ACE00000BF03208B680022F0E788681022C27042
:10ACF00000BF8F68032000220873BA708B6880251C
:10AD00009D70FDF7FDBFA9681022CA7000BF032126
:10AD1000A8680022DEE6A9681022CA7000BFA868F1
:10AD20000321002229738270AB6880279F70FEF791
:10AD3000E8B8A9681022CA7000BFA86803210022E1
:10AD400029738270AB6880279F70FEF734B88868DB
:10AD50001022C27000BF8F68032000220873BA70EF
:10AD60008B6880259D70FEF76CB888681025C570CB
:10AD700000BF8B680320002208739A708E688022BF
:10AD8000B270FEF702B98B680125DD7000BF8F68D5
:10AD9000E4E78E680127F77000BF8B68ECE7AB68CB
:10ADA0000127DF7000BFA868CAE78B680125DD7046
:10ADB00000BF8F68A0E7AB680127DF7000BFA868FD
:10ADC000B0E700BF8368196891F8641001B170475B
:10ADD00010B5044604484FF4004200680DF098F99D
:10ADE000A068FDF7E1FE10BDACA8022010B4036816
:10ADF00041681A7890F809C00C78037A14EA0C0FAD
:10AE000002EA03021DD0847A04F003010AB141F082
:10AE1000040141F008039A1003F1FF3C8272BCF177
:10AE20000D0F0BD8DFE80CF021071B070A152121B5
:10AE3000150A071B0721C268531EC3605DF8044B47
:10AE40007047817A01F00303002AE4D043F0040341
:10AE5000E1E7C3689C1EC4605DF8044B7047C1689D
:10AE60005DF8044B0231C1607047C4680134C460AE
:10AE70005DF8044B704700BF08B5034BD3F8B8002A
:10AE8000FFF7B4FF08BD00BFB8A8022008B5034B08
:10AE9000D3F8B400FFF7AAFF08BD00BFB8A802208E
:10AEA00008B5034BD3F8B000FFF7A0FF08BD00BF03
:10AEB000B8A8022008B5034BD3F8AC00FFF796FF03
:10AEC00008BD00BFB8A8022008B5034BD3F8A800FE
:10AED000FFF78CFF08BD00BFB8A8022008B5034BE0
:10AEE000D3F8A400FFF782FF08BD00BFB8A8022076
:10AEF00008B5034BD3F8A000FFF778FF08BD00BFEB
:10AF0000B8A8022008B5034BD3F89C00FFF76EFFEA
:10AF100008BD00BFB8A8022008B5034BD3F89800BD
:10AF2000FFF764FF08BD00BFB8A8022008B5034BB7
:10AF3000D3F89400FFF75AFF08BD00BFB8A802205D
:10AF400008B5034BD3F89000FFF750FF08BD00BFD2
:10AF5000B8A8022008B5034BD3F88C00FFF746FFD2
:10AF600008BD00BFB8A8022008B5034BD3F888007D
:10AF7000FFF73CFF08BD00BFB8A8022008B5034B8F
:10AF8000D3F88400FFF732FF08BD00BFB8A8022045
:10AF900008B5034BD3F88000FFF728FF08BD00BFBA
:10AFA000B8A8022008B5024BD86FFFF71FFF08BDF5
:10AFB000B8A8022008B5024B986FFFF717FF08BD2D
:10AFC000B8A8022008B5024B586FFFF70FFF08BD65
:10AFD000B8A8022008B5024B186FFFF707FF08BD9D
:10AFE000B8A8022008B5024BD86EFFF7FFFE08BDD7
:10AFF000B8A8022008B5024B986EFFF7F7FE08BD0F
:10B00000B8A8022008B5024B586EFFF7EFFE08BD46
:10B01000B8A8022008B5024B186EFFF7E7FE08BD7E
:10B02000B8A8022008B5024BD86DFFF7DFFE08BDB7
:10B03000B8A8022008B5024B986DFFF7D7FE08BDEF
:10B04000B8A8022008B5024B586DFFF7CFFE08BD27
:10B05000B8A8022008B5024B186DFFF7C7FE08BD5F
:10B06000B8A8022008B5024BD86CFFF7BFFE08BD98
:10B07000B8A8022008B5024B986CFFF7B7FE08BDD0
:10B08000B8A8022008B5024B586CFFF7AFFE08BD08
:10B09000B8A8022008B5024B186CFFF7A7FE08BD40
:10B0A000B8A8022008B5024BD86BFFF79FFE08BD79
:10B0B000B8A8022008B5024B986BFFF797FE08BDB1
:10B0C000B8A8022008B5024B586BFFF78FFE08BDE9
:10B0D000B8A8022008B5024B186BFFF787FE08BD21
:10B0E000B8A8022008B5024BD86AFFF77FFE08BD5A
:10B0F000B8A8022008B5024B986AFFF777FE08BD92
:10B10000B8A8022008B5024B586AFFF76FFE08BDC9
:10B11000B8A8022008B5024B186AFFF767FE08BD01
:10B12000B8A8022008B5024BD869FFF75FFE08BD3A
:10B13000B8A8022008B5024B9869FFF757FE08BD72
:10B14000B8A8022008B5024B5869FFF74FFE08BDAA
:10B15000B8A8022001380B463A2800F25C82DFE8EA
:10B1600010F053024C0245023E023702300229021F
:10B1700022021B02AE01A701A001990192018B01DD
:10B1800084017D0176016F01680161015A0153015B
:10B190004C0145013E0137013001290122011B010B
:10B1A00013010B010301FB00F300EB00E300DB00E4
:10B1B000D300CB00C300BB00B300AB00A3009B00D7
:10B1C00093008B0083007B0073006B0063005B00C7
:10B1D00053004B0043003B00BC4ABD49C2F8EC3071
:10B1E0003B20042209F036BDB848BA49C0F8E8301F
:10B1F00004223A2009F02EBDB44AB749C2F8E4301F
:10B200003920042209F026BDB048B449C0F8E03026
:10B210000422382009F01EBDAC4AB149C2F8DC3026
:10B220003720042209F016BDA848AE49C0F8D8302E
:10B230000422362009F00EBDA44AAB49C2F8D4302E
:10B240003520042209F006BDA048A849C0F8D03036
:10B250000422342009F0FEBC9C4AA549C2F8CC3037
:10B260003320042209F0F6BC9848A249C0F8C8303F
:10B270000422322009F0EEBC944A9F49C2F8C4303F
:10B280003120042209F0E6BC90489C49C0F8C03047
:10B290000422302009F0DEBC8C4A9949C2F8BC3047
:10B2A0002F20042209F0D6BC88489649C0F8B8304F
:10B2B00004222E2009F0CEBC844A9349C2F8B4304F
:10B2C0002D20042209F0C6BC80489049C0F8B03057
:10B2D00004222C2009F0BEBC7C4A8D49C2F8AC3057
:10B2E0002B20042209F0B6BC78488A49C0F8A8305F
:10B2F00004222A2009F0AEBC744A8749C2F8A4305F
:10B300002920042209F0A6BC70488449C0F8A03066
:10B310000422282009F09EBC6C4A8149C2F89C3066
:10B320002720042209F096BC68487E49C0F898306E
:10B330000422262009F08EBC644A7B49C2F894306E
:10B340002520042209F086BC60487849C0F8903076
:10B350000422242009F07EBC5C4A7549C2F88C3076
:10B360002320042209F076BC58487249C0F888307E
:10B370000422222009F06EBC544A6F49C2F884307E
:10B380002120042209F066BC50486C49C0F8803086
:10B390000422202009F05EBC4C4A6949D3671F2073
:10B3A000042209F057BC49486649836704221E20DD
:10B3B00009F050BC454A644953671D20042209F036
:10B3C00049BC42486149036704221C2009F042BC81
:10B3D0003E4A5F49D3661B20042209F03BBC3B4830
:10B3E0005C49836604221A2009F034BC374A5A4962
:10B3F00053661920042209F02DBC344857490366CE
:10B400000422182009F026BC304A5549D36517207C
:10B41000042209F01FBC2D485249836504221620DE
:10B4200009F018BC294A504953651520042209F037
:10B4300011BC26484D4903650422142009F00ABCBA
:10B44000224A4B49D3641320042209F003BC1F484D
:10B45000484983640422122009F0FCBB1B4A464978
:10B4600053641120042209F0F5BB184843490364D2
:10B470000422102009F0EEBB144A4149D3630F2087
:10B48000042209F0E7BB11483E49836304220E20E1
:10B4900009F0E0BB0D4A3C4953630D20042209F03A
:10B4A000D9BB0A483949036304220C2009F0D2BBF6
:10B4B000064A3749D3620B20042209F0CBBB03486C
:10B4C0003449836204220A2009F0C4BBB8A80220D0
:10B4D000B91B0000251B0000911A0000FD19000097
:10B4E00069190000D518000041180000AD170000D0
:10B4F0001917000085160000F11500005D15000009
:10B50000C914000079AE00008DAE0000A1AE0000AD
:10B51000B5AE0000C9AE0000DDAE0000F1AE000027
:10B5200005AF000019AF00002DAF000041AF0000D3
:10B5300055AF000069AF00007DAF000091AF000083
:10B54000A5AF0000B5AF0000C5AF0000D5AF00004B
:10B55000E5AF0000F5AF000005B0000015B0000039
:10B5600025B0000035B0000045B0000055B0000027
:10B5700065B0000075B0000085B0000095B0000017
:10B58000A5B00000B5B00000C5B00000D5B0000007
:10B59000E5B00000F5B000001F4A204953620920C1
:10B5A000042209F057BB1C481D49036204220820ED
:10B5B00009F050BB184A1B49D3610720042209F047
:10B5C00049BB1548184983610422062009F042BB93
:10B5D000114A164953610520042209F03BBB0E486D
:10B5E000134903610422104609F034BB0A4A114989
:10B5F000D3600320042209F02DBB07480E49836065
:10B600000422022009F026BB034A0C4953600120A2
:10B61000042209F01FBB7047B8A8022005B1000042
:10B6200015B1000025B1000035B1000045B10000A2
:10B63000091E0000751D0000E11C00004D1C0000EB
:10B640002DE9F04F8B0903F180428BB0541EA50009
:10B650000695069E8768864ADFF858A23744079702
:10B6600013680993099D06E016680896089F7C1BDD
:10B67000642C00F2F9809AF8006006F0FF04002EB6
:10B68000F2D18B4600F508411C317A4FDFF8009269
:10B69000794E039001940091CDF814B0079B039A62
:10B6A000019C00981568DFF810B2049523440293BA
:10B6B000C0F800387149724DD1F8008009F09CFF44
:10B6C000044604E009F098FF021BAA42F2D833684E
:10B6D000D907F7D46B4A6C48C2F80080CBF8000059
:10B6E00009F08AFF664C054604E009F085FF431B1C
:10B6F000A342DFD83968654B0B40002BF5D05D487D
:10B700005C4A0568C9F800501560D9F800405F4BE5
:10B710005F492340012BCDD15E480568EA05C9D5B4
:10B7200000240C605C495D4A08788AF80030009B70
:10B73000136010B9029D6A020292594C594B51494B
:10B740000298594D594A086025601A60584BA36009
:10B7500009F052FF4A4D044604E009F04DFF031B77
:10B76000AB4279D89AF800100029F6D1D9F8000038
:10B770004E4A0240022A6FD1019D009C043504F616
:10B7800008010C2D0195009188D1DDF814C0039EAD
:10B790000CF03F0706F5843807EE907A08F5DE7462
:10B7A00006F5023AB8EEE70A04F580390AF52F7B70
:10B7B00001205C4588ED6D0AC8F8B801B646C9F8A5
:10B7C00000C138D0039A02F58C3303F5E6754FF0CB
:10B7D000FF3655F810ECBEF1000F30D00EF1FF30FF
:10B7E0000021814212D20F187A0854F832309C4559
:10B7F0002AD006D92BE054F83370BC4525D028D880
:10B800001A4650188A424FEA5003F4D854F831309F
:10B810009C4500D901318E458CBF0B46334601391A
:10B8200005E90A0004F58054103405F58055A34558
:10B8300005F11005CDD100200BB0BDE8F08F45F823
:10B84000086C45F8046CEDE71346591CE3E7134612
:10B850000246591C1046C4E704984FF4F472312193
:10B8600008F0C6FE002887D105200BB0BDE8F08F98
:10B8700000AB022030100B4024100B40D8AA02204D
:10B8800040420F0008100B4000001A0D01000F008D
:10B89000DCAA022010100B40CCAA022000100B40A2
:10B8A00004100B4038100B400002040002007F110E
:10B8B00037003A12E0AA02200C100B404F2901D9A0
:10B8C000082070472DE9F04FAB4AAC4C136889B0A3
:10B8D0000793079D06E016680696069F7B1B642B60
:10B8E00000F22681277807F0FF06002FF3D1A44B42
:10B8F0000591054603FB01F303F108014C33029067
:10B9000005F114020068AB6069604423F7F7BEF8E4
:10B91000002800F00D8105F5843C0196DCF8B0416B
:10B92000009604F5004704F5FF4B3C37314604947C
:10B930000CF5E47C0BF17C0A0397A14601265AF82A
:10B94000043FB3F5807F00F2EF804FEA4308CCF864
:10B95000F48FCCF8F88F002B00F084800198049CC1
:10B96000034404EBC30EC9EB0E02A2F1080799E8E9
:10B970001400ACF10C0B4CF80C2C09F108024FF040
:10B98000FF3372452CF8086C2CF8061C4CF8044C5C
:10B99000C7F3C105ABF80C30ACF802100CF104038E
:10B9A00060D05DB3012D1AD0022D0CD092E81100A9
:10B9B00018604FF0FF309E80D9809C609881D981BB
:10B9C00008320CF1140392E811009C604FF0FF3430
:10B9D00018609E80D9809C81D9810832103392E80A
:10B9E000110008324FF0FF37724518609E80D980F1
:10B9F0009C609F81D98103F1100333D01568D2F880
:10BA00000CB0506894681D604FF0FF3715699F8136
:10BA100003F120071C611D62546998604FF0FF35E7
:10BA2000C3F818B09E80D2F818B0D980D9819E8210
:10BA3000D9829D83D98303F13000BC60203252F853
:10BA4000044CBE807245F980BD81F98103F1400349
:10BA500043F810BC23F80C6C23F80A1C8460858121
:10BA6000C181CBD1B8F1000F66D03CF908EC5CF88D
:10BA70000C0CBEF1010F57D1009A029D02F5045340
:10BA80003833434405EBC307CCEB0708C8F3C104C4
:10BA90006346724604B35CF804BC834544D36346F2
:10BAA00033F9082B501C3FD1012C584614D0022CDE
:10BAB00008D053F8045C5D4536D333F9082B724542
:10BAC00032D1284653F8044C84422DD333F9080B65
:10BAD000D04229D102462046BB421D4603F1180E32
:10BAE0002AD053F8048C804503F120031CD335F988
:10BAF000084BD442AB4617D155F8042C424513D31A
:10BB00003BF9080BE0420FD15BF8048C90450BD356
:10BB1000B5F90850C54207D15EF8040C404503D37F
:10BB2000BEF90020EA42D7D0102009B0BDE8F08F5E
:10BB3000052009B0BDE8F08F009F019C03980CF52B
:10BB4000805C07F2022304F5807582450CF1100C2D
:10BB5000009309F5006901957FF4F1AE029E059FFF
:10BB6000326802EB870A3046DAF840303361F7601A
:10BB70000021FFF765FDDCE700AB0220E0AA022010
:10BB8000796E01002DE9F04FD0F84C6A90F8A65A72
:10BB900091B004463046F7F721F920B3B2689378A4
:10BBA00043F030009070B26842F21071D778BF064F
:10BBB0000AD492F803905FEA896005D492F803A052
:10BBC0005FEA8A6740F13A846D0045F00101CFB227
:10BBD0001771B36842F21072D878810703D4DD7808
:10BBE000AF0740F1BC83D4F84C3A5E7B012E00F0E5
:10BBF000E883986D5D6DA842C0F004830023D4F8FB
:10BC0000A86A84F8A43A304694F8025BF7F7E6F89D
:10BC100020B3B268917841F030079770B26842F271
:10BC20001071D07887060AD492F803A05FEA8A6080
:10BC300005D492F803B05FEA8B6040F103836D0096
:10BC400045F00101C8B21071B36842F21072DF789A
:10BC5000B90703D4DD78AF0740F15A83D4F8A83A86
:10BC60005E7B012E00F018839F6D5D6DAF42C0F0CA
:10BC7000C482002304F6A45604F6D45A564584F828
:10BC8000003BB54D73D0B54FA9464FF0000B4FF0B8
:10BC9000010856F8040B02681168B94240F0A98205
:10BCA0008369027F93F85830D5F800C00169CDF858
:10BCB00028C0134103F001020A9B002900F077829B
:10BCC000591A4368994208D3002A00F0B282C0F89A
:10BCD00010B080F814B080F815B0306802681168B0
:10BCE000B94240F072828369027F93F85830D5F8E8
:10BCF00000E00169CDF828E0134103F001020A9B3E
:10BD0000002900F06482591A4368994208D3002A36
:10BD100000F08682C0F810B080F814B080F815B03A
:10BD2000706802681168B94206F1080640F0638243
:10BD30008369027F93F85830D5F800C00169CDF8C7
:10BD400028C0134103F001020A9B002900F0488239
:10BD5000591A4368994208D3002A00F05882C0F863
:10BD600010B080F814B080F815B0B24591D194F8B5
:10BD7000380C94F858AC94F8987C94F8D86C94F8F3
:10BD8000782D94F858BD94F8983D94F8591C94F87F
:10BD9000789C84F87C0094F8F8EC94F8390C84F8DA
:10BDA0007DA094F818CD84F8807094F838AD94F89C
:10BDB000B87C84F8816084F8852094F8996D94F8B3
:10BDC000D92C84F87FB084F8843084F8877084F8A4
:10BDD000880084F88A1084F88B6084F8892084F8BD
:10BDE0007E9084F883E084F882C084F886A094F87A
:10BDF000799D2B680F93D4F8386E0F9FD4F8E42DFB
:10BE000094F839BD94F8B90C84F88C90B91B914220
:10BE100084F88DB084F88E0004F158064E4B40F241
:10BE2000F58672B6D4F8F42D62B61F680B970B9F97
:10BE3000D4F8081ED4F80C0E9308181AA7EB0101C9
:10BE4000C4F80C3ED4F8103E18BFC4F8087E01298F
:10BE5000B8BF0121820292FBF1F7002B40F00D8365
:10BE600003EB4301CF1948BF0337BB1083EAE37EDE
:10BE7000AEEBE37C3A49ACF1020A81FB0A72A2EB19
:10BE8000EA777A1CD4F8141EC4F8103E00FB0210A6
:10BE9000C4F8140E72B6D4F8F41D62B62B680C9375
:10BEA0000C9FD4F8182ED4F81C0E8908BB1AC4F8BD
:10BEB0001C1ED4F8202E091A18BFC4F8187E012BB6
:10BEC000B8BF01238F0297FBF3F0002A40F0FA82FB
:10BED00002EB42073A1848BF0332901080EAE0793B
:10BEE000A9EBE07BABF10203012BC4F8200E40F379
:10BEF000EB879F10A7F1040CA7F10B022CEAEC7E54
:10BF0000002AA8BF96440137BE44D4F8240E01FB92
:10BF10000E01C4F8241E72B6D4F8F43D62B62F6840
:10BF20000D970D9FD4F8282ED4F82C0E9B08B91A23
:10BF3000C4F82C3ED4F8302E1B1A18BFC4F8287E43
:10BF40000129B8BF01219F0297FBF1F052B10028EF
:10BF500040F06B8706E000BF00AB0220DD0A000066
:10BF6000ABAAAA2A02EB4207381848BF0330811057
:10BF700081EAE17AAAEBE179A9F10202012AC4F887
:10BF8000301E40F3B4879710A7F10B00391F20EA49
:10BF9000E07B0029A8BF8B4401375F44012F00F0EC
:10BFA000A687BA00A2F1020E2F68D4F8341E0E97AD
:10BFB0000E98C4F8380E0EFB0313C4F8343ED4F8C0
:10BFC000147ED4F8242EC4F89830C4F89070C4F8C5
:10BFD000942072B6D4F8481E62B68808C4F89C0053
:10BFE00004F50B3A94F8600E09F0BCFADAF8EC317B
:10BFF000B0FA80F71A687909184684F8A01031461B
:10C00000166904F1A402B047DAF8EC0103689F68EE
:10C01000B84704F1F00904F1A00E234601269DE083
:10C0200028680790079A02F07F07402F40F2A98006
:10C0300093F8082B0A420CBF4FF0010E4FF0000E90
:10C040004FF0010CD3F8041BD3F80C0BBEF1000F1A
:10C0500040F0A48091F8597006FA00FA27EA0A0E17
:10C0600081F859E0D3F804ABD3F8101B9AF85920A3
:10C07000BCF1000F40F06B8406FA01F022EA0007E1
:10C080008AF85970DBF80410880603F1100340F1B8
:10C090005C8228680790079F07F07F02402A00F221
:10C0A000908293F809CBD3F80C0B1CEA010FD3F85C
:10C0B00004CB0CBF012100219CF8597006FA00F056
:10C0C00047EA00025FFA82FA8CF859A0D3F804CB51
:10C0D000D3F810EB9CF85970002940F0328406FA2E
:10C0E0000EF127EA01028CF85920DBF808108A06C5
:10C0F0000BF1080E03F1100B40F108822A68079239
:10C10000079F07F07F00402800F248829BF8098BC8
:10C11000DBF804ABDBF80C2B18EA010F0CBF012194
:10C1200000219AF8598006FA02F248EA02075FFAFB
:10C1300087FC8AF859C0DBF8042BDBF810CB92F8A7
:10C140005900002940F04A8206FA0CFB203320EA0D
:10C150000B07994582F8597000F04A82DEF8041006
:10C1600088060EF1040B3FF55BAFC80640F1F5837E
:10C170002A680892089FC7F3080ABAF5807F3FF63D
:10C1800057AF93F809EBD3F80C0B1EEA010FD3F865
:10C19000041B0CBF4FF0010C4FF0000C91F859201C
:10C1A00006FA00F042EA00075FFA87FE58E7002A25
:10C1B0007FF493ADD9F800100991099B03613068B1
:10C1C00002681168B9423FF48EAD8847A8E5002A9D
:10C1D0007FF4A6ADD9F800100991099B03619FE592
:10C1E000002A7FF4C2ADD9F800100991099B0361C0
:10C1F000BBE5884771E58847B7E5791C1F44996519
:10C200003B7D37E5411C18449965037DF7E482685E
:10C2100080F814808A428CBF002101214175A4E579
:10C22000826880F814808A428CBF00210121417508
:10C2300076E5826880F814808A428CBF0021012153
:10C2400041754AE592F803C05FEA8C633FF5F7ACAD
:10C2500092F803E05FEA8E673FF5F1AC92F8039045
:10C260005FEA89603FF5EBACD3789B063FF5E7AC1E
:10C27000D778BF063FF5E3AC08397FF4D2AC9170B4
:10C28000B0688023837000BFD4F8A83A01223273CB
:10C290005E7B012E7FF4E8AC00208DF803009DF852
:10C2A00003209A6842F21070D678360600F1B28404
:10C2B000D7783D0600F1AE84D5782D0600F1AA842A
:10C2C00092F803A05FEA0A6100F1A48492F803B037
:10C2D0005FEA0B6700F19E8492F803C05FEA0C6688
:10C2E00000F1988492F803E05FEA0E6500F1928411
:10C2F00092F803905FEA096100F18C840838D3D189
:10C3000090709F688025BD7000BF01201873B0E455
:10C3100093F803A05FEA8A773FF5A0AC93F803B0E7
:10C320005FEA8B753FF59AAC93F803C05FEA8C70B7
:10C330003FF594AC93F803E05FEA8E713FF58EAC65
:10C3400093F803905FEA89773FF588ACD9788D0739
:10C350003FF584AC083A7FF47AAC9A7090E793F892
:10C3600003905FEA89703FF53EAC93F803A05FEA63
:10C370008A713FF538AC93F803B05FEA8B773FF5ED
:10C3800032AC93F803C05FEA8C753FF52CAC93F8A0
:10C3900003E05FEA8E703FF526ACD97889073FF558
:10C3A00022AC083A7FF418AC9A70B7688023BB704F
:10C3B00000BFD4F84C3A012232735E7B012E7FF429
:10C3C00018AC00278DF802709DF802209A6842F29E
:10C3D0001070D678350600F18E84D578290600F1E4
:10C3E0008A8492F803905FEA096600F1848492F8E7
:10C3F00003A05FEA0A6500F17E8492F803B05FEA69
:10C400000B6100F1788492F803C05FEA0C6700F1D9
:10C41000728492F803E05FEA0E6600F16C84D178D2
:10C420000D0600F168840838D3D190709D6880278C
:10C43000AF7000BF01201873FFF7E0BB92F803B0A4
:10C440005FEA8B603FF5C0AB92F803C05FEA8C6394
:10C450003FF5BAAB92F803E05FEA8E673FF5B4AB05
:10C46000D37898063FF5B0ABD07883063FF5ACABF8
:10C4700008397FF49BAB917097E7002F3FF4F0AC45
:10C4800007EE907AB8EEE70AB5EEC00AF1EE10FAC0
:10C4900040F3478501EE903AB8EEE12AB5EEC02AA6
:10C4A000F1EE10FA3FF7DCAC09D4F7EE002A9FED6D
:10C4B0004A1AB4EE621AF1EE10FA3FF4D1AC01223E
:10C4C0000023DFE400283FF403AD03EE100AF8EE8A
:10C4D000C33AF5EEC03AF1EE10FA40F3E68405EE09
:10C4E000902AB8EEE56AB5EEC06AF1EE10FA3FF7B1
:10C4F000EFAC00F1E684F7EE006A9FED375AB4EE38
:10C50000665AF1EE10FA40F0DC84E1E4CA063CD44D
:10C510009BF8087B9BF8090B0F420CBF4FF00108FA
:10C520004FF0000808420CBF01210021DBF804ABEA
:10C53000DBF80C2BB8F1000F7FF4F3AD9AF85980BB
:10C5400006FA02F028EA000CF3E5C80630D493F8A6
:10C5500008AB93F8092B1AEA010F0CBF4FF0010A40
:10C560004FF0000A0A420CBF01210021D3F804CB8E
:10C57000D3F80C0BBAF1000F7FF49EAD9CF8592054
:10C5800006FA00FE22EA0E0A9EE52A680892089F33
:10C59000C7F30800B0F5807F7FF6B8AD9BF8087B45
:10C5A0000F420CBF4FF001084FF000080121BDE71A
:10C5B00028680890089FC7F30802B2F5807F7FF6CD
:10C5C00070AD93F8087B0F420CBF4FF0010A4FF09B
:10C5D000000A0121CAE700BF0000000001FA0CF1C7
:10C5E00001432033CFB2994582F859707FF4B6AD3C
:10C5F000D4F8E4309A0640F1DA822A680192019870
:10C6000000F07F01402940F2DE8294F8F82B1A42B4
:10C610000CBF012200220126D4F8F41BD4F8FC0B35
:10C62000002A40F0DA8291F859800122824028EAFB
:10C63000020A81F859A0D4F8F42BD4F8007C002E1B
:10C6400040F0DC82012192F859C0B9402CEA010B7C
:10C6500082F859B0D4F8E070B80640F179822A68BF
:10C660000392039901F07F03402B40F27D8294F8FE
:10C67000182C3A420CBF012200220126D4F8141CC7
:10C68000D4F81C0C002A40F0798291F85920012737
:10C69000874022EA070881F85980D4F8142CD4F88E
:10C6A000207C002E40F07B82012192F859A0B940F5
:10C6B0002AEA010C82F859C0D4F8E8309A0640F111
:10C6C00018822D680595059A02F07F07402F40F2E9
:10C6D0001C8294F8085C1D420CBF01250025012630
:10C6E000D4F8047CD4F80C0C002D40F0188297F894
:10C6F00059B0012585402BEA050987F85990D4F8EF
:10C70000047CD4F8100C002E40F01A82012697F811
:10C710005950864025EA060804F6DC0A04F604317E
:10C720008A4587F8598000F0098104F63813CC1A3D
:10C73000D64FA00807FB00F727F040465C2505FB15
:10C7400006A7B837B0248025012602214FF0100E2D
:10C750004FF0030C4FF0000853F85C0C13F8029CE8
:10C76000826842F2107B92F803A01AF0200F00F0CA
:10C77000078192F803A01AF0200F00F0018192F8CF
:10C7800003A01AF0200F00F0FB8092F803A01AF02B
:10C79000200F00F0F58092F803A01AF0200F00F0AF
:10C7A000EF8092F803A01AF0200F00F0E98092F8D1
:10C7B00003A01AF0200F00F0E38092F803A01AF013
:10C7C000200F00F0DD80BBF1080BCCD182F802B065
:10C7D0008268957000BF8268067392F802A04AF0E2
:10C7E000300B82F802B0826842F2107B92F803A00C
:10C7F0001AF0200F23D192F803A01AF0200F1ED1B7
:10C8000092F803A01AF0200F19D192F803A01AF0A1
:10C81000200F14D192F803A01AF0200F0FD192F834
:10C8200003A01AF0200F0AD192F803A01AF0200FEB
:10C8300005D192F803A01AF0200F00F031834FEADF
:10C8400049095FFA89FB82F804B0826842F21079E4
:10C8500092F803A01AF0020F1ED192F803B01BF059
:10C86000020F19D192F803A01AF0020F14D192F816
:10C8700003B01BF0020F0FD192F803A01AF0020FC1
:10C880000AD192F803B01BF0020F05D192F803A071
:10C890001AF0020F00F0E88253F85C2C906842F224
:10C8A000107A90F803B01BF0800F40F0A68090F84B
:10C8B000039019F0800F40F0A08090F803B01BF0B7
:10C8C000800F40F09A8090F8039019F0800F40F0AC
:10C8D000948090F803B01BF0800F40F08E8090F8A9
:10C8E000039019F0800F40F0888090F803B01BF09F
:10C8F000800F40F0828090F8039019F0800F7CD177
:10C90000BAF1080ACDD180F802A09068857000BF06
:10C91000167353F85CBCDBF8080090F8029009F03D
:10C92000C7028270DBF8082042F2107AD0788006C5
:10C9300000F1AE805C339F427FF40EAF11B0BDE8D2
:10C94000F08F01FA0EF03843C2B2FFF7CCBB0CFAFD
:10C9500001F11143CFB2FFF793BB93F808EB93F8C3
:10C96000090B1EEA010F0CBF4FF0010E4FF0000E35
:10C9700008420CBF4FF0010C4FF0000CFFF762BBF8
:10C980009470826842F2107B92F803A01AF0200F94
:10C990002CD192F803A01AF0200F27D192F803A00F
:10C9A0001AF0200F22D192F803A01AF0200F1DD107
:10C9B00092F803A01AF0200F18D192F803A01AF0F1
:10C9C000200F13D192F803A01AF0200F0ED192F885
:10C9D00003A01AF0200F09D1BBF1080BD4D182F8C3
:10C9E00002B08268957000BF067355E792F803B0F5
:10C9F0001BF0200F3FF450AFEFE613F803BCC170FB
:10CA0000D2F808A09AF8020040F010098AF80290C3
:10CA1000906880F804B0D2F808B042F2107A9BF81F
:10CA200003905FEA89701FD49BF8030080071BD432
:10CA30009BF803905FEA897016D49BF80300800787
:10CA400012D49BF803905FEA89700DD49BF8030021
:10CA5000800709D49BF803905FEA897004D49BF89F
:10CA60000300800740F111829BF803A08BF80310AC
:10CA70005FFA8AFB1BF0100940F047825FEACB7037
:10CA800000F139829268D17043E700BFA737BD2912
:10CA900092F803905FEA89607FF54CAFD07880060A
:10CAA0007FF548AF92F803905FEA89607FF542AF67
:10CAB000D07880067FF53EAF92F803905FEA8960F8
:10CAC0007FF538AFD07880067FF534AF92F80390C9
:10CAD0005FEA89607FF52EAFBAF1080A7FF426AFCE
:10CAE00082F802A0DBF80820957000BF8BF80C607C
:10CAF00020E7DF0640F171812F6806970699C1F3A0
:10CB00000800B0F5807F3FF6E4AD94F8091CD4F836
:10CB1000047CD4F80C0C19420CBF0126002697F8AF
:10CB20005920012303FA00F111435FFA81F987F8D4
:10CB30005990D4F8047CD4F8100C002E3FF4E6ADE4
:10CB400097F8593006FA00F213435FFA83F8E3E5E9
:10CB5000F90640F15C8129680491049BC3F3080045
:10CB6000B0F5807F3FF683AD94F8190CD4F8141C0F
:10CB70003842D4F81C0C0CBF0126002691F85970DD
:10CB8000012303FA00F038435FFA80F881F85980F6
:10CB9000D4F8142CD4F8207C002E3FF485AD92F804
:10CBA000593006FA07F003435FFA83FC82E5DF069B
:10CBB00040F1208129680291029FC7F30809B9F565
:10CBC000807F3FF622AD94F8F97BD4F8F41BD4F8BB
:10CBD000FC0B1F420CBF0126002691F8597001235F
:10CBE00003FA00F038435FFA80FA81F859A0D4F8CC
:10CBF000F42BD4F8007C002E3FF424AD92F8593089
:10CC000006FA07F003435FFA83FB21E5D4F8343ECC
:10CC1000FFF7D5B9917801F0E70090709A6816791E
:10CC2000F7B28DF80370957845F008019170986817
:10CC30000222C2709A6842F21070D678B10722D4EC
:10CC4000D778BF071FD4D578AF071CD492F803A0BC
:10CC50005FEA8A7617D492F803B05FEA8B7512D434
:10CC600092F803C05FEA8C710DD492F803E05FEA9A
:10CC70008E7708D492F803905FEA897603D4083857
:10CC8000DBD1FFF73DBB917801F0C70090709A6847
:10CC900042F21071D678B60628D5D778BD0625D5CC
:10CCA000D578AD0622D592F803A05FEA8A601DD53B
:10CCB00092F803B05FEA8B6718D592F803C05FEA79
:10CCC0008C6613D592F803E05FEA8E650ED592F874
:10CCD00003905FEA896009D50839DBD191709868C3
:10CCE0008022827000BF01219A681973022613798D
:10CCF000D670FEF7BFBF977807F0E70090709A688C
:10CD00001679F5B28DF8025092F8029049F00801B8
:10CD100091709F680220F8709A6842F21070D6787D
:10CD2000B70722D4D578AE071FD492F803A05FEAE4
:10CD30008A711AD492F803B05FEA8B7715D492F80F
:10CD400003C05FEA8C7610D492F803E05FEA8E7538
:10CD50000BD492F803905FEA897106D4D1788F07DB
:10CD600003D40838DBD1FFF760BB977807F0C70022
:10CD700090709A6842F21071D678B50628D5D578A9
:10CD8000A80625D5D778BD0622D592F803A05FEA7C
:10CD90008A601DD592F803B05FEA8B6718D592F8C8
:10CDA00003C05FEA8C6613D592F803E05FEA8E65F4
:10CDB0000ED592F803905FEA896009D50839DBD176
:10CDC000917098688022827000BF01219A6819735F
:10CDD00002261379D670FEF712BF94F8085C94F817
:10CDE000092C1D420CBF012500251A420CBF01264B
:10CDF000002675E494F8F82B94F8F90B1A420CBF4E
:10CE00000122002218420CBF0126002604E494F8F7
:10CE1000182C94F8199C3A420CBF0122002219EAFE
:10CE2000070F0CBF0126002628E407EE900AB8EE93
:10CE3000E70AB5EEC00AF1EE10FA49DD01EE902ADC
:10CE4000B8EEE12AB5EEC02AF1EE10FA3FF78AA853
:10CE50004AD4F7EE002A9FED461AB4EE621AF1EEBC
:10CE600010FA41D1FFF77EB892F803B01BF0020F21
:10CE70007FF412ADB9F108097FF4EAAC82F80290B0
:10CE80008268957000BF067306E5BAF1080A7FF460
:10CE9000C6AD8BF802A09068857000BF167338E5A8
:10CEA000BBF1080B7FF4A2AC99E553D4DFED306AF7
:10CEB00004EE102AF8EEC44AF5EEC04AF1EE10FA7C
:10CEC00050DD0023C4F8203E4FF0010EFFF71DB8DF
:10CED0003DD4DFED272A07EE102AF8EEC70AF5EE5B
:10CEE000C00AF1EE10FA38DD0021C4F8301E4FF010
:10CEF000010EFFF759B89068C67000BF90681173B3
:10CF000080F8029090688570BCE5906880F803E036
:10CF100000BF906882F80CC080F80280906885702D
:10CF2000B0E511D4DFED122A07EE103AF8EEC70A89
:10CF3000F5EEC00AF1EE10FA3FF7C1AA7FF5B7AAE5
:10CF4000BFEE001AFFF7B5BAFFEE002AECE7FFEEDE
:10CF5000002AC0E7FFEE006AAAE77FF57CAFBFEECC
:10CF6000001A7AE77FF5C9AABFEE005AFFF7C7BAE1
:10CF7000000000002DE9F04F2DED028B0446D44B4C
:10CF8000D44E8BB040F21B120280002158306360F7
:10CF90004C2203900BF0BCF8CF4BA24603F5A07EC9
:10CFA0001F689A689C691D6A986A196BD3F838B033
:10CFB00006EBC70906EBC208D9F804705A683A6054
:10CFC0001F69D8F804C0DA68CCF8002006EBC7095E
:10CFD00006EBC408D9F804C05C69CCF80040D8F866
:10CFE0000470DA693A6006EBC50506EBC0006C68B0
:10CFF0005F6A27604268DD6A156006EBC101586B05
:10D000004C6806EBCB0B2060DA6BDBF80470403326
:10D010009E453A60C4D1DFF8D4B2B04DDBF834009D
:10D02000DBF838300768DBF83010CAF8F05000221F
:10D030003B4302278AF8F4708AF8FC208AF8FD2026
:10D04000CAF80021CAF84421CAF848210360CAF886
:10D05000F8100A70DAF8F800A14F4270DAF8F830E8
:10D06000A04D9A70DAF8F800FF21C170DAF8F830B4
:10D070005A71DAF8F80050218171DAF8F830DA7173
:10D08000DAF8F800817801F07F038370DAF8F800AD
:10D0900096460AF1F001122204915446C270F046FD
:10D0A000F4464FF0FF314FF0010A8F4A0AFA0EF9A9
:10D0B0000020A2E0C3F5742A0AF510738B4202D255
:10D0C0001946F0468446B2F802A009FB0AF3B7FB02
:10D0D000F3FAAA4500F1010000F2A680CAF5742A0D
:10D0E0000AF510738B4202D21946F04684469388A3
:10D0F00009FB03F3B7FBF3F3AB4200F1010A40F283
:10D10000A080A3F57423A3F510738B4205D2D446F7
:10D11000F046002B00F0EC801946D38809FB03F39E
:10D12000B7FBF3F3AB4200F1020A40F29580A3F59E
:10D130007423A3F510738B4205D2D446F046002B1E
:10D1400000F0D6801946138909FB03F3B7FBF3F30C
:10D15000AB4200F1030A40F28A80A3F57423A3F5E1
:10D1600010738B4205D2D446F046002B00F0C080ED
:10D170001946538909FB03F3B7FBF3F3AB4200F104
:10D18000040A7FD9A3F57423A3F510738B4205D24B
:10D19000D446F046002B00F0AB801946938909FB7A
:10D1A00003F3B7FBF3F3AB4200F1050A74D9A3F51F
:10D1B0007423A3F510738B4205D2D446F046002B9E
:10D1C00000F096801946B2F80EA009FB0AF3B7FBEF
:10D1D000F3F3AB4202F10E0200F1060A66D9A3F5A1
:10D1E0007423A3F510738B4204D2D446F046002B6F
:10D1F0007ED019460730402864D0538809FB03FAD3
:10D20000B7FBFAF3AB4202F102027FF653AFA3F58C
:10D21000742AAAF510738B42BFF455AFF0468446CA
:10D22000002B65D019464EE7AAF57423A3F51073B9
:10D230008B42BFF45CAFF0468446002B58D01946B1
:10D2400055E7C3F5742303F510738B42BFF465AF44
:10D25000D4461946F04660E7C3F5742303F510730E
:10D260008B42BFF470AFD4461946F0466BE7C3F566
:10D27000742303F510738B42BFF47BAFD446194679
:10D28000F04676E7C3F5742303F510738B4285D21D
:10D29000D4461946F04681E7C3F5742303F51073AD
:10D2A0008B4290D2D4461946F0468CE7C3F57423DE
:10D2B00003F510738B429DD207304028D44619469F
:10D2C000F0469AD1BEF1020F12D00EF1010EEAE63D
:10D2D000B0C5010034CE010070C40100FCC00100E3
:10D2E000008793033F420F00CACC010084CC0100A9
:10D2F0000CF03F02D4F8F810E94F42EA8810C3B2AC
:10D300004B70D4F8F8506A7942F020006871D4F874
:10D31000F81091F8029049F080038B7094F8F4A013
:10D320000AEB4A050BEBC50C4FF00109DCF80C20A9
:10D330005009810001F1604808F5614ED94902F0B9
:10D340001F03002509FA03F2049BCEF800200820F1
:10D350008B60C4F8F070C4F8505184F85451C4F88C
:10D36000585107F073FC2946824607F0DFFAD4F8DB
:10D37000F870C4F850A1B878DFF858C3CA4BCB4A4C
:10D3800000F0FE01B970D4F8507138798CF80000C3
:10D3900094F8F480D4F8507108EB480E0BEBCE0AE9
:10D3A00097F804C0DAF810000CF1804101F5043858
:10D3B00000F03F0747F0800088F8005088F8000030
:10D3C000D4F8507194F8F4A097F804E0B84F0AEB41
:10D3D0004A0C0BEBCC010EF11008486947F8280005
:10D3E0004FEA6E11880000F1604AD4F850010EF047
:10D3F0001F070AF5614E006809FA07F1CEF8001020
:10D40000878B1FFA87F949F0080CA0F81CC0B0F808
:10D410001C801FFA88FA4AF002018183A14804990E
:10D42000816040F6FF7E04F5B8774FF00C09A14803
:10D43000A4F86AE1294684F86C51C4F86401A4F8A0
:10D440006891384606F018FE9B4AC4F8805404F5EB
:10D45000B273C4F8845438460821136006F0C6FF3E
:10D460003846494606F0B8FD3846022106F08EFCE3
:10D470003846022106F05EFF3846904F06F076FCF3
:10D48000039B8F4AC4F88C54C4F8883410253B465B
:10D4900013211120C4F86421C4F890541222C4F856
:10D4A000A454BB42874DC4F89814C4F8B414C4F80B
:10D4B0009404C4F8AC04C4F89C24C4F8BC24C4F894
:10D4C000A054C4F8A854C4F8B054C4F8B85404F52F
:10D4D000946804F5976A4FF001010CD198F80400A4
:10D4E00008F04EF8C2450BD058F8080F0368BB424D
:10D4F0004FF00101F2D0012140469847C245F3D1D7
:10D50000D4F88834C4F8C4341F1D981D03F10A01EF
:10D5100003F1020803F10E0203F11205C4F8D474FA
:10D52000C4F8DC0403F1160703F11800C4F8EC1486
:10D5300003F11C0103F1080C03F10C0903F1100EB7
:10D5400003F1140AC4F8CC84C4F8FC2403F11A08CB
:10D5500007221E33C4F80C55C4F81C75092503278F
:10D56000C4F82405C4F8341504200F21C4F8E4C419
:10D570000193C4F8F494C4F804E54FF002094FF0A5
:10D580000A0E4FF0060CC4F814A5C4F82C854FF011
:10D590000C0A4FF001080823C4F8C824C4F8D85472
:10D5A0000D220025C4F8E874C4F8F0040E27052005
:10D5B000C4F800150B21C4F8C034C4F8D0C4C4F8B2
:10D5C000E0A440F6FF7CC4F8F884C4F80825C4F849
:10D5D0001095C4F82075C4F8280504F24C57C4F817
:10D5E0003015344AC4F81855C4F838E5019BA4F83E
:10D5F00046C54146C4F83C353846A4F844A584F8ED
:10D600004885C4F84025304B304A06F035FD2A4A9B
:10D61000C4F85C5804F5A8633846C4F8605808217B
:10D62000536006F0E3FE5146384606F0D5FC494605
:10D63000384606F0ABFB4946384606F07BFE3846D6
:10D6400006F094FBDBF80410DBF808300868DBF820
:10D650000020DFF88490C4F8409503430398C4F891
:10D6600064084FF0200C04F1780E1F271848C4F806
:10D670007C0804F17A0AC4F86CC8C4F870E8C4F8ED
:10D680007478C4F8685884F8805884F8885884F806
:10D690008958C4F88C58C4F8D058C4F8D4581DE040
:10D6A00008C10100C0AA0220E4CB0100E8CB0100C0
:10D6B0000002FF1FE8C00100B8A90220050D00000C
:10D6C0002CC1010014C10100E6CB010035CC0100E2
:10D6D000FCC001001A80004040C10100C4F878A8D5
:10D6E0000B60C4F884281570D4F88418DFF85CE265
:10D6F0004D70D4F88438934F9D70D4F88408FF227D
:10D70000C270D4F884184D71D4F8843850209871C0
:10D71000D4F88428CDF80880D571D4F8841891F80D
:10D72000029009F07F038B70D4F8840804F67C0122
:10D7300012220191C270A846AC464FF0FF31029B05
:10D74000814A03FA05F900209AE0CAF5C333A033F1
:10D75000994202D919468446A846B2F802A009FBAC
:10D760000AF3BEFBF3FABA4500F1010000F29F8014
:10D77000CAF5C333A033994202D919468446A84654
:10D78000938809FB03F3BEFBF3F3BB4200F1010AEC
:10D7900040F29980A3F5C333A03B994205D9D44602
:10D7A000A846002B00F0D4801946D38809FB03F368
:10D7B000BEFBF3F3BB4200F1020A40F28E80A3F5F8
:10D7C000C333A03B994205D9D446A846002B00F0AC
:10D7D000BF801946138909FB03F3BEFBF3F3BB4279
:10D7E00000F1030A40F28380A3F5C333A03B9942C2
:10D7F00005D9D446A846002B00F0AA8019465389C3
:10D8000009FB03F3BEFBF3F3BB4200F1040A77D933
:10D81000A3F5C333A03B994205D9D446A846002BB3
:10D8200000F096801946938909FB03F3BEFBF3F3DE
:10D83000BB4200F1050A6CD9A3F5C333A03B994262
:10D8400005D9D446A846002B00F082801946B2F8CC
:10D850000EA009FB0AF3BEFBF3F3BB4202F10E027A
:10D8600000F1060A5ED9A3F5C333A03B994204D95F
:10D87000D446A846002B6BD01946073040285CD010
:10D88000B2F802A009FB0AF3BEFBF3FABA4502F1B3
:10D8900002027FF65AAFAAF5C333A03B99427FF646
:10D8A0005CAFA8468446002B52D0194655E7AAF52E
:10D8B000C333A03B99427FF663AFA8468446002B52
:10D8C00046D019465CE7C3F5C333A03399427FF6CF
:10D8D0006CAFD4461946A84667E7C3F5C333A033F7
:10D8E00099427FF677AFD4461946A84672E7C3F54A
:10D8F000C333A033994282D9D4461946A8467EE75D
:10D90000C3F5C333A03399428DD9D4461946A846EE
:10D9100089E7C3F5C333A033994298D9D446194651
:10D92000A84694E7C3F5C333A0339942A5D907307D
:10D930004028D4461946A846A2D1022D08D0013568
:10D94000FDE600BF9F860100CACC0100008793035B
:10D950000CF03F02D4F88418B34FB44D42EA88105B
:10D96000C3B24B70D4F88428507940F02001517133
:10D97000D4F8842892F8029049F08003937094F8C8
:10D9800080A80AEB4A000BEBC00C4FF00108DCF852
:10D990000C104A09930001F01F0003F1604B08FAD4
:10D9A00000F204F6DC01A248019B02910BF56149EB
:10D9B0004FF0000EC9F8002003600298C4F8DC386C
:10D9C00071464022C4F8E808C4F8E0E8C4F8F0E87A
:10D9D000C4F8E478C4F8EC5804F6F4000AF098FBB4
:10D9E000D4F88428202184F8361992F802A00AF08D
:10D9F000BF039370D4F8E00884F8898858B10268AE
:10DA00008C4953688B4204F6E40241F06780406819
:10DA10000221F5F747FA04F63813002194F8340987
:10DA2000019AC4F8382984F83509C4F84439C4F88F
:10DA30003C19C4F84C194022C4F84079C4F848593C
:10DA400004F5156006930AF063FBD4F884082121DD
:10DA500084F89219827802F0BF038370D4F83C09ED
:10DA6000012184F8891858B10268724953688B42C1
:10DA700004F5146241F0378040680221F5F712FA8C
:10DA800004F69413002194F89009019AC4F894299B
:10DA900084F89109C4F8A039C4F89819C4F8A819F1
:10DAA0004022C4F89C79C4F8A45904F6AC1005933C
:10DAB0000AF02EFBD4F88408222184F8EE1982782B
:10DAC00002F0BF038370D4F89809012184F8891803
:10DAD00058B10268574953688B4204F69C1240F0D3
:10DAE000F88740680221F5F7DDF904F51F6300218E
:10DAF00094F8EC09019AC4F8F02984F8ED09C4F807
:10DB0000FC39C4F8F419C4F8041A4022C4F8F879AE
:10DB1000C4F8005A04F6082007930AF0F9FAD4F87A
:10DB20008408232184F84A1A827802F0BF038370A4
:10DB3000D4F8F409012184F8891858B102683D49E4
:10DB400053688B4204F6F81240F0DC8740680221EB
:10DB5000F5F7A8F9002194F8480A019AC4F84C2A6C
:10DB600004F64C2B84F8490AC4F8501AC4F8601A19
:10DB70004022C4F8547AC4F85C5AC4F858BA04F67F
:10DB800064200AF0C5FAD4F88408242184F8A61A7F
:10DB900090F802C00CF0BF038370D4F8500A012241
:10DBA00084F8892858B1036822495B688B4204F6DF
:10DBB000542240F09D8740680221F5F773F9002157
:10DBC00094F8A40A019AC4F8A82A04F6A82AC4F86A
:10DBD000B07AC4F8B85A84F8A50AC4F8AC1AC4F8E4
:10DBE000BC1A4022C4F8B4AA04F52C600AF090FADA
:10DBF0002527D4F8845884F8027BA97801F0BF0364
:10DC0000AB70D4F8AC0A012284F88928A0B1076867
:10DC1000084D7B68AB4204F52B6240F06E8740688C
:10DC20000221F5F73FF907E054C101003109000076
:10DC3000C0AA0220913300004FF00107029884F837
:10DC4000097B84F8197B84F8297B012700250423AC
:10DC50004FF002094FF0060E4FF0030C079AC4F87C
:10DC6000340BC4F8440BC4F82C7B059884F8397B3A
:10DC700084F8497B84F8597B0727C4F8042BC4F83F
:10DC8000142BC4F8242BC4F8540BC4F8640B84F888
:10DC9000083B84F8183B84F8283B84F8383BC4F8E8
:10DCA0003C3B84F8483B84F8583BC4F80CEBC4F880
:10DCB00040EBC4F85CEBC4F8107BC4F84C7BC4F8B0
:10DCC000607BC4F81CCBC4F8209BC4F8305B94F88C
:10DCD000007B01974FF0010784F8697B84F8797B1A
:10DCE00084F8897B84F8997B0727C4F8A07B4FF0E0
:10DCF000010784F8A97B0127C4F8B07B84F8B97BBD
:10DD000084F8C97B01270521C4F8CC7B069FC4F8A1
:10DD1000501B84F8683BC4F870CB84F8783BC4F897
:10DD200080CB84F8883BC4F88C3BC4F8901B84F803
:10DD3000983BC4F89CEB84F8A83BC4F8AC5B84F82F
:10DD4000B83BC4F8BC3BC4F8C01B84F8C83BC4F85B
:10DD5000747BC4F86C9BC4F87C9BC4F8847BC4F8C7
:10DD6000947BC4F8C47B4FF0010784F8D97BC4F8D6
:10DD7000FC1B0127C4F8101CC4F8201C0299C4F82D
:10DD8000A40BC4F8B42BC4F8D05B84F8D83BC4F817
:10DD9000DC5B84F8E83BC4F8ECCBC4F8003C84F8C6
:10DDA000083CC4F80C5CC4F81C3CC4F8305CC4F8F3
:10DDB000345C84F8385C84F8395CC4F8D41BC4F84B
:10DDC000E41BC4F8E07B84F8E97BC4F8F09B84F89A
:10DDD000F89B84F8F97B84F8097C84F8189C84F813
:10DDE000197C059F84F8A03C019B94F9A51AC4F8FE
:10DDF000F47B63F0300704F6244361F02101C4F89A
:10DE0000A43D04F664434FF014084FF4FA70F24A4C
:10DE10000191C4F8AC3D04F644414FF00103C4F84D
:10DE200004BCC4F814ACC4F82C0CC4F8242CC4F8FA
:10DE30003CBCC4F8A81D84F8403C0499C4F84C0CC0
:10DE4000C4F8505CC4F8545C84F8585C84F8595C9D
:10DE5000C4F8442CC4F86C0CC4F8705CC4F8745C4E
:10DE600084F8785C84F8795CC4F8642CC4F8288C55
:10DE7000C4F8488C84F8609CC4F8688C84F880CC22
:10DE80009DF8043084F8A53A04F68443C4F8B03D04
:10DE90004FF0070384F8E03C04F62453C4F88C0CDC
:10DEA000C4F8905CC4F8945C84F8985C84F8995C3D
:10DEB000C4F8842CC4F8AC0CC4F8B05CC4F85CBCE6
:10DEC000C4F87CBCC4F89CBCC4F8B45C84F8B85CEE
:10DED00084F8B95CC4F8A42C84F8C0ECC4F8CC0C69
:10DEE000C4F8D05CC4F8D45C84F8D85C84F8D95CFD
:10DEF000C4F8C42CC4F8EC0CC4F8F05CC4F8888CEA
:10DF0000C4F8A88CC4F8C88CC4F8E88CC4F8F45CD5
:10DF100001934FF0010384F8203D04F6C44384F8D4
:10DF2000F85C84F8F95CC4F8E42C84F8005DC4F86B
:10DF30000C0DC4F8105DC4F8145D84F8185D84F805
:10DF4000195DC4F8042DC4F8BCBCC4F8DCBCC4F82A
:10DF5000FCACC4F81CAD84F860CDC4F8B83DC4F87E
:10DF60002C0DC4F8305DC4F8345D84F8385D84F855
:10DF7000395DC4F8242DC4F84C0DC4F8505DC4F8C4
:10DF8000545D84F8585DC4F8088DC4F8288D84F871
:10DF9000409DC4F8488D84F8595D84F8017B4FF0AA
:10DFA000070704F6045C019BC4F8442DC4F86C0D0B
:10DFB000C4F8642D84F880EDC4F88C0D04F6E44EAA
:10DFC000C4F83CADC4F85CADC4F87CAD04F6A44024
:10DFD000C4F8842D84F8A07D04F6445204F6D45786
:10DFE000C4F89CAD04F6645B04F6845AC4F8B43DEE
:10DFF000C4F8BCEDC4F8C0CDC4F8705DC4F8745D5D
:10E0000084F8785D84F8795DC4F8905DC4F8945D17
:10E0100084F8985D84F8995DC4F8C40DC4F8C82DDF
:10E0200038466E4AC4F8688DC4F8888DC4F8CCBDF3
:10E03000C4F8D0AD0297F5F7B3F91C276FF0004292
:10E040001B2084F8E25D84F8F25D654DC4F8F42D80
:10E05000C4F8F85DC4F8005E4946C4F8FC0DC4F885
:10E06000047EC4F8E48D07F08BFA494694F8040E58
:10E0700007F086FAD6F8D8104FF0010001F50073CA
:10E0800084F8F00DC4F8E83DD6F8E02084F8F10DEE
:10E0900002F500774846C4F8EC7D07F0CFFAD4F8D3
:10E0A000E85D94F8F01D2878084205D094F8F29DB8
:10E0B00049F0010884F8F28DD4F8EC2D94F8F1EDD4
:10E0C000137813EA0E0F05D094F8F27D47F002059D
:10E0D00084F8F25D04F6E85B59461B20FDF73AF838
:10E0E00059461C20FDF736F800233E4A3C493C4D7A
:10E0F000C4F8083E18206FF00047C4F80C3EC4F87E
:10E10000103EC4F8183EC4F81C3EC4F8203EC4F8C3
:10E11000283EC4F82C3EC4F8303E84F8463E1A230C
:10E12000C4F8583EC4F8142EC4F8242EC4F8342E73
:10E13000C4F84C1EC4F8545EC4F8487EC4F8500EAF
:10E14000022107F01DFA022194F8580E07F018FA80
:10E15000D6F8C0004FF0010C00F50072C4F83C2E58
:10E1600084F844CED6F8D06084F845CE06F5007128
:10E17000C4F8401E022007F061FAD4F83C7E94F8FF
:10E18000445E3B782B4205D094F8460E40F00102E5
:10E1900084F8462ED4F8406E94F8451E37780F4226
:10E1A00005D094F8465E45F0020A84F846AE04F6BF
:10E1B0003C6949461820FCF7CDFF49461A20FCF778
:10E1C000C9FF094D064BC4F85C3E1920C4F8600E27
:10E1D000022107F0D5F909E060C10100F8FB022037
:10E1E00014C1010001000080D0C101000FCD04F670
:10E1F0006467DFF8BC84C7F8008004F6686EAEE898
:10E200000F000FCDAEE80F000FCDAEE80F0095E880
:10E21000070004F6A4668EE8070004F668650C2083
:10E22000019707F0A1F8B54237D0019F287897ED04
:10E23000000AAB4607F0A8F85BF8040B0021C0B257
:10E2400006F0B8FE287997ED000A07F09DF82879C6
:10E25000002106F0AFFE97ED000A9BF8040007F0DE
:10E2600093F800219BF8040006F0A4FE287B97EDAC
:10E27000000A07F089F8287B002106F09BFE287C25
:10E2800097ED000A07F080F8143515F8040C00210A
:10E2900006F090FEAE42C9D1019741F6DC6201233F
:10E2A00004F5F751A354029F039800228846C4F84E
:10E2B000A42E84F8AC2EC4F8B02E84F8B42E84F8C2
:10E2C000B52E04F5274C8F6004F52F4A04F5374529
:10E2D000019F0A7141F6F86904F53F4BC8F80C70CC
:10E2E0004FF0FF3E0861E9484E61086044F809605C
:10E2F000C1F824E004F55F498CF810308CF8183828
:10E300008AF8203804F54F4C85F8283804F5474A38
:10E310008BF8303804F5574504F5674B8AF83838E0
:10E3200004F57F4E8CF8403804F56F4085F8483886
:10E3300004F5774A89F8503804F5873C8BF858384B
:10E3400004F5833904F58B3504F58F3B80F860388C
:10E3500018318AF868388EF8703804F5943A89F8DC
:10E3600078398CF8803985F888398BF89039C84B22
:10E3700001F5843C04F593300AF11C0E1E600AF18D
:10E38000B409143104F50A36C0F81422CB46C0F89B
:10E39000182206F5DA75CEF88020CEF88420CCF865
:10E3A000AC21CCF8B0110BF58051584641F2100267
:10E3B00001F1100B002109F0ABFEAB45F3D1A945EB
:10E3C000019700F0B180C9EB0502A2F5805709F56D
:10E3D0008050A7F1100300F1100A41F210024846E4
:10E3E0000021C3F3021709F093FE554500F09C800D
:10E3F000002F53D0012F45D0022F39D0032F2DD01D
:10E40000042F21D0052F15D0062F09D0504641F2F8
:10E410001002002109F07CFE0AF5805A0AF1100A68
:10E42000504641F21002002109F072FE0AF5805CAC
:10E430000CF1100A504641F21002002109F068FE6A
:10E440000AF5805909F1100A5046002141F21002E4
:10E4500009F05EFE0AF5805101F1100A504641F2C2
:10E460001002002109F054FE0AF5805B0BF1100A3E
:10E47000504641F21002002109F04AFE0AF580528E
:10E4800002F1100A0AF5805E504641F210020EF1C8
:10E49000100A002109F03CFE554545D0019F41F28C
:10E4A00010020021504609F033FE0AF5805041F277
:10E4B00010020021103009F02BFE0AF5005041F245
:10E4C00010020021203009F023FE0AF5405041F2ED
:10E4D00010020021303009F01BFE0AF5804041F2A5
:10E4E00010020021403009F013FE0AF5A04041F26D
:10E4F00010020021503009F00BFE0AF5C04041F235
:10E5000010020021603009F003FE0AF5E0400AF530
:10E51000004303F1800A703041F21002002109F03B
:10E52000F7FD5545BBD101974FF4FA75C6F8B851C0
:10E5300008F502300025574F5749C6F8BC113C2258
:10E5400000F5367CC6F8C05186F8C451294600F55E
:10E550003A70C7F800C009F0DBFD06F5017206F558
:10E56000137BC6F8D05386F80452C6F8D4539FEDF7
:10E570004B8AC2F870B04FF0FF3706F5157E06F5EE
:10E58000177A4FF0020BD7645560D560D5631564D8
:10E590005564956406F28D20C6F878E2C6F87CA230
:10E5A000C6F85CB24FF0040A0123F7EE008A06F5C4
:10E5B000197C06F51B7B4FF0030EC6F86CA2C6F85B
:10E5C0005872C6F86072C6F86872C6F87072C6F8FB
:10E5D0005432C6F880C2C6F864E2C6F884B2039327
:10E5E000176182F8883006F57677C2F88450556155
:10E5F000157682ED2A8A82ED2C8A82ED078AC2ED99
:10E600002D8AC6F88D52052685604560C0F80B50EE
:10E610002946166282F8A75004F50B3682F8B850E6
:10E6200082F8B950C2F8C850C2F8C45038464C22DB
:10E6300009F06EFD039987F84D1087F84E504FF0A2
:10E640007C50C6F850A0C6F87CA0154ADFF864904C
:10E65000144BDFF864C0C6F8883006F1DC0A06F116
:10E66000940B7064B06330677066C6F88C500E4FC0
:10E670000E481168C6F830C0C6F834C0C6F85CC091
:10E68000C6F860C0C6F8807018E000BF78C101000D
:10E69000D4AA0220B0A80220553D010000000000CD
:10E6A0003C800440B50AFF1F6CC10100A0C10100FD
:10E6B000BFE164464CCD01000AD7233C86ED0A8AAF
:10E6C000C6ED0B8A86ED0F8A86ED108AC6ED128A9A
:10E6D000F56486ED158AC6ED168A86ED1A8A86EDF2
:10E6E0001B8AC6ED1D8AB567C6F884808BF8045076
:10E6F000C6F894008AF80450D9F80430CE481F4672
:10E700003943D9F8003011601A68C6F8DC3042F499
:10E71000804706F1BA0E06F19A012022CAF80810C5
:10E72000CAF80CE0CAF81020CAF81450CAF81850F9
:10E73000CAF81C50C0F800A01F601968BF4841F01B
:10E7400001071F601968826841F4806018601F68C3
:10E7500042F0605247F400614FF47C101960DA60B7
:10E7600018601F6827F001021A601968B44F21F47D
:10E7700080401860082006F069FA2946039006F0E8
:10E78000D5F8039ACAF8182011793970DAF8180008
:10E79000D6F8DC3007683833B3F1804F3B60BD807A
:10E7A000FD7180F09081016801228A600168DAF8C9
:10E7B0001830A4481F680025CD60FD7196F8E0C0B0
:10E7C000DAF818306C2202FB0C9E1979DEF80C7016
:10E7D00001F1804C0CF5043307F03F0242F0800158
:10E7E0001D701970DAF818109AF804700A7950F848
:10E7F00027E0954F02F1100053119B0047F820E0ED
:10E8000003F1604C0CF5614E02F01F020120096813
:10E8100000FA02F3CEF800308F8BBAB242F0020059
:10E820008883B1F81CC0864F1FFA8CFE4EF0080397
:10E830008B83082006F00AFA2946039006F076F842
:10E84000039ACAF81C2010793870DAF81C70D6F8D0
:10E85000DC30396834338D71B3F1804F0B618D82B8
:10E860003B6801D39D6815B901229A603B68DAF8CC
:10E870001C7076483A68764900259D61957196F836
:10E88000E070DAF81C306C2202FB079993F804C0A0
:10E89000D9F810700CF1804E0EF5043307F03F02EA
:10E8A00042F080071D701F70DAF81C200492D2F825
:10E8B00000C0BCF81C701FFA87FE4EF0080206F17B
:10E8C000FC03644FACF81C2003934FF00A0C019B2F
:10E8D000C6F8FC70C6F80401029FC6F800C1022009
:10E8E000C6F808B1C6F80C11C6F810512946CBF885
:10E8F00080701E22C6F81831C6F8245186F81C0113
:10E9000086F81D0186F81E01C6F82051C6F8275169
:10E9100086F81F0186F8200106F5967009F0F8FBCD
:10E9200029463C2206F5A67009F0F2FB29463C2256
:10E9300006F5C47009F0ECFBD6F8DC208BF83051FA
:10E940001168DFF81CB1DFF8F8E0434841F001033B
:10E950001360116841F480631360116841F400632F
:10E960001360C2F82CB0116821F001031360049AFF
:10E9700011798EF80010DAF818301A798EF8002024
:10E98000DAF81820DAF810301168DAF808C08D715A
:10E99000D2F800E0C1F810C04FF0010BA1F814B09C
:10E9A000CEF808B0D2F800C099B2ACF81E101268C8
:10E9B0005B42CCF81830D182DAF818100A68DAF81D
:10E9C0001CE09561DEF80020DAF81030DAF80C105F
:10E9D000D5711160DEF80010A2F804B0C1F808B0DB
:10E9E000DEF800101FFA83FCA1F81EC0DEF800E07C
:10E9F0005A42CA60AEF816C0DAF81C301968CD6009
:10EA00001A790270DAF8183019790170D6F8DC300A
:10EA100003981A6B406842F4403119631A6B06F58B
:10EA2000827942F0407119634A460321F4F73AFAB9
:10EA30000A4BC6F8D07115E0E4AA022024CE0100EA
:10EA40001A8000405C5CFF1F0002FF1F94C10100A0
:10EA5000F906FF1F14C101001B80004000AB02201B
:10EA600000000ADA1A680992099B019FC6F8E03192
:10EA70002748284BC6F8C801272104F1080AC6F820
:10EA8000E81186F8CC5106F50070A6F8DAB1C6F8A0
:10EA9000D471A6F8D85186F8DC51802286F8F0515E
:10EAA000C6F8F451C6F8E431C6F8EC811A49C6F844
:10EAB000FC51C6F8F8A105F0DFFF20460BB0BDEC15
:10EAC000028BBDE8F08F01688D68002D3FF46CAEBD
:10EAD0006DE6114602229847FFF707B81146022259
:10EAE0009847FEF798BF114602229847FEF7C8BF25
:10EAF000114602229847FFF762B811460222984752
:10EB0000FFF79AB8114602229847FFF723B800BFD3
:10EB1000BCC1010014C101000CC201001E4B2DE953
:10EB2000F041002493F8C074C3F88C441E461D467F
:10EB3000D5F8A00447FA04F1826801F0010105F557
:10EB4000946001349047042C05F10805F0D1134876
:10EB5000134C05F093FC4221104805F0A9FC00235A
:10EB6000C6F868380F4805F089FCD6F868780D4873
:10EB700006EBC70898F86C1805F09AFCD4F8EC017D
:10EB80000668F568A847D4F8EC0101680122027113
:10EB90000B68BDE8F04118472C7A00209C7B0020D0
:10EBA0002CA60220787F002008B50248FCF7EAFF77
:10EBB00008BD00BF2C7A00202DE9F04F203A8DB01F
:10EBC000D3B2672B099000F26882B24850F8230054
:10EBD00090F800E0B04EB14CB368B26AD6F820B0FD
:10EBE0000593099BF569776A089026680BEB02008C
:10EBF00000245A1C0233069007942F4401F10208A6
:10EC000001F1010C0A920B9310461C46099A0297D7
:10EC10000023019604914EFA03F111F0010F27D061
:10EC2000019E954206EB002706EB0229039706EBAF
:10EC3000042A3CDDA54240F3D280854218DC0299CB
:10EC4000814215DD049EB34503DC0699B14200F311
:10EC50009682E34503DC069E664500F36982D8454B
:10EC600006DB069EB04503DA039F059947F8281096
:10EC70000133062B02F1030200F1030004F1030447
:10EC8000C9D107980499029F019E01300828079076
:10EC900008F1030801F103010CF1030C00F0E0811D
:10ECA000089C0A9814F801EF08940B9CAEE70299AF
:10ECB0008C424EDBAC4280F2F380854200F3A680AA
:10ECC000914240F3DE81049FBB45BA4626DC06999B
:10ECD000B94223DD029E059F49F82A70864227DD4E
:10ECE000039E049F059946F82710029991421FDC64
:10ECF0000299814240F3C181E34540F36B82029E59
:10ED00009642ACDDD845B3DB069FB845B0DA029E2B
:10ED1000059949F828108642A6DCA9E7029F874298
:10ED200006DD049EB34540F3B38102999142DFDDD5
:10ED3000E345DDDC069E6645DADD029E059949F86D
:10ED40002C10864240F32B820399059F41F82C70CA
:10ED5000D5E7AC4276DA854258DC914240F38A81AD
:10ED6000049FBB45BA461FDC0699B9421CDD029ED2
:10ED7000059F49F82A70864220DD039E049F05996D
:10ED800046F827100299914218DC0299814240F31B
:10ED90007481E34540F30F82029E96427FF75FAF96
:10EDA000D845FFF665AFAFE7029F874206DD049EB8
:10EDB000B34540F3058202999142E6DDE345E4DC88
:10EDC000069E6645E1DD029E059949F82C108642B3
:10EDD00040F3DE810399059F41F82C70DCE7029E29
:10EDE000A64200F3AC8085423FF742AF86427FF7F0
:10EDF0003FAF049FBB453FF72CAF0699B9427FF761
:10EE000028AF039E059946F8271022E791427FF725
:10EE10002FAF049FBB45BA4603DC0699B94200F305
:10EE20004481E34503DC069E664500F33A81D845FC
:10EE3000FFF61EAF069FB845BFF61AAF059949F811
:10EE4000281015E7814200F3B480914240F3D3804B
:10EE5000049FBB4540F33781E3450BDC069F6745C4
:10EE600008DD059E49F82C60029F05994AF82C1090
:10EE7000974273DDD845FFF6FBAE069EB045BFF660
:10EE8000F7AE059949F82810D146059949F8281098
:10EE9000EEE600BF8CC20100B8790020ACA80220C9
:10EEA000A842B3DB914240F3DE80049FBB45BA46E3
:10EEB0002ADC0699B94227DD029E059F49F82A708F
:10EEC000B0422BDA039E049F059946F82710029959
:10EED000914223DC0299884280F2C880E34540F3E6
:10EEE0007481029E96427FF7BAAED845FFF6C0AE57
:10EEF000069FB845BFF6BCAE029E059949F828109A
:10EF0000B042FFF6B1AEB3E6029FB84206DA049E05
:10EF1000B34540F34B8102999142DBDDE345D9DCF7
:10EF2000069E6645D6DD029E059949F82C10B04232
:10EF300080F22A810399059F41F82C70D1E7854220
:10EF400015DD049EB34503DC069FB74200F30F8135
:10EF5000E34503DC069E664500F30D81D845FFF6C8
:10EF600087AE069EB045BFF683AED1468DE786429A
:10EF700055DD049FBB4540F3B680E34537DC069E74
:10EF8000664534DD0399059F41F82C700299059F71
:10EF90004AF82C708142E1DDD845FFF669AE069E45
:10EFA000B045BFF665AE0399059F41F82870D1467C
:10EFB0006BE7914203DD049EB34540F3AF80854289
:10EFC00045DC049EB34540F3C480029E964202DDB8
:10EFD000E34540F39980854233DCE34540F3AD805F
:10EFE0000299914201DDD84563DA8542B6DCD84505
:10EFF000FFF63EAED3E7049EB34509DC069FB74259
:10F0000006DD059F4AF82670029E96423FF724AF20
:10F01000E345A3DC069961453FF726AF9EE7049FD1
:10F02000BB4508DC0699B94205DD059E4AF8276014
:10F03000029F8742A1DCE34590DC06996145A5DC8F
:10F040008CE7E345CCDC069F67457EDCC8E7049F80
:10F05000BB45BADC069F049EB74200F38480B4E748
:10F060000DB0BDE8F08F8842FFF651AF91427FF7B7
:10F07000FFAD3AE781423FF79AAE91427FF7F8AD94
:10F0800040E681423FF74DAE91427FF7F1AD39E660
:10F090000699B1427FF749AE22E651484FF0000E83
:10F0A00098E5059949F82C10C1E6059F49F82A70A2
:10F0B000B7E6069EB04598DA059F49F82870854264
:10F0C0007FF771AF4DE70699B9427FF7C5AE3E466F
:10F0D000059949F82710059F4AF82670029E964226
:10F0E0003FF7BAAE94E70699B9427FF746AF039E61
:10F0F0000599B146059E49F827104AF82760029FF6
:10F1000087423FF73AAF96E7069F67457FF763AFC1
:10F11000059E49F82C60854213DD94E70699B142BB
:10F120007FF74DAF059949F82610854215DD91E727
:10F13000039F059947F82C1091E5069961457FF7E3
:10F140004FAF039E059946F82C10059F4AF82C7086
:10F1500046E7069FB7427FF738AF039E049F0599A5
:10F1600046F827103E4605994AF826102DE7059FD8
:10F170004AF82670ECE6059F4AF82C70EEE6BA468F
:10F1800005994AF8261064E596423FF7AEAE6FE562
:10F1900096423FF7B7AD86423FF761AD68E59642CC
:10F1A0003FF7B0AD86427FF763AD58E50699B142AF
:10F1B0007FF7B1AE86E6069F67457FF7EDAD09E6BE
:10F1C0000699B1427FF7F7ADD7E5069F67457FF710
:10F1D00088AEAFE6069F67457FF791ADB4E500BF07
:10F1E000ACC801002DE9F04F203AD3B2672B85B0AF
:10F1F00000F28180434C54F823201778424BDFF80B
:10F2000010E19C6ADE695D6AD3F820809B680293F6
:10F210009246DEF800300393421C08EB040B06EB29
:10F22000050E01F1010C4FF000090192144602464F
:10F23000002300903CE0724509DA414507DB59455F
:10F2400005DA039D029805EB022545F82100B4423A
:10F2500054DBA64549DD414507DB594505DA039DE9
:10F26000029805EB042545F8210096420FDC724513
:10F270000BDAE04507DCE34505DD039D029805EB6D
:10F28000022545F82C00A6420BDCA64509DDE04529
:10F2900007DCE34505DD039D029805EB042545F8F1
:10F2A0002C000133062B04F1020402F102020ED0FD
:10F2B00047FA03F0C007F4D59642BCDDA642C8DD8C
:10F2C0000133062B04F1020402F10202F0D109F12C
:10F2D0000209B9F1100F00980CF1020C01F10201C2
:10F2E00006D01AF8017F019CA1E79642BFDDD8E75E
:10F2F00005B0BDE8F08F054A00277FE77245B8DB0F
:10F30000CFE700BF8CC20100B8790020ACC8010073
:10F31000ACA80220203AD2B22DE9F04F672A96BF5E
:10F320008A4B8B4A53F822208A4B8B4F1B68FC690F
:10F330007D6A3E6AD7F828B0BF688BB0013A019267
:10F3400000F1010903EB002200F10208049203EB33
:10F35000092200F1030C059203EB0822039700F148
:10F36000040E471D069203EB0C22B344079203EBF5
:10F370000E2203EB072308922544019A099301F119
:10F38000080ACDF808B001905378D80702F10102BD
:10F3900007D50198A04204DBA84202DA8E4240F36E
:10F3A000CB80980706D54C4504DC4D4502DD8E42E6
:10F3B00040F3B880580706D5444504DC454502DDD6
:10F3C0008E4240F3A580180706D5644504DC6545E8
:10F3D00002DD8E4240F39280D80605D5744503DCE9
:10F3E000754501DD8E427FDD9B0605D5BC4203DC01
:10F3F000BD4201DD8E426FDD5378D80701F1010176
:10F4000002F1010206D50198A04203DBA84201DA0D
:10F410008E4258DD980705D54C4503DC4D4501DD8E
:10F420008E4247DD580705D5444503DC454501DDDF
:10F430008E4236DD180705D5644503DC654501DDE0
:10F440008E4225DDD80605D5744503DC754501DD02
:10F450008E4214DD9B060CD5BC420ADCBD4208DDA1
:10F460008E4206DC029B8B4203DD0998039B40F829
:10F47000213001318A4587D10BB0BDE8F08F029869
:10F480008842E7DD0898834603984BF82100E1E7BE
:10F4900002988842D6DD0798834603984BF82100EE
:10F4A000D0E702988842C5DD0698834603984BF85A
:10F4B0002100BFE702988842B4DD0598834603988F
:10F4C0004BF82100AEE702988842A3DD04988346FA
:10F4D00003984BF821009DE7029B8B428CDD099835
:10F4E000039B40F8213087E7029888427FF77CAF82
:10F4F0000898834603984BF8210075E702988842E4
:10F500007FF76AAF0798834603984BF8210063E7BB
:10F51000029888427FF757AF0698834603984BF8C6
:10F52000210050E7029888427FF744AF0598834650
:10F5300003984BF821003DE7029888427FF731AFEE
:10F540000498834603984BF821002AE78CC20100F7
:10F55000ACC80100ACA80220B87900202DE9F04F1A
:10F560009E4FD7F83080D7F800A07C68B8F1000F24
:10F570008DB0054640F3D980B8F1030F55DC28461D
:10F5800008F03EFE2B78002B58D000284FF00006E4
:10F59000B8BF6FF00040B446691E4FF0010E11F87D
:10F5A000012F32B990B911F8012F4FF0FF30002A26
:10F5B000F8D00A2A03D01F2AF1D90636EFE7B4455E
:10F5C000B8BFB4460EF1010E0026E8E7F96A01F172
:10F5D000080966450EFB09FBD7F80C90B8BF6646D4
:10F5E00008FB06F6B9F1010F039608FB0BF02DD0CE
:10F5F000B9F1020F04BF039EC6EB0A0A3E69012E51
:10F600002CD0022E08BF241AFA697E6A0492961939
:10F61000B2451146DFF8C4E104DA039A0AEB020CA2
:10F62000614520DB0DB0BDE8F08F032328463B6326
:10F63000984608F0E5FD2B78002BA6D1D7F80C9062
:10F640000393B9F1010F4FEAC800D1D1039A3E6983
:10F6500002EBD271012EAAEB610AD2D100EBD07B72
:10F66000A4EB6B04D0E7DEF82020DEF82810069229
:10F6700011448C42D6DA20448242D3DA002BD1D016
:10F68000DEF82C209EF814000790083208FB02F2E6
:10F690000592A2EBC8001A464B1E0A93059BCDF8B3
:10F6A00024A0013E1C44C11A0B960891CDF8149079
:10F6B000A2469B460A2ACBEB0A012E4600F08C801C
:10F6C0001346002001E00A2B6FD01F2B16F8013FD4
:10F6D00088BF0130002BF6D100EB400044000598B4
:10F6E000012808FB04F36AD0022870D0099C07980F
:10F6F00058BB0899B8F1020F01EB0A0919D0B8F10B
:10F70000030F46D142B909E020464946FFF754FAB3
:10F7100015F8012F12340AB10A2AF5D13278DA44E9
:10F72000002A3FF47FAF3546C4E7012038638046A6
:10F7300025E7002AF2D00A2AF0D020464946FFF7F2
:10F7400051FD0C3415F8012FF3E7B86900902344FC
:10F750000B985A1E8242A8BF024606988142B8BF43
:10F7600001460A980AF1FF338342A8BF0346049872
:10F77000A042B8BF2046F3F7C9FA089AB8F1020FC1
:10F7800002EB0A092A78D4D0B8F1030FBAD0002AC4
:10F79000C4D00A2AC2D020464946FFF7BBFD15F85F
:10F7A000012F0634002AF4D1B8E700EB40046300CF
:10F7B00008FB03F30598012806F1010694D1039C88
:10F7C000E01A099C00EBD07904EB69048FE7039CF5
:10F7D0000998E41A04448AE70023EBE7B87900208B
:10F7E0002DE9804887B09F4A02919F4CDFF89882AC
:10F7F0009E4E9F4D9F4FA049DFF890C2DFF890E2E8
:10F80000DFF890A281469D48202388F800308CF8CC
:10F8100000308EF800301370237033702B703B7003
:10F820000B70974F9371A371B3710124AB71037087
:10F830008B71137309F6D4520192A046D9F8D46D96
:10F8400096F8646006B1FEE731464FF40042DAF8FC
:10F85000000008F05DFCDAF800503146482205F55A
:10F86000577008F055FC314605F25C40482208F01C
:10F870004FFC314605F25C50482208F049FC05F582
:10F88000FC435C3305F25C66CDF80C90A9461D463E
:10F8900048220021304606F5807B08F039FC4822DA
:10F8A0000021584608F034FC06F50070482200217B
:10F8B00008F02EFC4822002106F5407008F028FCD4
:10F8C0004822002106F5806008F022FC4822002131
:10F8D00006F5A06008F01CFC4822002106F5C06077
:10F8E00008F016FC06F5E0604822002106F50066E7
:10F8F00008F00EFCB542CBD14846DDF80C9000F57F
:10F90000157C00F52971CCF80440CCF80840CCF8FF
:10F910000C40CCF81040CCF81440CCF81840CCF88F
:10F920001C40CCF82040CCF824404CF8284F6145CE
:10F93000E9D1C0F8584200F5FA45C0F85843C0F87C
:10F94000584400F5A06EC0F85845C0F85846CEF8A7
:10F950005847CEF85848CEF85849CEF85842CEF815
:10F960005843CEF85844CEF85845CEF858460EF5D0
:10F97000006EAE45EBD100F5FC4300F5FD4254337B
:10F9800024325C609C60DC601C615C619C61DC61B9
:10F990001C625C6243F8284F9A42F2D12E1A00F59D
:10F9A000807BA6F580715D45C0F8A442C1F30220BA
:10F9B0003ED048B3012821D002281BD0032815D0FF
:10F9C00004280FD0052809D006281CBFCBF8A44274
:10F9D0000BF5807B0BF5807BCBF8A441CBF8A442E0
:10F9E0000BF5807BCBF8A4420BF5807BCBF8A442CF
:10F9F0000BF5807BCBF8A4420BF5807BCBF8A442BF
:10FA00000BF5807B5D4513D0CBF8A447CBF8A44819
:10FA1000CBF8A449CBF8A442CBF8A443CBF8A44438
:10FA2000CBF8A445CBF8A4460BF5006B5D45EBD1B4
:10FA3000144D2B680593059AC2F30806B6F5807F2E
:10FA40000CD93F2220230298C7F80C80C7F81080F9
:10FA5000C7F8308087E80C00FFF780FD0198F9F7C0
:10FA6000A3F8EBE603E400E004E400E005E400E0D2
:10FA700006E400E007E400E008E400E00DE400E054
:10FA8000B879002000AB022000E400E001E400E0CF
:10FA900002E400E0ACA802200FB410B582B004ABC1
:10FAA000054C53F8042B01934021204608F050FCEC
:10FAB00021460248FFF794FEEC7900202C7A0020C2
:10FAC0002DE9F041D0F8C080B8F1000F00F0878038
:10FAD000D0F810E0BEF1000F7EDB0EEB8E0308EBDA
:10FAE000830600F16004D6F84C21D6F85051D6F8C0
:10FAF0005411D6F85C31D6F85871C264C3664565B6
:10FB0000C165476600F168030122012A60D05E6882
:10FB1000996877684D68AF4258DD022A9E60596047
:10FB200056D0D3F800C0DCF80460B5424EDAD71ED8
:10FB3000002F83E8021049DD66687768BD4245DA28
:10FB4000052A1E60616043D123685A68954201DA34
:10FB500043672160D0F8BC40224904F5004340339C
:10FB60001F685E689D68C0F8A050C0F89870C0F823
:10FB70009C609A891C4F93F80EC080F8A6C00023A1
:10FB800008EB8E08A0F8A420C0F89130C0F88930A6
:10FB9000C0F88D30C0F89430D8F80C30C36348F208
:10FBA000500548F2540681FB031887FB037CD917E4
:10FBB0006759A4594460C1EBE802C1EBEC3302641D
:10FBC000436480F888708460BDE8F081052AC1D064
:10FBD00001320434043398E70448FFF75DFF04481A
:10FBE000FFF75AFF6766666673B2E745E0C5010036
:10FBF000D0C501002DE9F04791F82A3088B023B92B
:10FC000090F82A40002C40F0438491F82B6026B9EC
:10FC100090F82B70002F40F0248491F82D5025B9D6
:10FC200090F82D40002C40F0F48391F8283053BB1D
:10FC300090F828703FB392F8894002F1890E02F1E2
:10FC4000970334B100F0AFBD1EF8017F002F40F0E4
:10FC5000AA859E45F8D14FF0080ED2F8CC31D2F8E3
:10FC6000D041013303F01F03A3420CD0D2F8CC7172
:10FC700002F1CC0A0AEBC70C00240AF837E0CCF8F2
:10FC80000440C2F8CC3191F8273043B9D76B002F2C
:10FC900000F0A88390F82770002F40F0AF8391F810
:10FCA000253093B990F825707FB192F8894002F120
:10FCB000890C02F1970334B100F054BD1CF8017FA8
:10FCC000002F40F04F856345F8D191F82430DBB91F
:10FCD00090F82440C4B192F88970002F40F0078456
:10FCE00092F88A30002B40F0028492F88B40002C6E
:10FCF00040F0FD8392F88C70002F40F0F88392F86A
:10FD00008D30002B40F0F38391F8264024B990F811
:10FD10002630002B40F0478391F8294024B990F811
:10FD20002930002B40F0278391F8334004B390F83A
:10FD30003330EBB95468002C40F0C183D2F8CC3199
:10FD4000D2F8D041013303F01F03A34200F0F08248
:10FD5000D2F8CC71D2F83CA002F1CC0909EBC70E65
:10FD6000022409F83740CEF804A0C2F8CC31DFE213
:10FD700091F82C70002F00F08582002D40F06682F3
:10FD80000D6C066CAF1B18D087EAE778A8EBE77418
:10FD9000642C00F31086322CC8BFBF00D368CF4D4F
:10FDA000146CA5FB036307EB1316A642B8BF26EA43
:10FDB000E67404EB8407BD00D56091F82E3003B3E0
:10FDC00090F82E40ECB992F8008008F1FF37012F2F
:10FDD00017D9D2F8CC51D2F8D061013505F01F0304
:10FDE000B3420ED0D2F8CC51D76802F1CC0C0CEB58
:10FDF000C50A4FF0020E0CF835E0CAF80470C2F8DC
:10FE0000CC314C6C466C136AA51B2B440E2B00F3B3
:10FE10005483002BB8BF0F33136225B1B04F3C6839
:10FE20000494049E566291F83650002D00F06E83C3
:10FE300090F83650002D40F06983052B59DC02EB19
:10FE4000C30E5768DEF84C40D2F8C060BC429446FE
:10FE500000F0DE85002E00F06E861469002CC0F2E2
:10FE6000678604EB84094B4406EB830802F1600AC1
:10FE7000C8F84C7102F16803CEF84C700124C2F846
:10FE80008450012C00F013865F689D687E68D5F869
:10FE900004E0764540F30886022C9F605D6000F028
:10FEA0000686D3F80080D8F80470BE4580F2FC8541
:10FEB000E61E002E83E8200140F3F685DAF8047090
:10FEC0007E68B64580F2F085052C1F60CAF80450A4
:10FED00040F0ED85DAF8004063689E4503DACCF81F
:10FEE0007440CAF800507E4D2F680797079ECCF8E3
:10FEF000C86092F800C00CF1FF35012D40F2C780B8
:10FF00000E8840F25557BE4221D90388BB421ED805
:10FF100092F8A740002C00F0128592F88970B7B1D2
:10FF2000D2F8CC51D2F8D041013505F01F03A342DD
:10FF30000DD0D2F8CC5102F1CC0A0AEBC50C002648
:10FF400002270AF83560CCF80470C2F8CC31B1F859
:10FF5000029040F25558C14521D9448844451ED8E5
:10FF600092F8A730002B00F0CC8492F88A70B7B1D9
:10FF7000D2F8CC51D2F8D041013505F01F039C4294
:10FF80000DD0D2F8CC5102F1CC0909EBC5080026FE
:10FF9000022709F83560C8F80470C2F8CC31B1F80E
:10FFA00004A040F2555CE24521D9848864451ED8FE
:10FFB00092F8A730002B00F0868492F88B70B7B1CE
:10FFC000D2F8CC51D2F8D041013505F01F039C4244
:10FFD0000DD0D2F8CC5102F1CC0A0AEBC50C0026A8
:10FFE00002270AF83560CCF80470C2F8CC31B1F8B9
:10FFF000069040F25558C14521D9C48844451ED8C1
:020000021000EC
:1000000092F8A730002B00F0408492F88C70B7B1C2
:10001000D2F8CC51D2F8D041013505F01F039C42F3
:100020000DD0D2F8CC5102F1CC0909EBC50800265D
:10003000022709F83560C8F80470C2F8CC31B1F86D
:1000400008A040F2555CE24521D9048964451ED8D8
:1000500092F8A730002B00F0908492F88D70B7B121
:10006000D2F8CC51D2F8D041013505F01F03A3429C
:100070000DD0D2F8CC5102F1CC0A0AEBC50C002607
:1000800002270AF83560CCF80470C2F8CC310C8C29
:10009000D0ED1A6A90ED1B5AD0ED197A90ED177ACF
:1000A00091F8489082F8B99006EE104AB8EE460AE8
:1000B00077EEC75A70EE660AE5EE206AF4EEE56A5E
:1000C000F1EE10FAC0ED1A6A40F1528276EE877AAC
:1000D000836FC0ED197A436718E000BFCDCCCCCC5C
:1000E00000AB022001088039A470FDBFCDC7BCBFA2
:1000F000332EA3BF76E807BEADC8893DC74D9C3FF0
:1001000061E7B53FA470FD3F86120F3F002B40F31F
:10011000618390ED183AD0ED161A73EE033AB6EEFD
:10012000004AF7EE004A21EE846AF4EE643AF1EEFA
:1001300010FA76EE476AC8BFF0EE643AA6EEA37AEC
:100140005D1E456780ED177A90ED145A90ED1C7A8C
:1001500090ED152A35EE210AF0EE450A77EEC05AE9
:10016000E5EE870AF4EEC20AF1EE10FA08D5B4EE15
:10017000E05AF1EE10FA54BFB0EE452AB0EE602A14
:10018000FCEEC27A5FED291ACDED017ABDF804606C
:100190005FED2B2A03EE106AF8EEC33AB8EE007A50
:1001A00063EEA14AB1EE004AB0EE476AA4EE846A5B
:1001B000B4EEE26AF1EE10FA40F2F8815FED356AD2
:1001C000B4EEE66AF1EE10FA40F2F1821FED387AF1
:1001D000B4EEC76AF1EE10FA40F2F9821FED3B0A65
:1001E000B4EEC06AF1EE10FA40F26E845FED3E5A52
:1001F000B4EEE56AF1EE10FA40F207845FED410AD1
:10020000B4EEE06AF1EE10FA40F276841FED441A83
:10021000B4EEC16AF1EE10FA40F287841FED472A6E
:10022000B4EEC26AF1EE10FA0DD876EE417A5FEDC7
:100230004A1AC7EEA12AB7EE003AF4EEC32AF1EE4D
:1002400010FA00F17B84F0EE003AB1E1002E73D099
:1002500092F8B8C092F8B940A44502D0D36B002BF5
:100260006AD192F800A00AF1FF36012E64D9117EFE
:1002700080F84C100127072580F84E70157608B0DD
:10028000BDE8F08790F82C40002C3FF476AD90F854
:100290003330002B7FF471ADD2F88430042B00F39F
:1002A000ED8203F11C0752F827406768002F80F2A7
:1002B000C58203F1010EBEF1050F39D003F11D080F
:1002C00052F828406768002F80F2B58203F1020ED1
:1002D000BEF1050F2CD003F11E0A52F82A406768C0
:1002E000002F80F2A88203F1030EBEF1050F1FD08C
:1002F0000EF11C0952F829406768002F80F29B829A
:1003000003F1040EBEF1050F12D003F1200C52F8D8
:100310002C406768002F80F28E820533052B07D0B2
:1003200003F11C0452F824406768002F80F2848295
:100330000023C2F8843020E5CB6BC46BB3EB040917
:100340003FF43BADD7688F4D566CDFF83CE2A5FB20
:100350000743DC0BA144B1458B4D91F82E300EFBC9
:100360001477B8BF29EAE97605FB0676D660002B3C
:100370003FF447AD24E5D2F8CC31D2F8D071013347
:1003800003F01F03BB423FF4CFACD2F8CCE102F143
:10039000CC0909EBCE0C0A2709F83E70CCF80440D2
:1003A000C2F8CC31C0E492F8008008F1FF37012F89
:1003B0003FF6B2ACD2F8CC31D2F8D071013303F0B1
:1003C0001F03BB423FF4A8ACD2F8CCE102F1CC0948
:1003D00009EBCE0A012709F83E70CAF80440C2F8BA
:1003E000CC3199E492F8008008F1FF34012C3FF6FB
:1003F00056AC90F82730002B3FF451AC92F8B890EF
:100400004FF07E5A89F0010482F8B840C2F8B4A0D7
:1004100045E490F83470002F7FF407AC92F800C0E8
:100420000CF1FF33012B7FF600AC92F888300133DA
:10043000022B40F39A802B46A846544CD2F8BC704D
:100440002468029448F2500E029C82F888804FF093
:100450007E59C2F8B49047F80E30C2F8C440FFF796
:10046000E4BB92F8009009F1FF33012B7FF6D5AB86
:1004700092F8B9A092F8B840A24503D0D56B002DF0
:100480007FF4CBAB1769576102231376FFF7C5BB27
:1004900015786E1E012E7FF6B8AB92F8B97092F8FF
:1004A000B880474503D0D36B002B7FF4AEAB146903
:1004B000546101251576FFF7A8BB0F3BACE4D2F8D9
:1004C000CC41D2F8D071013404F01F04BC423FF497
:1004D0002FAFD2F8CCE102F1CC0909EBCE0C022708
:1004E00009F83E70CCF80430C2F8CC4120E792F80D
:1004F00000A00AF1FF34012C7FF606AC92F8A77039
:1005000087F0010C82F8A7C0FFF7FEBB91F82F70AF
:10051000002F7FF4EEAC90F82F40002C3FF4E9ACB4
:1005200090F83660002E7FF4E4ACD51895F8897009
:10053000002F40F04382D2F8CC41D2F8D061013490
:1005400004F01F04A6420DD0D2F8CC6102F1CC0910
:1005500009EBC6084FF0060E09F836E0C8F804307B
:10056000C2F8CC4100255562C3E45FFA83F864E722
:1005700037EE871AF4EEC16AF1EE10FA00F340810B
:10058000436FC3E573B2E745C0D4010000AB02205E
:100590009A9999BD9A99993D01088039CDCC6C3FC3
:1005A000A470FD3FAE51013F00000000F0EE473A5D
:1005B0004F8C90ED250AD0ED264AD0ED245A90EDCF
:1005C000227AC2ED2A3A04EE107AB8EE446A35EE89
:1005D000C75A76EE406AA4EEA60AB4EEC50AF1EE5A
:1005E00010FA80ED250A40F19B8070EE075AD0F892
:1005F000A440C0ED245AC0F8A040002C40F3F58080
:10060000D0ED237A90ED211A77EEA72AB6EE003AC4
:10061000B7EE004A21EE030AF4EE442AF1EE10FA96
:1006200070EE474AC8BFF0EE442AA4EEA27A631ED9
:10063000C0F8A03080ED227A90ED1F7A90ED275A15
:10064000D0ED206A37EE016A75EEC60AF0EE475A21
:10065000E0EE855AF4EEE65AF1EE10FA08D5B4EE63
:10066000E57AF1EE10FA54BFF0EE476AF0EE656AF3
:10067000BCEEE62A5FED381A8DED012ABDF80400C4
:100680005FED3D2A07EE900AB8EEE73AB0EE004A79
:1006900023EE210ABFEE003AF0EE434AE0EE044AB0
:1006A000F4EEE24AF1EE10FA47D91FED467AF4EE85
:1006B000C74AF1EE10FA3DDB34EEC76A5FED490A36
:1006C000C6EE205AB7EE003AF4EEC35AF1EE10FA35
:1006D00000F1A680C98B1FED504A82ED2B3A02EE45
:1006E000901AF8EEE27AB0EE007A27EE840A70EE05
:1006F000004AE4EE833AF4EEC73AF1EE10FA0AD576
:10070000B8EE005AF4EEC53AF1EE10FAD4BFB0EEEE
:10071000457AB0EE637A82ED2C7A08B0BDE8F087B6
:1007200075EE870AB4EEE00AF1EE10FA6FDCD0F84D
:10073000A04062E71FED643ACCE7B7EE001A74EE12
:10074000816A1FED6A2AC6EE821AF4EEC11AF1EE32
:1007500010FAEFD5F5EEC01AF1EE10FABADD31EE6F
:10076000C13AB7E792F8008008F1FF34012C7FF618
:10077000ACAAD2F8CC31D2F8D071013303F01F0308
:10078000BB423FF4A2AAD2F8CC7102F1CC0909EB2A
:10079000C70E002409F837400127CEF80470C2F8CC
:1007A000CC31FFF792BA4FF0090EFFF756BA1FEDA2
:1007B000842A5FED841A76EE027AF7EE002A87EE3D
:1007C000A13AB4EEE23AF1EE10FA00F11381FFEE35
:1007D000003AEDE6D0ED161A90ED182A71EEC72A10
:1007E000A2EE227A80ED177AAEE490ED211A90ED18
:1007F000232A71EE471AA2EE217A80ED227A1BE7B6
:1008000076EEC77A836FC0ED197A43677EE470EEA7
:10081000475AD0F8A440C0ED245AC0F8A040ECE6F6
:100820001FED9F3AF4EEC35AF1EE10FA7FF752AF84
:1008300035EE833A4EE77346C2F88430D2F8CCE105
:10084000D2F8D0810EF1010A0AF01F0EC6450DD074
:10085000D2F8CC8102F1CC0C0CEBC8094FF0020AA3
:100860000CF838A0C9F80470C2F8CCE1B74F24687E
:100870003F6803970A34039F42F824700133042B26
:10088000C2F884307FF779AA52E5546E002CFFF647
:10089000D6ABD2F8CC61D2F8D051013606F01F03A6
:1008A0009D423FF4CCABD2F8CC6102F1CC0A0AEB0A
:1008B000C60C4FF0020E0AF836E0CCF80440C2F83D
:1008C000CC31FFF7BCBBD46D002CFFF690ABD2F857
:1008D000CC61D2F8D051013606F01F039D423FF49F
:1008E00086ABD2F8CC6102F1CC0909EBC6084FF017
:1008F000020E09F836E0C8F80440C2F8CC31FFF720
:1009000076BB546D002CFFF64AABD2F8CC61D2F81E
:10091000D051013606F01F039D423FF440ABD2F8A0
:10092000CC6102F1CC0A0AEBC60C4FF0020E0AF8B9
:1009300036E0CCF80440C2F8CC31FFF730BBD46CC1
:10094000002CFFF604ABD2F8CC61D2F8D0510136BE
:1009500006F01F03AB423FF4FAAAD2F8CC6102F1D1
:10096000CC0909EBC6084FF0020E09F836E0C8F8CA
:100970000440C2F8CC31FFF7EABAD46E002CFFF67F
:1009800086ABD2F8CC61D2F8D051013606F01F0305
:10099000AB423FF47CABD2F8CC6102F1CC0909EB5D
:1009A000C6084FF0020E09F836E0C8F80440C2F855
:1009B000CC31FFF76CBB3F01FFF7F0B9D2F8CC7137
:1009C000D2F8D051013707F01F04A5420DD0D2F85C
:1009D000CC6102F1CC0C0CEBC60A4FF0070E0CF800
:1009E00036E0CAF80430C2F8CC41584B1F6805976E
:1009F000059DB8E5B5EEC03AF1EE10FA7FF7D6AD39
:100A0000F0EE003A73EE633AD2E5DFED513ACFE50E
:100A1000002E00F090801769002FC0F2898007EB4C
:100A200087094B4406EB83084FF0FF36C8F84C614A
:100A300002F1600ACEF84C6002F16803C2F88450FB
:100A40000124012C3BD05E689D687768D5F804E0EE
:100A5000BE4532DA022C9E605D6030D0D3F8008053
:100A6000D8F80460764528DDE71E002F83E82001D2
:100A700023DDDAF804607768BE451EDA052C1E60B7
:100A8000CAF804501BD1DAF800406368734503DDEF
:100A9000CCF87440CAF800502C4D2E680696069F7C
:100AA000CCF8C870FFF725BA052C3FF41CAA013416
:100AB0000AF1040A0433FFF7E4B9052CECD0013441
:100AC0000AF1040A0433BCE79FED220ADFED226A33
:100AD00076EE000AF7EE005A80EEA61AB4EEE51A9A
:100AE000F1EE10FA91D5B5EEC01AF1EE10FA7FF7DB
:100AF0006EAE71EE653A5BE576EE654A9FED176A7C
:100B000084EE865AB7EE007AB4EEC75AF1EE10FAC8
:100B10007FF54CAD9FED0E7AB4EEC75AF1EE10FAA8
:100B20007FF744AD75EE073A42E5F7EE003A3FE550
:100B30000B48FEF7B1FF0B48FEF7AEFFF5EEC02AFB
:100B4000F1EE10FAF1DD72EE833A31E500AB0220EE
:100B500000000000332EA33F2431923F3CB1933F6D
:100B6000E0C50100D0C501002DE9F04F00F50335C7
:100B700005F1F80999F84D3085B090460F46002BE5
:100B800040F0218100F5023404F5497A9AF81860A2
:100B9000072E4DD8DFE816F0A7010800B301F201D7
:100BA0004C004C004C006E0191F82A60EEB999F8A7
:100BB0002A00D0B1D4F8F034D4F8F414013303F09F
:100BC0001F028A4204F57C7C0CD0D4F8F034DAF8A9
:100BD00014600CEBC30B03200CF83300CBF804605B
:100BE000C4F8F02400218AF8181097F825202AB9B3
:100BF00099F8253013B103268AF81860DAF8100046
:100C0000002804DB97F82E60002E00F0E68194F8AF
:100C10003C63D5F83451FA6B531B09D0DAF8140051
:100C200003444E2BD4BF23EAE3734F23CAF8143096
:100C300039464846492203F01FFF66B13C22002195
:100C4000404607F065FA0027C8F83C70C8F84470C1
:100C500005B0BDE8F08FC04F94F8AD6394F8AE5383
:100C600094F8AF03396894F8B03394F8B123019144
:100C7000C8F8006094F8B51394F8B263C8F804504B
:100C800094F8B353C8F8080094F8B403C8F80C30CB
:100C9000C8F8102094F8B63394F8BB23C8F8146051
:100CA00094F8B763C8F8185094F8B853C8F81C0003
:100CB00094F8B903C8F8201094F8BA13C8F834109F
:100CC000C8F82860C8F82C50C8F83000C8F824309C
:100CD000C8F83820019BD4F8486340F2DB55981BD4
:100CE000A84207D8D4F8441358F8212042F004034E
:100CF00048F821303E680396039DD4F84C03291A26
:100D0000B1F5C87F58D33E680396039DD4F85003CD
:100D1000291AB1F5C87F05D2D8F8042042F024037F
:100D2000C8F804303E680396039DD4F85403291A8A
:100D3000B1F5C87F05D2D8F8082042F02403C8F8DE
:100D400008303E680396039DD4F85803291AB1F57C
:100D5000C87F05D2D8F80C2042F02403C8F80C3024
:100D60003F680397039ED4F85C53701BB0F5C87FAF
:100D700005D2D8F8101041F02402C8F8102094F8D9
:100D8000DC9394F8DD3394F8CB7394F824439945BD
:100D90000CBF01260226C8F83C60002F64D0142145
:100DA000A4F10104B4FA84F25309C8F84030C8F839
:100DB000441005B0BDE8F08FD8F8002042F02403BD
:100DC000C8F800309FE74C8C0F8CDFED646A644EEE
:100DD000DFF89CE1DFF89CB1DFF89CA1C5F8506119
:100DE00007EE904A07EE107AF8EE670AB8EE470A67
:100DF000002719234FF07C5C00F50234C5F85461DC
:100E0000C5F87C61C5F88061C5F86C71C5F87031B2
:100E1000C5ED526AC5F84CB1C5F858A185ED570A21
:100E200085ED580AC5F864C1C5F868E14922C5F8DE
:100E30009C31C5F898714846C5ED5D6AC5F878B132
:100E4000C5F884A1C5F890C1C5F894E1C5ED620A62
:100E5000C5ED630A03F010FE94F83C6389F84D7009
:100E6000002E3FF4F8AEE9E6A4F10205B5FA85F0EC
:100E7000410995E791F82D0048B999F82D2032B134
:100E800099F84E10002900F0F88089F84E00354E90
:100E9000326812F0010A00F0BE8097F82E503248F6
:100EA000324925B190F82E30002B00F09E80D1F809
:100EB000F431806BBE6B012BA6EB000200F0BA8010
:100EC000022B00F0BF80002B00F09D8039464922A4
:100ED000254803F0D1FD39464846492294F83C6341
:100EE00003F0CAFDA9E652464846FEF783FE39469E
:100EF0004846492294F83C6303F0BEFD9DE691F814
:100F00002B30D3B999F82B20BAB1D4F8F004D4F827
:100F1000F414013000F01F038B4204F57C7B0CD0ED
:100F2000D4F8F024DAF814E00BEBC20004210BF83B
:100F30003210C0F804E0C4F8F03497F82E30002BDB
:100F40007FF467AE99F82E20002A3FF462AE8AF84B
:100F500018301E465DE600BF00AB02200000000016
:100F600000001442F068FF1FF468FF1F2CA6022047
:100F70000B5B823F00F07F45CDCC4C3D91F82520A6
:100F800091F82E30EAB995F81D11D1B1D4F8F0647A
:100F9000D4F8F404013606F01F02824204F57C7B8B
:100FA0000CD0D4F8F014DAF814E00BEBC1060520ED
:100FB0000BF83100C6F804E0C4F8F02401268AF8E2
:100FC0001860002B7FF434AE95F82651002D3FF4C5
:100FD0002FAE8AF818301E462AE699F82E100029FE
:100FE0003FF415AE8AF8186013E6D1F8F4212E4EBE
:100FF000013286FB025CACEBE27E0EEB4E05531B2E
:10100000C1F8F43155E7D1F8F8110D68154405F031
:1010100001030B605AE7304603F00EFE00283FF450
:101020003CAF51464C22214807F072F8304603F09D
:1010300009FE32E7D1F8F8114B68134403F00100C0
:10104000486043E7D1F8F811194ECB681A440E2ACC
:10105000D4BF22EAE2730F23581C06F1FF3B154A66
:1010600016F830A01BF830C082F8E1AD012582F8F7
:10107000E0CD82F8E25DCB6028E7DAF8C06086B1A7
:101080000D4D0E4906F5F260502203F0F5FC2B6879
:10109000029399F84CB00298CAF8C8008AF818B0C0
:1010A000F5E60748FEF7F8FC56555555F468FF1F5E
:1010B00029A802202C7A002000AB0220347A0020DC
:1010C000D0C501000FB410B582B004AB074C53F883
:1010D000042B01934021204607F03AF92046FEF701
:1010E0003DFA02B0BDE8104004B0704778790020A6
:1010F00007EE903A9FEDC90ADFEDC96ADFEDC95AE4
:10110000B8EEE76A2DE9F04F66EE000AC64CDFF84C
:10111000248320EEA61A84FB0346FDEEC11ADF17D6
:1011200011EE905AC5EB0514C7EBE619A60007EEC1
:10113000106A4FF4FA67B8EEC72A07FB19332DED92
:10114000028B96EE262A174687B008EE103AF8EE84
:10115000C82AFDEEC23A22EEA53A0C46064611EE2A
:10116000901AB248C8F800604FEA4709C8F804402E
:10117000C8F83020CDED013AFDEEC38AFFF7A2FF9B
:1011800009EB070007EB800104EB09020E44BD19CF
:1011900007EB020A0AF1FF346B1E049202940593D6
:1011A00000F1E881002CC0F2EC817F2E00F3C981B0
:1011B0003F2A60DC7F2B194626EAE67EA8BF7F2106
:1011C0003F2CA346A8BF4FF03F0B8E4522EAE27C9E
:1011D00051DC974A039615680CEB8E1405EB8400DE
:1011E0004B1C021F0BF1010401211E46E3453BDBB2
:1011F0006FEA0C050CF101002544A042516005F096
:10120000070502F104032FD015B3012D1BD0022DC9
:1012100016D0032D11D0042D0CD0052D07D0062D8E
:101220001CBF43F8041F013043F8041F013043F88A
:10123000041F013043F8041F013043F8041F01303C
:1012400043F8041F01300130A04243F8041F0BD0C3
:101250000830A04259609960D9601961596199615B
:10126000D96143F8201FF3D10EF1010EB64502F506
:101270008072BBD1039E09EB0A0B07EB0B00451EE6
:10128000039500F16481BBF13F0F5DDC059B039981
:101290007F2BA8BF7F2326EAE67E3F29A8BF3F21F8
:1012A0009E452BEAEB7C8A464EDC614A14680CEBC7
:1012B0008E1504EB8500051F03F10109481C01226E
:1012C000D4453BDC6FEA0C030CF10101034481427D
:1012D00003F007046A6005F104032FD014B3012C56
:1012E0001BD0022C16D0032C11D0042C0CD0052CB2
:1012F00007D0062C1CBF43F8042F013143F8042FFC
:10130000013143F8042F013143F8042F013143F830
:10131000042F013143F8042F01310131814243F898
:10132000042F0BD0083181425A609A60DA601A614A
:101330005A619A61DA6143F8202FF3D10EF1010E60
:10134000CE4505F58075BBD1C7EBC701D8F8003095
:1013500036484C00264423440199C8F800303744ED
:10136000FFF7B0FE013F019700F1DC80029A002AEE
:10137000C0F226817F2E00F3D58004983F286DDCD3
:10138000019D02997F2DA8BF7F2526EAE67E3F2991
:10139000A8BF3F21AE4520EAE07C8A465EDC244BB4
:1013A0001A680CEB8E1702EB8700071F05F1010985
:1013B000481C0122E2454BDB6FEA0C050CF10101F0
:1013C000054481427A6005F0070507F104033FD028
:1013D00095B3012D1BD0022D16D0032D11D0042D55
:1013E0000CD0052D07D0062D1CBF43F8042F01316A
:1013F00043F8042F013143F8042F013143F8042F3F
:10140000013143F8042F013143F8042F0131013138
:10141000814243F8042F1BD00EE000BF8988883C2E
:101420006F12033ACDCC4C3DD34D621088C60100FB
:10143000ACA80220B8790020083181425A609A6035
:10144000DA601A615A619A61DA6143F8202FF3D1A8
:101450000EF1010ECE4507F58077ABD10399002937
:1014600060DBBBF13F0F5DDC019B039A7F2BA8BFC4
:101470007F2326EAE6763F2AA8BF3F229E422BEA38
:10148000EB7994464EDC574F396809EB861501EB32
:10149000850B5F1CABF104020CF1010A0120E14550
:1014A0003BDCCAEB090309F10101DD438A455060C9
:1014B00005F0070502F104032FD015B3012D1BD051
:1014C000022D16D0032D11D0042D0CD0052D07D0E0
:1014D000062D1CBF43F8040F013143F8040F0131FE
:1014E00043F8040F013143F8040F013143F8040FAE
:1014F000013143F8040F013101318A4543F8040FEB
:101500000BD008318A4558609860D86018615861DE
:101510009861D86143F8200FF3D10136B74202F544
:101520008072BCD1D8F800502F48254418EE901A8C
:10153000C8F80050FFF7C6FD07B0BDEC028BBDE850
:10154000F08F09EB0A0B07EB0B03591E0391C7EB56
:10155000C702D8F800502448019954002644254475
:101560003744C8F80050FFF7ADFD013F01977FF504
:1015700001AFD7E709EB0A0B07EB0B00451E0395FC
:10158000E2E609EB0A0B07EB0B04601E03901BD489
:101590007F2E7FF778AEC7EBC701D8F8003012482E
:1015A0004C00264423440199C8F800303744FFF723
:1015B00089FD013F0197B5D47F2E7FF752AFB1E788
:1015C000039D002DF8DAADE7D8F800200648019910
:1015D000C7EBC70674002244C8F80020FFF772FD6D
:1015E000A0E700BFACA8022088C60100D0F8803078
:1015F000196891F8641001B1704730B5044611487C
:1016000083B04FF40042006806F082FD0E4A0F4B93
:1016100015680195019A1E25142003211D6058604C
:101620001963D30505D4D4F88000F7F7BDFA03B0E9
:1016300030BD0748FFF746FDD4F88000F7F7B4FA4D
:1016400003B030BDACA8022000AB0220B879002066
:1016500090C601002DE9F04F2DED048B83B00123DE
:1016600001916949684E0B601D224A600B63202579
:10167000FDF774FF65483560DFED659ADFED658A3B
:101680009FED659A604DFDF769FF02274FF0000856
:1016900007E008F10108B8F1070F07F1090700F0AA
:1016A000AB8001984269D11E41444F29F1D8D0F84E
:1016B000C04001EB810A04EB8A0C04EB810BDCF8DF
:1016C0004C61DBF80CB0002E0CF5A67E00F399807F
:1016D000DEF80430002B00F39480DEF808000028C8
:1016E00000F38F80DEF80C20002A00F38A80DEF8F9
:1016F0001040002CD4BF002401240094424A4748E3
:1017000025230131012682E888001663FFF7DAFC01
:101710003D4B434831211960FDF720FFBBF1000F1D
:10172000B7D007EE90BAB8EEE78A3E2228EE290A33
:101730003A482A6060EE280A6F60BDEEE01A2E6318
:1017400011EE10AA11EE101AFFF7BCFCCAEB0A103A
:10175000840001EE904AB8EEE12ADFF8D0A02B68B1
:10176000DAF800102D4898EE282A01F5964CBA1C9C
:101770007C1DFDEEC22A4CF822600E3312EE901A48
:101780004CF8246091462B60FFF79CFC25484FEAFB
:10179000EB7180FB0B32C1EBE2134FF4FA6C0CFBE4
:1017A00013B203EE102AF8EEC33ADAF800102B68F1
:1017B0001A4823EE894A01F5B24BFDEEC44A4BF8B4
:1017C00029600E334BF8246014EE901A2B60FFF75B
:1017D00079FC009C002C3FF45CAF6D2212486F60D6
:1017E00008F101082E632A60FDF7B8FEB8F1070F73
:1017F00007F109077FF455AF03B0BDEC048BBDE8DA
:10180000F08F0126009679E7B879002094C6010090
:101810008988883C6F12033ACDCC4C3D88C60100C4
:1018200098C60100D34D62109CC60100ACA80220EE
:101830002DE9F043704B1C6883B0582206460D46D4
:1018400004F55070002106F063FC5822002104F5D5
:10185000886006F05DFC04F5A8605822002106F0BF
:1018600057FC04F5FC4808F1400804F5C867582205
:101870000021384607F5807906F04AFC58220021FD
:10188000484606F045FC07F500705822002106F096
:101890003FFC5822002107F5407006F039FC582221
:1018A000002107F5806006F033FC5822002107F57F
:1018B000A06006F02DFC5822002107F5C06006F05C
:1018C00027FC07F5E0605822002107F5006706F0C5
:1018D0001FFCB845CBD104F50E7004F5267101222A
:1018E00042608260C260026142618261C26140F80E
:1018F000202F8142F4D10123C4F83C3204F5FA4090
:10190000C4F83C33C4F83C3404F5A06CC4F83C354E
:10191000C4F83C36CCF83C37CCF83C38CCF83C39F1
:10192000CCF83C32CCF83C33CCF83C34CCF83C35E9
:10193000CCF83C360CF5006C8445EBD104F5FC4743
:1019400004F5FD413837183101227A60BA60FA6037
:101950003A617A61BA61FA6147F8202FB942F4D14D
:10196000031B04F5807EA3F5807701228645C7F32B
:101970000221C4F8982243D049B3012921D0022979
:101980001BD0032915D004290FD0052909D0062919
:101990001CBFCEF898220EF5807E0EF5807ECEF824
:1019A0009821CEF898220EF5807ECEF898220EF57A
:1019B000807ECEF898220EF5807ECEF898220EF525
:1019C000807ECEF898220EF5807E864518D0CEF81F
:1019D0009827CEF89828CEF89829CEF89822CEF8F5
:1019E0009823CEF89824CEF89825CEF898260EF5B0
:1019F000006E8645EBD103E0ACA802200000F8425F
:101A000004F580790023C4F89C33C4F8A033C4F8EB
:101A1000A433C4F8A833C4F8AC33C4F8B033C4F862
:101A2000B433C4F8B83304F5F648C9F89C33C9F8A0
:101A3000A033C9F8A433C9F8A833C9F8AC33C9F83E
:101A4000B033C9F8B433C9F8B833C9F89C34C9F80D
:101A5000A034C9F8A434C9F8A834C9F8AC34C9F81A
:101A6000B034C9F8B434C9F8B83404F54072C2F8D7
:101A70009C33C2F8A033C2F8A433C2F8A833C2F82A
:101A8000AC33C2F8B033C2F8B433C2F8B83302F59D
:101A9000807C02F5407E02F5806702F5A06102F5C8
:101AA000C0624245CCF89C33CCF8A033CCF8A433C8
:101AB000CCF8A833CCF8AC33CCF8B033CCF8B43392
:101AC000CCF8B833CCF89C34CCF8A034CCF8A4349F
:101AD000CCF8A834CCF8AC34CCF8B034CCF8B4346E
:101AE000CCF8B834CEF89C33CEF8A033CEF8A4337B
:101AF000CEF8A833CEF8AC33CEF8B033CEF8B4334A
:101B0000CEF8B833C7F89C33C7F8A033C7F8A4336E
:101B1000C7F8A833C7F8AC33C7F8B033C7F8B43345
:101B2000C7F8B833C1F89C33C1F8A033C1F8A43367
:101B3000C1F8A833C1F8AC33C1F8B033C1F8B4333D
:101B4000C1F8B83393D1031B04F580780127A3F5BE
:101B5000807980453A46C4F89C72C4F8A072C4F8F3
:101B6000A472C4F8A872C4F8AC72C4F8B072C4F815
:101B7000B472C4F8B872C4F8BC72C4F89872C9F3ED
:101B8000022142D059B3012921D002291BD00329B7
:101B900015D004290FD0052909D006291CBFC8F883
:101BA000987208F5807808F58078C8F89871C8F8B8
:101BB000982208F58078C8F8982208F58078C8F847
:101BC000982208F58078C8F8982208F58078C8F837
:101BD000982208F5807880454FF0010715D0C8F8A5
:101BE0009827C8F89828C8F89829C8F89822C8F8FB
:101BF0009823C8F89824C8F89825C8F8982608F5B6
:101C0000006880454FF00107E9D104F5FC4C031B47
